LX51 LINKER/LOCATER V4.64.0.0                                                           04/13/2020  14:54:03  PAGE 1


LX51 LINKER/LOCATER V4.64.0.0, INVOKED BY:
C:\KEIL\C51\BIN\LX51.EXE .\hex\main.obj, .\hex\delay.obj, .\hex\system_clock.obj, .\hex\uart.obj, .\hex\interrupt.obj, .
>> \hex\debug.obj, .\hex\ts_api.obj, .\TS_Lib\Sources\ts_sevice.LIB, .\hex\STARTUP.obj TO .\hex\ca51f2 PRINT (.\lst\ca51
>> f2.map) REMOVEUNUSED CLASSES (XDATA (X:0X0-X:0XFFF), HDATA (X:0X0-X:0XFFF), CODE (C:0X0-C:0X3FFF), CONST (C:0X0-C:0X3
>> FFF), ECODE (C:0X0-C:0X3FFF), HCONST (C:0X0-C:0X3FFF))


CPU MODE:     8051 MODE
MEMORY MODEL: SMALL


INPUT MODULES INCLUDED:
  .\hex\main.obj (MAIN)
         COMMENT TYPE 0: C51 V9.51
  .\hex\delay.obj (DELAY)
         COMMENT TYPE 0: C51 V9.51
  .\hex\system_clock.obj (SYSTEM_CLOCK)
         COMMENT TYPE 0: C51 V9.51
  .\hex\uart.obj (UART)
         COMMENT TYPE 0: C51 V9.51
  .\hex\interrupt.obj (INTERRUPT)
         COMMENT TYPE 0: C51 V9.51
  .\hex\debug.obj (DEBUG)
         COMMENT TYPE 0: C51 V9.51
  .\hex\ts_api.obj (TS_API)
         COMMENT TYPE 0: C51 V9.51
  .\TS_Lib\Sources\ts_sevice.LIB (TS_SEVICE)
         COMMENT TYPE 0: C51 V9.51
  .\hex\STARTUP.obj (?C_STARTUP)
         COMMENT TYPE 1: A51 / ASM51 Assembler
  C:\KEIL\C51\LIB\C51S.LIB (?C_INIT)
         COMMENT TYPE 1: A51 / ASM51 Assembler
  C:\KEIL\C51\LIB\C51S.LIB (?C?CLDOPTR)
         COMMENT TYPE 1: A51 / ASM51 Assembler
  C:\KEIL\C51\LIB\C51S.LIB (?C?CSTPTR)
         COMMENT TYPE 1: A51 / ASM51 Assembler
  C:\KEIL\C51\LIB\C51S.LIB (?C?CSTOPTR)
         COMMENT TYPE 1: A51 / ASM51 Assembler
  C:\KEIL\C51\LIB\C51S.LIB (?C?IMUL)
         COMMENT TYPE 1: A51 / ASM51 Assembler
  C:\KEIL\C51\LIB\C51S.LIB (?C?UIDIV)
         COMMENT TYPE 1: A51 / ASM51 Assembler
  C:\KEIL\C51\LIB\C51S.LIB (?C?SIDIV)
         COMMENT TYPE 1: A51 / ASM51 Assembler
  C:\KEIL\C51\LIB\C51S.LIB (?C?IILDX)
         COMMENT TYPE 1: A51 / ASM51 Assembler
  C:\KEIL\C51\LIB\C51S.LIB (?C?ULDIV)
         COMMENT TYPE 1: A51 / ASM51 Assembler
  C:\KEIL\C51\LIB\C51S.LIB (?C?LSTXDATA)
         COMMENT TYPE 1: A51 / ASM51 Assembler
  C:\KEIL\C51\LIB\C51S.LIB (?C?OFFXADD)
         COMMENT TYPE 1: A51 / ASM51 Assembler
  C:\KEIL\C51\LIB\C51S.LIB (?C?PLDCODE)
         COMMENT TYPE 1: A51 / ASM51 Assembler
  C:\KEIL\C51\LIB\C51S.LIB (?C?LIMUL)
         COMMENT TYPE 1: A51 / ASM51 Assembler


ACTIVE MEMORY CLASSES OF MODULE:  .\hex\ca51f2 (MAIN)

BASE        START       END         USED      MEMORY CLASS
==========================================================
X:000000H   X:000000H   X:000FFFH   00018DH   XDATA
X:000000H   X:000000H   X:000FFFH             HDATA
C:000000H   C:000000H   C:003FFFH   000CA4H   CODE
C:000000H   C:000000H   C:003FFFH   0000A2H   CONST
LX51 LINKER/LOCATER V4.64.0.0                                                         04/13/2020  14:54:03  PAGE 2


C:000000H   C:000000H   C:003FFFH             ECODE
B00:0000H   C:000000H   C:003FFFH             HCONST
I:000000H   I:000000H   I:00007FH   00002DH   DATA
I:000020H.0 I:000020H.0 I:00002FH.7 000000H.5 BIT
I:000000H   I:000000H   I:0000FFH   00000BH   IDATA


MEMORY MAP OF MODULE:  .\hex\ca51f2 (MAIN)


START     STOP      LENGTH    ALIGN  RELOC    MEMORY CLASS   SEGMENT NAME
=========================================================================

* * * * * * * * * * *   D A T A   M E M O R Y   * * * * * * * * * * * * *
000000H   000007H   000008H   ---    AT..     DATA           "REG BANK 0"
000008H   00001BH   000014H   BYTE   UNIT     DATA           _DATA_GROUP_
00001CH.0 00001FH.7 000004H.0 ---    ---      **GAP**
000020H.0 000020H.2 000000H.3 BIT    UNIT     BIT            ?BI?TS_API
000020H.3 000020H.3 000000H.1 BIT    UNIT     BIT            ?BI?DEBUG
000020H.4 000020H.4 000000H.1 BIT    UNIT     BIT            _BIT_GROUP_
000020H.5 000020H   000000H.3 ---    ---      **GAP**
000021H   00002CH   00000CH   BYTE   UNIT     DATA           ?DT?TS_API
00002DH   000031H   000005H   BYTE   UNIT     DATA           ?DT?DEBUG
000032H   00003BH   00000AH   BYTE   UNIT     IDATA          ?ID?TS_API
00003CH   00003CH   000001H   BYTE   UNIT     IDATA          ?STACK

* * * * * * * * * * *   C O D E   M E M O R Y   * * * * * * * * * * * * *
000000H   000002H   000003H   ---    OFFS..   CODE           ?CO??C_STARTUP?0
000003H   000042H   000040H   BYTE   INBLOCK  CODE           ?PR?INT6_ISR?INTERRUPT
000043H   000045H   000003H   BYTE   OFFS..   CODE           ?INTERRUPT?00043
000046H   00005AH   000015H   BYTE   INBLOCK  CODE           ?PR?MAIN?MAIN
00005BH   00005DH   000003H   BYTE   OFFS..   CODE           ?INTERRUPT?0005B
00005EH   000067H   00000AH   BYTE   INBLOCK  CODE           ?PR?DEBUG
000068H   00006AH   000003H   ---    ---      **GAP**
00006BH   00006DH   000003H   BYTE   OFFS..   CODE           ?INTERRUPT?0006B
00006EH   00018EH   000121H   BYTE   INBLOCK  CODE           ?PR?TS_SEVICE
00018FH   000290H   000102H   BYTE   INBLOCK  CODE           ?PR?TSKEY_DATADEAL?TS_API
000291H   000356H   0000C6H   BYTE   INBLOCK  CODE           ?PR?TS_RUNINIT?TS_API
000357H   000410H   0000BAH   BYTE   INBLOCK  CODE           ?PR?TS_DATAFILTERING?TS_API
000411H   0004C3H   0000B3H   BYTE   INBLOCK  CODE           ?PR?TS_API
0004C4H   000571H   0000AEH   BYTE   INBLOCK  CODE           ?PR?TS_ISR?TS_API
000572H   0005FCH   00008BH   BYTE   INBLOCK  CODE           ?PR?TS_GETKEY?TS_API
0005FDH   00066FH   000073H   BYTE   INBLOCK  CODE           ?PR?I2C_ISR?DEBUG
000670H   0006D9H   00006AH   BYTE   INBLOCK  CODE           ?PR?TS_INIT?TS_API
0006DAH   000738H   00005FH   BYTE   INBLOCK  CODE           ?PR?_TS_GETDATAAREA?TS_SEVICE
000739H   000794H   00005CH   BYTE   INBLOCK  CODE           ?PR?INT8_ISR?INTERRUPT
000795H   0007E7H   000053H   BYTE   INBLOCK  CODE           ?PR?DEBUG_PARAMLOAD?DEBUG
0007E8H   0007FAH   000013H   BYTE   INBLOCK  CODE           ?PR?_TS_AREACONFIRMTIMERSET?TS_SEVICE
0007FBH   0007FFH   000005H   ---    ---      **GAP**
000800H   000849H   00004AH   BYTE   INBLOCK  CODE           ?PR?TS_SCANSTART?TS_SEVICE
00084AH   000888H   00003FH   BYTE   INBLOCK  CODE           ?PR?INT3_ISR?INTERRUPT
000889H   0008C1H   000039H   BYTE   INBLOCK  CODE           ?PR?TS_ACTION?TS_API
0008C2H   0008F0H   00002FH   BYTE   INBLOCK  CODE           ?PR?TS_IO_INIT?TS_SEVICE
0008F1H   00091EH   00002EH   BYTE   INBLOCK  CODE           ?PR?TS_MS_ISR?TS_API
00091FH   00094CH   00002EH   BYTE   INBLOCK  CODE           ?PR?_TS_AREADEVIATEDETECTION?TS_SEVICE
00094DH   000979H   00002DH   BYTE   INBLOCK  CODE           ?PR?TS_HS_ISR?TS_API
00097AH   00099DH   000024H   BYTE   INBLOCK  CODE           ?PR?_SYS_CLK_SET_PLL?SYSTEM_CLOCK
00099EH   0009BCH   00001FH   BYTE   INBLOCK  CODE           ?PR?DEBUG_INIT?DEBUG
0009BDH   0009D8H   00001CH   BYTE   INBLOCK  CODE           ?PR?SYSTEMINIT?MAIN
0009D9H   0009E0H   000008H   BYTE   INBLOCK  CODE           ?PR?SYSTEM_CLOCK
0009E1H   000C13H   000233H   BYTE   UNIT     CODE           ?C?LIB_CODE
000C14H   000C9FH   00008CH   BYTE   UNIT     CODE           ?C_C51STARTUP
000CA0H   000CABH   00000CH   BYTE   UNIT     CODE           ?C_INITSEG
000CACH   000CF3H   000048H   BYTE   UNIT     CONST          ?CO?TS_SEVICE
000CF4H   000D2FH   00003CH   BYTE   UNIT     CONST          ?CO?TS_API
LX51 LINKER/LOCATER V4.64.0.0                                                         04/13/2020  14:54:03  PAGE 3


000D30H   000D4DH   00001EH   BYTE   UNIT     CONST          ?CO?DEBUG

* * * * * * * * * * *  X D A T A   M E M O R Y  * * * * * * * * * * * * *
000000H   0000B1H   0000B2H   BYTE   UNIT     XDATA          ?XD?TS_API
0000B2H   0000B2H   000001H   BYTE   UNIT     XDATA          ?XD?DEBUG
0000B3H   007FFFH   007F4DH   ---    ---      **GAP**
008000H   008000H   000001H   BYTE   OFFS..   XDATA          ?XD?MAIN?132
008001H   008001H   000001H   BYTE   OFFS..   XDATA          ?XD?MAIN?140
008002H   008002H   000001H   BYTE   OFFS..   XDATA          ?XD?MAIN?149
008003H   008003H   000001H   BYTE   OFFS..   XDATA          ?XD?MAIN?161
008004H   008004H   000001H   BYTE   OFFS..   XDATA          ?XD?MAIN?176
008005H   008005H   000001H   BYTE   OFFS..   XDATA          ?XD?MAIN?190
008006H   008006H   000001H   BYTE   OFFS..   XDATA          ?XD?MAIN?204
008007H   008007H   000001H   BYTE   OFFS..   XDATA          ?XD?MAIN?217
008008H   008008H   000001H   BYTE   OFFS..   XDATA          ?XD?MAIN?139
008009H   008009H   000001H   BYTE   OFFS..   XDATA          ?XD?MAIN?148
00800AH   00800AH   000001H   BYTE   OFFS..   XDATA          ?XD?MAIN?160
00800BH   00800BH   000001H   BYTE   OFFS..   XDATA          ?XD?MAIN?175
00800CH   00800CH   000001H   BYTE   OFFS..   XDATA          ?XD?MAIN?189
00800DH   00800DH   000001H   BYTE   OFFS..   XDATA          ?XD?MAIN?203
00800EH   00800EH   000001H   BYTE   OFFS..   XDATA          ?XD?MAIN?216
00800FH   00800FH   000001H   BYTE   OFFS..   XDATA          ?XD?MAIN?11
008010H   008010H   000001H   BYTE   OFFS..   XDATA          ?XD?MAIN?147
008011H   008011H   000001H   BYTE   OFFS..   XDATA          ?XD?MAIN?159
008012H   008012H   000001H   BYTE   OFFS..   XDATA          ?XD?MAIN?174
008013H   008013H   000001H   BYTE   OFFS..   XDATA          ?XD?MAIN?188
008014H   008014H   000001H   BYTE   OFFS..   XDATA          ?XD?MAIN?202
008015H   008015H   000001H   BYTE   OFFS..   XDATA          ?XD?MAIN?215
008016H   008016H   000001H   BYTE   OFFS..   XDATA          ?XD?MAIN?10
008017H   008017H   000001H   BYTE   OFFS..   XDATA          ?XD?MAIN?20
008018H   008018H   000001H   BYTE   OFFS..   XDATA          ?XD?MAIN?158
008019H   008019H   000001H   BYTE   OFFS..   XDATA          ?XD?MAIN?173
00801AH   00801AH   000001H   BYTE   OFFS..   XDATA          ?XD?MAIN?187
00801BH   00801BH   000001H   BYTE   OFFS..   XDATA          ?XD?MAIN?201
00801CH   00801CH   000001H   BYTE   OFFS..   XDATA          ?XD?MAIN?214
00801DH   00801DH   000001H   BYTE   OFFS..   XDATA          ?XD?MAIN?9
00801EH   00801EH   000001H   BYTE   OFFS..   XDATA          ?XD?MAIN?19
00801FH   00801FH   000001H   BYTE   OFFS..   XDATA          ?XD?MAIN?27
008020H   008020H   000001H   BYTE   OFFS..   XDATA          ?XD?MAIN?172
008021H   008021H   000001H   BYTE   OFFS..   XDATA          ?XD?MAIN?186
008022H   008022H   000001H   BYTE   OFFS..   XDATA          ?XD?MAIN?200
008023H   008023H   000001H   BYTE   OFFS..   XDATA          ?XD?MAIN?213
008024H   008024H   000001H   BYTE   OFFS..   XDATA          ?XD?MAIN?8
008025H   008025H   000001H   BYTE   OFFS..   XDATA          ?XD?MAIN?18
008026H   008026H   000001H   BYTE   OFFS..   XDATA          ?XD?MAIN?26
008027H   008027H   000001H   BYTE   OFFS..   XDATA          ?XD?MAIN?34
008028H   008028H   000001H   BYTE   OFFS..   XDATA          ?XD?MAIN?185
008029H   008029H   000001H   BYTE   OFFS..   XDATA          ?XD?MAIN?199
00802AH   00802AH   000001H   BYTE   OFFS..   XDATA          ?XD?MAIN?212
00802BH   00802BH   000001H   BYTE   OFFS..   XDATA          ?XD?MAIN?7
00802CH   00802CH   000001H   BYTE   OFFS..   XDATA          ?XD?MAIN?17
00802DH   00802DH   000001H   BYTE   OFFS..   XDATA          ?XD?MAIN?25
00802EH   00802EH   000001H   BYTE   OFFS..   XDATA          ?XD?MAIN?33
00802FH   00802FH   000001H   BYTE   OFFS..   XDATA          ?XD?MAIN?38
008030H   008030H   000001H   BYTE   OFFS..   XDATA          ?XD?MAIN?198
008031H   008031H   000001H   BYTE   OFFS..   XDATA          ?XD?MAIN?211
008032H   008032H   000001H   BYTE   OFFS..   XDATA          ?XD?MAIN?6
008033H   008033H   000001H   BYTE   OFFS..   XDATA          ?XD?MAIN?16
008034H   008034H   000001H   BYTE   OFFS..   XDATA          ?XD?MAIN?24
008035H   008035H   000001H   BYTE   OFFS..   XDATA          ?XD?MAIN?32
008036H   008036H   000001H   BYTE   OFFS..   XDATA          ?XD?MAIN?37
008037H   008037H   000001H   BYTE   OFFS..   XDATA          ?XD?MAIN?39
008038H   008038H   000001H   BYTE   OFFS..   XDATA          ?XD?MAIN?210
008039H   008039H   000001H   BYTE   OFFS..   XDATA          ?XD?MAIN?5
00803AH   00803AH   000001H   BYTE   OFFS..   XDATA          ?XD?MAIN?15
LX51 LINKER/LOCATER V4.64.0.0                                                         04/13/2020  14:54:03  PAGE 4


00803BH   00803BH   000001H   BYTE   OFFS..   XDATA          ?XD?MAIN?23
00803CH   00803CH   000001H   BYTE   OFFS..   XDATA          ?XD?MAIN?31
00803DH   00803DH   000001H   BYTE   OFFS..   XDATA          ?XD?MAIN?36
00803EH   00803FH   000002H   ---    ---      **GAP**
008040H   008040H   000001H   BYTE   OFFS..   XDATA          ?XD?MAIN?74
008041H   008041H   000001H   BYTE   OFFS..   XDATA          ?XD?MAIN?77
008042H   008042H   000001H   BYTE   OFFS..   XDATA          ?XD?MAIN?103
008043H   008047H   000005H   ---    ---      **GAP**
008048H   008048H   000001H   BYTE   OFFS..   XDATA          ?XD?MAIN?57
008049H   008049H   000001H   BYTE   OFFS..   XDATA          ?XD?MAIN?58
00804AH   00804AH   000001H   BYTE   OFFS..   XDATA          ?XD?MAIN?59
00804BH   00804BH   000001H   BYTE   OFFS..   XDATA          ?XD?MAIN?60
00804CH   00804CH   000001H   BYTE   OFFS..   XDATA          ?XD?MAIN?127
00804DH   00804DH   000001H   BYTE   OFFS..   XDATA          ?XD?MAIN?197
00804EH   00804EH   000001H   BYTE   OFFS..   XDATA          ?XD?MAIN?30
00804FH   00804FH   000001H   ---    ---      **GAP**
008050H   008050H   000001H   BYTE   OFFS..   XDATA          ?XD?MAIN?108
008051H   008051H   000001H   BYTE   OFFS..   XDATA          ?XD?MAIN?104
008052H   008052H   000001H   BYTE   OFFS..   XDATA          ?XD?MAIN?110
008053H   008053H   000001H   BYTE   OFFS..   XDATA          ?XD?MAIN?105
008054H   008054H   000001H   BYTE   OFFS..   XDATA          ?XD?MAIN?112
008055H   008055H   000001H   BYTE   OFFS..   XDATA          ?XD?MAIN?106
008056H   008056H   000001H   BYTE   OFFS..   XDATA          ?XD?MAIN?114
008057H   008057H   000001H   BYTE   OFFS..   XDATA          ?XD?MAIN?107
008058H   008058H   000001H   BYTE   OFFS..   XDATA          ?XD?MAIN?81
008059H   008059H   000001H   BYTE   OFFS..   XDATA          ?XD?MAIN?56
00805AH   00805AH   000001H   BYTE   OFFS..   XDATA          ?XD?MAIN?54
00805BH   00805BH   000001H   BYTE   OFFS..   XDATA          ?XD?MAIN?48
00805CH   00805CH   000001H   BYTE   OFFS..   XDATA          ?XD?MAIN?47
00805DH   00805FH   000003H   ---    ---      **GAP**
008060H   008060H   000001H   BYTE   OFFS..   XDATA          ?XD?MAIN?88
008061H   008061H   000001H   BYTE   OFFS..   XDATA          ?XD?MAIN?73
008062H   008062H   000001H   BYTE   OFFS..   XDATA          ?XD?MAIN?83
008063H   008063H   000001H   BYTE   OFFS..   XDATA          ?XD?MAIN?76
008064H   008064H   000001H   BYTE   OFFS..   XDATA          ?XD?MAIN?79
008065H   008065H   000001H   BYTE   OFFS..   XDATA          ?XD?MAIN?80
008066H   008066H   000001H   BYTE   OFFS..   XDATA          ?XD?MAIN?157
008067H   008067H   000001H   BYTE   OFFS..   XDATA          ?XD?MAIN?22
008068H   008068H   000001H   BYTE   OFFS..   XDATA          ?XD?MAIN?90
008069H   008069H   000001H   BYTE   OFFS..   XDATA          ?XD?MAIN?92
00806AH   00806AH   000001H   BYTE   OFFS..   XDATA          ?XD?MAIN?93
00806BH   00806BH   000001H   BYTE   OFFS..   XDATA          ?XD?MAIN?94
00806CH   00806CH   000001H   BYTE   OFFS..   XDATA          ?XD?MAIN?95
00806DH   00806DH   000001H   BYTE   OFFS..   XDATA          ?XD?MAIN?96
00806EH   00806EH   000001H   BYTE   OFFS..   XDATA          ?XD?MAIN?97
00806FH   00806FH   000001H   BYTE   OFFS..   XDATA          ?XD?MAIN?98
008070H   008070H   000001H   BYTE   OFFS..   XDATA          ?XD?MAIN?100
008071H   008071H   000001H   BYTE   OFFS..   XDATA          ?XD?MAIN?101
008072H   008072H   000001H   BYTE   OFFS..   XDATA          ?XD?MAIN?41
008073H   008073H   000001H   BYTE   OFFS..   XDATA          ?XD?MAIN?42
008074H   008074H   000001H   BYTE   OFFS..   XDATA          ?XD?MAIN?87
008075H   008077H   000003H   ---    ---      **GAP**
008078H   008078H   000001H   BYTE   OFFS..   XDATA          ?XD?MAIN?29
008079H   008079H   000001H   BYTE   OFFS..   XDATA          ?XD?MAIN?44
00807AH   00807AH   000001H   BYTE   OFFS..   XDATA          ?XD?MAIN?40
00807BH   00807BH   000001H   BYTE   OFFS..   XDATA          ?XD?MAIN?82
00807CH   00807CH   000001H   BYTE   OFFS..   XDATA          ?XD?MAIN?75
00807DH   00807DH   000001H   BYTE   OFFS..   XDATA          ?XD?MAIN?102
00807EH   00807EH   000001H   BYTE   OFFS..   XDATA          ?XD?MAIN?99
00807FH   00807FH   000001H   ---    ---      **GAP**
008080H   008080H   000001H   BYTE   OFFS..   XDATA          ?XD?MAIN?116
008081H   008081H   000001H   BYTE   OFFS..   XDATA          ?XD?MAIN?121
008082H   008082H   000001H   BYTE   OFFS..   XDATA          ?XD?MAIN?117
008083H   008083H   000001H   BYTE   OFFS..   XDATA          ?XD?MAIN?68
008084H   008084H   000001H   BYTE   OFFS..   XDATA          ?XD?MAIN?64
LX51 LINKER/LOCATER V4.64.0.0                                                         04/13/2020  14:54:03  PAGE 5


008085H   008085H   000001H   BYTE   OFFS..   XDATA          ?XD?MAIN?70
008086H   008086H   000001H   BYTE   OFFS..   XDATA          ?XD?MAIN?67
008087H   008087H   000001H   BYTE   OFFS..   XDATA          ?XD?MAIN?109
008088H   008088H   000001H   BYTE   OFFS..   XDATA          ?XD?MAIN?55
008089H   008089H   000001H   BYTE   OFFS..   XDATA          ?XD?MAIN?52
00808AH   00808AH   000001H   BYTE   OFFS..   XDATA          ?XD?MAIN?69
00808BH   00808BH   000001H   BYTE   OFFS..   XDATA          ?XD?MAIN?66
00808CH   00808CH   000001H   BYTE   OFFS..   XDATA          ?XD?MAIN?65
00808DH   00808DH   000001H   BYTE   OFFS..   XDATA          ?XD?MAIN?62
00808EH   00808FH   000002H   ---    ---      **GAP**
008090H   008090H   000001H   BYTE   OFFS..   XDATA          ?XD?MAIN?86
008091H   008091H   000001H   BYTE   OFFS..   XDATA          ?XD?MAIN?85
008092H   008092H   000001H   BYTE   OFFS..   XDATA          ?XD?MAIN?184
008093H   008093H   000001H   BYTE   OFFS..   XDATA          ?XD?MAIN?138
008094H   0080FFH   00006CH   ---    ---      **GAP**
008100H   008100H   000001H   BYTE   OFFS..   XDATA          ?XD?MAIN?46
008101H   008101H   000001H   BYTE   OFFS..   XDATA          ?XD?MAIN?63
008102H   008102H   000001H   ---    ---      **GAP**
008103H   008103H   000001H   BYTE   OFFS..   XDATA          ?XD?MAIN?45
008104H   008105H   000002H   ---    ---      **GAP**
008106H   008106H   000001H   BYTE   OFFS..   XDATA          ?XD?MAIN?71
008107H   008107H   000001H   BYTE   OFFS..   XDATA          ?XD?MAIN?171
008108H   008108H   000001H   BYTE   OFFS..   XDATA          ?XD?MAIN?28
008109H   008109H   000001H   BYTE   OFFS..   XDATA          ?XD?MAIN?170
00810AH   00810AH   000001H   BYTE   OFFS..   XDATA          ?XD?MAIN?35
00810BH   00810BH   000001H   BYTE   OFFS..   XDATA          ?XD?MAIN?51
00810CH   00810CH   000001H   BYTE   OFFS..   XDATA          ?XD?MAIN?49
00810DH   00810DH   000001H   BYTE   OFFS..   XDATA          ?XD?MAIN?53
00810EH   00810EH   000001H   BYTE   OFFS..   XDATA          ?XD?MAIN?50
00810FH   00810FH   000001H   BYTE   OFFS..   XDATA          ?XD?MAIN?84
008110H   008110H   000001H   BYTE   OFFS..   XDATA          ?XD?MAIN?89
008111H   008116H   000006H   ---    ---      **GAP**
008117H   008117H   000001H   BYTE   OFFS..   XDATA          ?XD?MAIN?113
008118H   00811DH   000006H   ---    ---      **GAP**
00811EH   00811EH   000001H   BYTE   OFFS..   XDATA          ?XD?MAIN?4
00811FH   00811FH   000001H   BYTE   OFFS..   XDATA          ?XD?MAIN?43
008120H   008120H   000001H   BYTE   OFFS..   XDATA          ?XD?MAIN?120
008121H   008121H   000001H   BYTE   OFFS..   XDATA          ?XD?MAIN?123
008122H   008122H   000001H   BYTE   OFFS..   XDATA          ?XD?MAIN?126
008123H   008123H   000001H   BYTE   OFFS..   XDATA          ?XD?MAIN?131
008124H   008124H   000001H   BYTE   OFFS..   XDATA          ?XD?MAIN?137
008125H   008125H   000001H   BYTE   OFFS..   XDATA          ?XD?MAIN?146
008126H   008126H   000001H   BYTE   OFFS..   XDATA          ?XD?MAIN?156
008127H   008127H   000001H   BYTE   OFFS..   XDATA          ?XD?MAIN?169
008128H   008128H   000001H   BYTE   OFFS..   XDATA          ?XD?MAIN?122
008129H   008129H   000001H   BYTE   OFFS..   XDATA          ?XD?MAIN?125
00812AH   00812AH   000001H   BYTE   OFFS..   XDATA          ?XD?MAIN?130
00812BH   00812BH   000001H   BYTE   OFFS..   XDATA          ?XD?MAIN?136
00812CH   00812CH   000001H   BYTE   OFFS..   XDATA          ?XD?MAIN?145
00812DH   00812DH   000001H   BYTE   OFFS..   XDATA          ?XD?MAIN?155
00812EH   00812EH   000001H   BYTE   OFFS..   XDATA          ?XD?MAIN?168
00812FH   00812FH   000001H   BYTE   OFFS..   XDATA          ?XD?MAIN?183
008130H   008130H   000001H   BYTE   OFFS..   XDATA          ?XD?MAIN?124
008131H   008131H   000001H   BYTE   OFFS..   XDATA          ?XD?MAIN?129
008132H   008132H   000001H   BYTE   OFFS..   XDATA          ?XD?MAIN?135
008133H   008133H   000001H   BYTE   OFFS..   XDATA          ?XD?MAIN?144
008134H   008134H   000001H   BYTE   OFFS..   XDATA          ?XD?MAIN?154
008135H   008135H   000001H   BYTE   OFFS..   XDATA          ?XD?MAIN?167
008136H   008136H   000001H   BYTE   OFFS..   XDATA          ?XD?MAIN?182
008137H   008137H   000001H   BYTE   OFFS..   XDATA          ?XD?MAIN?196
008138H   008138H   000001H   BYTE   OFFS..   XDATA          ?XD?MAIN?128
008139H   008139H   000001H   BYTE   OFFS..   XDATA          ?XD?MAIN?134
00813AH   00813AH   000001H   BYTE   OFFS..   XDATA          ?XD?MAIN?143
00813BH   00813BH   000001H   BYTE   OFFS..   XDATA          ?XD?MAIN?153
00813CH   00813CH   000001H   BYTE   OFFS..   XDATA          ?XD?MAIN?166
LX51 LINKER/LOCATER V4.64.0.0                                                         04/13/2020  14:54:03  PAGE 6


00813DH   00813DH   000001H   BYTE   OFFS..   XDATA          ?XD?MAIN?181
00813EH   00813EH   000001H   BYTE   OFFS..   XDATA          ?XD?MAIN?195
00813FH   00813FH   000001H   BYTE   OFFS..   XDATA          ?XD?MAIN?209
008140H   008140H   000001H   BYTE   OFFS..   XDATA          ?XD?MAIN?133
008141H   008141H   000001H   BYTE   OFFS..   XDATA          ?XD?MAIN?142
008142H   008142H   000001H   BYTE   OFFS..   XDATA          ?XD?MAIN?152
008143H   008143H   000001H   BYTE   OFFS..   XDATA          ?XD?MAIN?165
008144H   008144H   000001H   BYTE   OFFS..   XDATA          ?XD?MAIN?180
008145H   008145H   000001H   BYTE   OFFS..   XDATA          ?XD?MAIN?194
008146H   008146H   000001H   BYTE   OFFS..   XDATA          ?XD?MAIN?208
008147H   008147H   000001H   BYTE   OFFS..   XDATA          ?XD?MAIN?3
008148H   008148H   000001H   BYTE   OFFS..   XDATA          ?XD?MAIN?141
008149H   008149H   000001H   BYTE   OFFS..   XDATA          ?XD?MAIN?151
00814AH   00814AH   000001H   BYTE   OFFS..   XDATA          ?XD?MAIN?164
00814BH   00814BH   000001H   BYTE   OFFS..   XDATA          ?XD?MAIN?179
00814CH   00814CH   000001H   BYTE   OFFS..   XDATA          ?XD?MAIN?193
00814DH   00814DH   000001H   BYTE   OFFS..   XDATA          ?XD?MAIN?207
00814EH   00814EH   000001H   BYTE   OFFS..   XDATA          ?XD?MAIN?2
00814FH   00814FH   000001H   BYTE   OFFS..   XDATA          ?XD?MAIN?14
008150H   008150H   000001H   BYTE   OFFS..   XDATA          ?XD?MAIN?150
008151H   008151H   000001H   BYTE   OFFS..   XDATA          ?XD?MAIN?163
008152H   008152H   000001H   BYTE   OFFS..   XDATA          ?XD?MAIN?178
008153H   008153H   000001H   BYTE   OFFS..   XDATA          ?XD?MAIN?192
008154H   008154H   000001H   BYTE   OFFS..   XDATA          ?XD?MAIN?206
008155H   008155H   000001H   BYTE   OFFS..   XDATA          ?XD?MAIN?1
008156H   008156H   000001H   BYTE   OFFS..   XDATA          ?XD?MAIN?13
008157H   008157H   000001H   BYTE   OFFS..   XDATA          ?XD?MAIN?21
008158H   008158H   000001H   BYTE   OFFS..   XDATA          ?XD?MAIN?162
008159H   008159H   000001H   BYTE   OFFS..   XDATA          ?XD?MAIN?177
00815AH   00815AH   000001H   BYTE   OFFS..   XDATA          ?XD?MAIN?191
00815BH   00815BH   000001H   BYTE   OFFS..   XDATA          ?XD?MAIN?205
00815CH   00815CH   000001H   BYTE   OFFS..   XDATA          ?XD?MAIN?0
00815DH   00815DH   000001H   BYTE   OFFS..   XDATA          ?XD?MAIN?12
00815EH   00FBFFH   007AA2H   ---    ---      **GAP**
00FC00H   00FC00H   000001H   BYTE   OFFS..   XDATA          ?XD?MAIN?119
00FC01H   00FC01H   000001H   BYTE   OFFS..   XDATA          ?XD?MAIN?115
00FC02H   00FC02H   000001H   BYTE   OFFS..   XDATA          ?XD?MAIN?118
00FC03H   00FC03H   000001H   BYTE   OFFS..   XDATA          ?XD?MAIN?61
00FC04H   00FC04H   000001H   BYTE   OFFS..   XDATA          ?XD?MAIN?111
00FC05H   00FC05H   000001H   BYTE   OFFS..   XDATA          ?XD?MAIN?78
00FC06H   00FC06H   000001H   BYTE   OFFS..   XDATA          ?XD?MAIN?72
00FC07H   00FC07H   000001H   BYTE   OFFS..   XDATA          ?XD?MAIN?91

* * * * * * * * *   R E M O V E D     S E G M E N T S   * * * * * * * *
   *DEL*:           00001DH   BYTE   INBLOCK  CODE           ?PR?_DELAY_50US?DELAY
   *DEL*:           00001BH   BYTE   INBLOCK  CODE           ?PR?_DELAY_MS?DELAY
   *DEL*:           00000BH   BYTE   INBLOCK  CODE           ?PR?SYS_CLK_SET_IRCH?SYSTEM_CLOCK
   *DEL*:           00000DH   BYTE   INBLOCK  CODE           ?PR?SYS_CLK_SET_IRCL?SYSTEM_CLOCK
   *DEL*:           00001FH   BYTE   INBLOCK  CODE           ?PR?SYS_CLK_SET_XOSCL?SYSTEM_CLOCK
   *DEL*:           00000DH   BYTE   INBLOCK  CODE           ?PR?SYS_CLK_SET_TFRC?SYSTEM_CLOCK
   *DEL*:           000037H   BYTE   INBLOCK  CODE           ?PR?TS_BASELINEFORCEUPDATE?TS_SEVICE
   *DEL*:           000001H   BYTE   UNIT     DATA           ?DT?TS_BASELINEFORCEUPDATE?TS_SEVICE
   *DEL*:           000041H   BYTE   INBLOCK  CODE           ?PR?_SETWHEELSLIDERREFCH?TS_SEVICE
   *DEL*:           000002H   BYTE   UNIT     DATA           ?DT?_SETWHEELSLIDERREFCH?TS_SEVICE
   *DEL*:           000214H   BYTE   INBLOCK  CODE           ?PR?_WHEELTOUCHJUDGE?TS_SEVICE
   *DEL*:           000014H   BYTE   UNIT     DATA           ?DT?_WHEELTOUCHJUDGE?TS_SEVICE
   *DEL*:           000000H.1 BIT    UNIT     BIT            ?BI?_WHEELTOUCHJUDGE?TS_SEVICE
   *DEL*:           000237H   BYTE   INBLOCK  CODE           ?PR?_SLIDERTOUCHJUDGE?TS_SEVICE
   *DEL*:           000014H   BYTE   UNIT     DATA           ?DT?_SLIDERTOUCHJUDGE?TS_SEVICE



OVERLAY MAP OF MODULE:   .\hex\ca51f2 (MAIN)


LX51 LINKER/LOCATER V4.64.0.0                                                         04/13/2020  14:54:03  PAGE 7


FUNCTION/MODULE                          BIT_GROUP   DATA_GROUP 
--> CALLED FUNCTION/MODULE              START  STOP  START  STOP
================================================================
INT8_ISR/INTERRUPT                      ----- -----  ----- -----
  +--> TS_MS_ISR/TS_API
  +--> TS_HS_ISR/TS_API

TS_MS_ISR/TS_API                        ----- -----  ----- -----
  +--> TS_API

TS_API                                  ----- -----  ----- -----
  +--> ?CO?TS_API

?CO?TS_API                              ----- -----  ----- -----

TS_HS_ISR/TS_API                        ----- -----  ----- -----
  +--> TS_API

*** NEW ROOT **************************

INT3_ISR/INTERRUPT                      ----- -----  ----- -----
  +--> TS_ISR/TS_API

TS_ISR/TS_API                           ----- -----  0008H 0014H
  +--> TS_API
  +--> TS_SCANSTART/TS_SEVICE

TS_SCANSTART/TS_SEVICE                  ----- -----  ----- -----

*** NEW ROOT **************************

INT6_ISR/INTERRUPT                      ----- -----  ----- -----
  +--> I2C_ISR/DEBUG

I2C_ISR/DEBUG                           ----- -----  ----- -----
  +--> DEBUG
  +--> ?CO?DEBUG

DEBUG                                   ----- -----  ----- -----

?CO?DEBUG                               ----- -----  ----- -----

*** NEW ROOT **************************

?C_C51STARTUP                           ----- -----  ----- -----
  +--> MAIN/MAIN
  +--> ?C_INITSEG

MAIN/MAIN                               ----- -----  ----- -----
  +--> SYSTEMINIT/MAIN
  +--> TS_INIT/TS_API
  +--> TS_ACTION/TS_API

SYSTEMINIT/MAIN                         ----- -----  ----- -----
  +--> _SYS_CLK_SET_PLL/SYSTEM_CLOCK

_SYS_CLK_SET_PLL/SYSTEM_CLOCK           ----- -----  ----- -----
  +--> SYSTEM_CLOCK

SYSTEM_CLOCK                            ----- -----  ----- -----

TS_INIT/TS_API                          ----- -----  ----- -----
  +--> DEBUG_INIT/DEBUG
  +--> ?CO?TS_API
  +--> TS_IO_INIT/TS_SEVICE
LX51 LINKER/LOCATER V4.64.0.0                                                         04/13/2020  14:54:03  PAGE 8



DEBUG_INIT/DEBUG                        ----- -----  ----- -----

TS_IO_INIT/TS_SEVICE                    ----- -----  ----- -----
  +--> ?CO?TS_SEVICE

?CO?TS_SEVICE                           ----- -----  ----- -----

TS_ACTION/TS_API                        ----- -----  ----- -----
  +--> TS_RUNINIT/TS_API
  +--> TS_DATAFILTERING/TS_API
  +--> TSKEY_DATADEAL/TS_API
  +--> DEBUG_PARAMLOAD/DEBUG
  +--> TS_INIT/TS_API
  +--> TS_GETKEY/TS_API

TS_RUNINIT/TS_API                       ----- -----  0015H 0015H
  +--> TS_SCANSTART/TS_SEVICE
  +--> TS_API
  +--> ?CO?TS_API
  +--> _TS_AREACONFIRMTIMERSET/TS_SEVICE
  +--> DEBUG_PARAMLOAD/DEBUG

_TS_AREACONFIRMTIMERSET/TS_SEVICE       ----- -----  ----- -----
  +--> ?CO?TS_API

DEBUG_PARAMLOAD/DEBUG                   ----- -----  ----- -----

TS_DATAFILTERING/TS_API                 ----- -----  0015H 001BH
  +--> TS_API

TSKEY_DATADEAL/TS_API                   ----- -----  0015H 0017H
  +--> TS_API
  +--> ?CO?TS_API
  +--> _TS_AREADEVIATEDETECTION/TS_SEVICE
  +--> _TS_AREACONFIRMTIMERSET/TS_SEVICE
  +--> _TS_GETDATAAREA/TS_SEVICE

_TS_AREADEVIATEDETECTION/TS_SEVICE      ----- -----  ----- -----

_TS_GETDATAAREA/TS_SEVICE               20H.4 20H.4  0018H 0019H
  +--> TS_SEVICE

TS_SEVICE                               ----- -----  ----- -----
  +--> ?CO?TS_API

TS_GETKEY/TS_API                        ----- -----  ----- -----
  +--> ?CO?TS_API

?C_INITSEG                              ----- -----  ----- -----



PUBLIC SYMBOLS OF MODULE:  .\hex\ca51f2 (MAIN)


      VALUE       CLASS    TYPE      PUBLIC SYMBOL NAME
      =================================================
      00000020H.4 BIT      BIT       ?_TS_GetDataArea?BIT
      010009E1H   CODE     ---       ?C?CLDOPTR
      00000000H   NUMBER   ---       ?C?CODESEG
      01000A20H   CODE     ---       ?C?CSTOPTR
      01000A0EH   CODE     ---       ?C?CSTPTR
      01000ADFH   CODE     ---       ?C?IILDX
      01000A42H   CODE     ---       ?C?IMUL
LX51 LINKER/LOCATER V4.64.0.0                                                         04/13/2020  14:54:03  PAGE 9


      01000BE7H   CODE     ---       ?C?LIMUL
      01000BC3H   CODE     ---       ?C?LSTXDATA
      01000BCFH   CODE     ---       ?C?OFFXADD
      01000BDBH   CODE     ---       ?C?PLDCODE
      01000AA9H   CODE     ---       ?C?SIDIV
      01000A54H   CODE     ---       ?C?UIDIV
      01000B31H   CODE     ---       ?C?ULDIV
      00000000H   NUMBER   ---       ?C?XDATASEG
      01000C5BH   CODE     ---       ?C_START
      01000000H   CODE     ---       ?C_STARTUP
*DEL*:00000000H   CODE     ---       _Delay_50us
*DEL*:00000000H   CODE     ---       _Delay_ms
*DEL*:00000000H   CODE     ---       _SetWheelSliderRefCh
*DEL*:00000000H   CODE     ---       _SliderTouchJudge
      0100097AH   CODE     ---       _Sys_Clk_Set_PLL
      010007E8H   CODE     ---       _TS_AreaConfirmTimerSet
      0100091FH   CODE     ---       _TS_AreaDeviateDetection
      010006DAH   CODE     ---       _TS_GetDataArea
*DEL*:00000000H   CODE     ---       _WheelTouchJudge
*SFR* 000000D0H.6 DATA     BIT       AC
*SFR* 000000E0H   DATA     BYTE      ACC
      0200808DH   XDATA    BYTE      ACPDHH
      0200808CH   XDATA    BYTE      ACPDHL
      0200808BH   XDATA    BYTE      ACPDLH
      0200808AH   XDATA    BYTE      ACPDLL
      00000027H   DATA     BYTE      ActiveTouchType
      02008089H   XDATA    BYTE      ADCALH
      02008088H   XDATA    BYTE      ADCALL
*SFR* 000000BDH   DATA     BYTE      ADCDH
*SFR* 000000BCH   DATA     BYTE      ADCDL
*SFR* 000000BBH   DATA     BYTE      ADCFGH
*SFR* 000000BAH   DATA     BYTE      ADCFGL
*SFR* 000000B9H   DATA     BYTE      ADCON
      01000D13H   CONST    ---       AREA_CONFIRM_TIME_TAB
*SFR* 000000C6H   DATA     BYTE      ATKMH
*SFR* 000000C5H   DATA     BYTE      ATKML
      02008093H   XDATA    BYTE      ATKNH
      02008092H   XDATA    BYTE      ATKNL
*SFR* 000000F0H   DATA     BYTE      B
      02008080H   XDATA    BYTE      CKCON
      02008082H   XDATA    BYTE      CKDIV
*SFR* 000000BFH   DATA     BYTE      CKMIF
*SFR* 000000BEH   DATA     BYTE      CKMON
      02008081H   XDATA    BYTE      CKSEL
      02008048H   XDATA    BYTE      CP0CON
      02008049H   XDATA    BYTE      CP1CON
      0200804AH   XDATA    BYTE      CP2CON
      0200804BH   XDATA    BYTE      CP3CON
      0200804CH   XDATA    BYTE      CPCKS
      0200804DH   XDATA    BYTE      CPSTA
      0200804EH   XDATA    BYTE      CPVTC
      0200805CH   XDATA    BYTE      CTMCNTH
      0200805BH   XDATA    BYTE      CTMCNTL
      02008058H   XDATA    BYTE      CTMCON
      0200805AH   XDATA    BYTE      CTMVTHH
      02008059H   XDATA    BYTE      CTMVTHL
*SFR* 000000D0H.7 DATA     BIT       CY
      0100099EH   CODE     ---       Debug_init
      01000795H   CODE     ---       Debug_ParamLoad
*SFR* 00000083H   DATA     BYTE      DP0H
*SFR* 00000082H   DATA     BYTE      DP0L
*SFR* 00000085H   DATA     BYTE      DP1H
*SFR* 00000084H   DATA     BYTE      DP1L
*SFR* 000000D0H.1 DATA     BIT       DPS
*SFR* 000000A8H.7 DATA     BIT       EA
LX51 LINKER/LOCATER V4.64.0.0                                                         04/13/2020  14:54:03  PAGE 10


      0200008EH   XDATA    BYTE      EnterStopScanTimer
*SFR* 000000FBH   DATA     BYTE      EPCON
*SFR* 000000F9H   DATA     BYTE      EPIE
*SFR* 000000FAH   DATA     BYTE      EPIF
*SFR* 000000A8H.4 DATA     BIT       ES0
*SFR* 000000A8H.6 DATA     BIT       ES1
*SFR* 000000A8H.1 DATA     BIT       ET0
*SFR* 000000A8H.3 DATA     BIT       ET1
*SFR* 000000A8H.5 DATA     BIT       ET2
*SFR* 000000A8H   DATA     BIT       EX0
*SFR* 000000A8H.2 DATA     BIT       EX1
*SFR* 000000E8H   DATA     BYTE      EXIE
*SFR* 000000F8H   DATA     BYTE      EXIP
*SFR* 000000D0H.5 DATA     BIT       F0
      0200FC01H   XDATA    BYTE      FSCMD
      0200FC02H   XDATA    BYTE      FSDAT
      02008051H   XDATA    BYTE      FT0SH
      02008050H   XDATA    BYTE      FT0SL
      02008053H   XDATA    BYTE      FT1SH
      02008052H   XDATA    BYTE      FT1SL
      02008055H   XDATA    BYTE      FT2SH
      02008054H   XDATA    BYTE      FT2SL
      02008057H   XDATA    BYTE      FT3SH
      02008056H   XDATA    BYTE      FT3SL
      0200811EH   XDATA    BYTE      FTCTL
      02008068H   XDATA    BYTE      HDCT0
      02008069H   XDATA    BYTE      HDCT1
      02008072H   XDATA    BYTE      HDCT10
      02008073H   XDATA    BYTE      HDCT11
      0200806AH   XDATA    BYTE      HDCT2
      0200806BH   XDATA    BYTE      HDCT3
      0200806CH   XDATA    BYTE      HDCT4
      0200806DH   XDATA    BYTE      HDCT5
      0200806EH   XDATA    BYTE      HDCT6
      0200806FH   XDATA    BYTE      HDCT7
      02008070H   XDATA    BYTE      HDCT8
      02008071H   XDATA    BYTE      HDCT9
*SFR* 000000AFH   DATA     BYTE      HVTH
      010005FDH   CODE     ---       I2C_ISR
*SFR* 000000B3H   DATA     BYTE      I2CADM
*SFR* 000000B2H   DATA     BYTE      I2CADR
*SFR* 000000B4H   DATA     BYTE      I2CCCR
*SFR* 000000B1H   DATA     BYTE      I2CCON
*SFR* 000000B5H   DATA     BYTE      I2CDAT
*SFR* 000000B7H   DATA     BYTE      I2CFLG
      02008101H   XDATA    BYTE      I2CIOS
*SFR* 000000B6H   DATA     BYTE      I2CSTA
*SFR* 000000FDH   DATA     BYTE      IDLSTH
*SFR* 000000FCH   DATA     BYTE      IDLSTL
*SFR* 000000A8H   DATA     BYTE      IE
*SFR* 00000088H.1 DATA     BIT       IE0
*SFR* 00000088H.3 DATA     BIT       IE1
      02008084H   XDATA    BYTE      IHCFGH
      02008083H   XDATA    BYTE      IHCFGL
      00000020H.3 BIT      BIT       iicReadMode
      02008086H   XDATA    BYTE      ILCFGH
      02008085H   XDATA    BYTE      ILCFGL
*SFR* 000000F7H   DATA     BYTE      INDEX
*SFR* 000000E8H   DATA     BIT       INT2EN
      0100084AH   CODE     ---       INT3_ISR
*SFR* 000000E8H.1 DATA     BIT       INT3EN
*SFR* 000000E8H.2 DATA     BIT       INT4EN
*SFR* 000000E8H.3 DATA     BIT       INT5EN
      01000003H   CODE     ---       INT6_ISR
*SFR* 000000E8H.4 DATA     BIT       INT6EN
LX51 LINKER/LOCATER V4.64.0.0                                                         04/13/2020  14:54:03  PAGE 11


*SFR* 000000E8H.5 DATA     BIT       INT7EN
      01000739H   CODE     ---       INT8_ISR
*SFR* 000000E8H.6 DATA     BIT       INT8EN
*SFR* 000000E8H.7 DATA     BIT       INT9EN
*SFR* 000000B8H   DATA     BYTE      IP
*SFR* 00000088H   DATA     BIT       IT0
*SFR* 0000008FH   DATA     BYTE      IT0CON
*SFR* 00000088H.2 DATA     BIT       IT1
*SFR* 0000008EH   DATA     BYTE      IT1CON
      020000B1H   XDATA    BYTE      Key_Cnt_Debug
      0200008FH   XDATA    BYTE      KeysFlagSN
      02000001H   XDATA    DWORD     KeysFlagSN_Debug
      0200FC03H   XDATA    BYTE      LOCK
*SFR* 000000EFH   DATA     BYTE      LVDCON
      02008117H   XDATA    BYTE      LXCAD
*SFR* 000000E2H   DATA     BYTE      LXCFG
*SFR* 000000E1H   DATA     BYTE      LXCON
*SFR* 000000E3H   DATA     BYTE      LXDAT
*SFR* 000000E5H   DATA     BYTE      LXDIVH
*SFR* 000000E4H   DATA     BYTE      LXDIVL
      01000046H   CODE     ---       main
      01000D0DH   CONST    ---       MASK_TAB
*SFR* 000000E6H   DATA     BYTE      MDUCON
*SFR* 000000E7H   DATA     BYTE      MDUDAT
      0200FC00H   XDATA    BYTE      MECON
      02008064H   XDATA    BYTE      MFPCON
      02008063H   XDATA    BYTE      MHLCON
      02008061H   XDATA    BYTE      MOTCFG
      02008065H   XDATA    BYTE      MOTCMD
      02008060H   XDATA    BYTE      MOTCON
      02008067H   XDATA    BYTE      MOTIF
      02008074H   XDATA    BYTE      MOTPLC
      02008062H   XDATA    BYTE      MTGCON
      02008066H   XDATA    BYTE      MTGDL
      02008040H   XDATA    BYTE      OPACON
      02008041H   XDATA    BYTE      OPBCON
      02008042H   XDATA    BYTE      OSTRIM
*SFR* 000000D0H.2 DATA     BIT       OV
*SFR* 000000D0H   DATA     BIT       P
*SFR* 00000080H   DATA     BYTE      P0
*SFR* 00000080H   DATA     BIT       P00
      02008120H   XDATA    BYTE      P00C
      02008000H   XDATA    BYTE      P00F
*SFR* 00000080H.1 DATA     BIT       P01
      02008121H   XDATA    BYTE      P01C
      02008001H   XDATA    BYTE      P01F
*SFR* 00000080H.2 DATA     BIT       P02
      02008122H   XDATA    BYTE      P02C
      02008002H   XDATA    BYTE      P02F
*SFR* 00000080H.3 DATA     BIT       P03
      02008123H   XDATA    BYTE      P03C
      02008003H   XDATA    BYTE      P03F
*SFR* 00000080H.4 DATA     BIT       P04
      02008124H   XDATA    BYTE      P04C
      02008004H   XDATA    BYTE      P04F
*SFR* 00000080H.5 DATA     BIT       P05
      02008125H   XDATA    BYTE      P05C
      02008005H   XDATA    BYTE      P05F
*SFR* 00000080H.6 DATA     BIT       P06
      02008126H   XDATA    BYTE      P06C
      02008006H   XDATA    BYTE      P06F
*SFR* 00000080H.7 DATA     BIT       P07
      02008127H   XDATA    BYTE      P07C
      02008007H   XDATA    BYTE      P07F
*SFR* 00000090H   DATA     BYTE      P1
LX51 LINKER/LOCATER V4.64.0.0                                                         04/13/2020  14:54:03  PAGE 12


*SFR* 00000090H   DATA     BIT       P10
      02008128H   XDATA    BYTE      P10C
      02008008H   XDATA    BYTE      P10F
*SFR* 00000090H.1 DATA     BIT       P11
      02008129H   XDATA    BYTE      P11C
      02008009H   XDATA    BYTE      P11F
*SFR* 00000090H.2 DATA     BIT       P12
      0200812AH   XDATA    BYTE      P12C
      0200800AH   XDATA    BYTE      P12F
*SFR* 00000090H.3 DATA     BIT       P13
      0200812BH   XDATA    BYTE      P13C
      0200800BH   XDATA    BYTE      P13F
*SFR* 00000090H.4 DATA     BIT       P14
      0200812CH   XDATA    BYTE      P14C
      0200800CH   XDATA    BYTE      P14F
*SFR* 00000090H.5 DATA     BIT       P15
      0200812DH   XDATA    BYTE      P15C
      0200800DH   XDATA    BYTE      P15F
*SFR* 00000090H.6 DATA     BIT       P16
      0200812EH   XDATA    BYTE      P16C
      0200800EH   XDATA    BYTE      P16F
*SFR* 00000090H.7 DATA     BIT       P17
      0200812FH   XDATA    BYTE      P17C
      0200800FH   XDATA    BYTE      P17F
*SFR* 000000A0H   DATA     BYTE      P2
*SFR* 000000A0H   DATA     BIT       P20
      02008130H   XDATA    BYTE      P20C
      02008010H   XDATA    BYTE      P20F
*SFR* 000000A0H.1 DATA     BIT       P21
      02008131H   XDATA    BYTE      P21C
      02008011H   XDATA    BYTE      P21F
*SFR* 000000A0H.2 DATA     BIT       P22
      02008132H   XDATA    BYTE      P22C
      02008012H   XDATA    BYTE      P22F
*SFR* 000000A0H.3 DATA     BIT       P23
      02008133H   XDATA    BYTE      P23C
      02008013H   XDATA    BYTE      P23F
*SFR* 000000A0H.4 DATA     BIT       P24
      02008134H   XDATA    BYTE      P24C
      02008014H   XDATA    BYTE      P24F
*SFR* 000000A0H.5 DATA     BIT       P25
      02008135H   XDATA    BYTE      P25C
      02008015H   XDATA    BYTE      P25F
*SFR* 000000A0H.6 DATA     BIT       P26
      02008136H   XDATA    BYTE      P26C
      02008016H   XDATA    BYTE      P26F
*SFR* 000000A0H.7 DATA     BIT       P27
      02008137H   XDATA    BYTE      P27C
      02008017H   XDATA    BYTE      P27F
*SFR* 000000B0H   DATA     BYTE      P3
*SFR* 000000B0H   DATA     BIT       P30
      02008138H   XDATA    BYTE      P30C
      02008018H   XDATA    BYTE      P30F
*SFR* 000000B0H.1 DATA     BIT       P31
      02008139H   XDATA    BYTE      P31C
      02008019H   XDATA    BYTE      P31F
*SFR* 000000B0H.2 DATA     BIT       P32
      0200813AH   XDATA    BYTE      P32C
      0200801AH   XDATA    BYTE      P32F
*SFR* 000000B0H.3 DATA     BIT       P33
      0200813BH   XDATA    BYTE      P33C
      0200801BH   XDATA    BYTE      P33F
*SFR* 000000B0H.4 DATA     BIT       P34
      0200813CH   XDATA    BYTE      P34C
      0200801CH   XDATA    BYTE      P34F
LX51 LINKER/LOCATER V4.64.0.0                                                         04/13/2020  14:54:03  PAGE 13


*SFR* 000000B0H.5 DATA     BIT       P35
      0200813DH   XDATA    BYTE      P35C
      0200801DH   XDATA    BYTE      P35F
*SFR* 000000B0H.6 DATA     BIT       P36
      0200813EH   XDATA    BYTE      P36C
      0200801EH   XDATA    BYTE      P36F
*SFR* 000000B0H.7 DATA     BIT       P37
      0200813FH   XDATA    BYTE      P37C
      0200801FH   XDATA    BYTE      P37F
*SFR* 000000C0H   DATA     BYTE      P4
*SFR* 000000C0H   DATA     BIT       P40
      02008140H   XDATA    BYTE      P40C
      02008020H   XDATA    BYTE      P40F
*SFR* 000000C0H.1 DATA     BIT       P41
      02008141H   XDATA    BYTE      P41C
      02008021H   XDATA    BYTE      P41F
*SFR* 000000C0H.2 DATA     BIT       P42
      02008142H   XDATA    BYTE      P42C
      02008022H   XDATA    BYTE      P42F
*SFR* 000000C0H.3 DATA     BIT       P43
      02008143H   XDATA    BYTE      P43C
      02008023H   XDATA    BYTE      P43F
*SFR* 000000C0H.4 DATA     BIT       P44
      02008144H   XDATA    BYTE      P44C
      02008024H   XDATA    BYTE      P44F
*SFR* 000000C0H.5 DATA     BIT       P45
      02008145H   XDATA    BYTE      P45C
      02008025H   XDATA    BYTE      P45F
*SFR* 000000C0H.6 DATA     BIT       P46
      02008146H   XDATA    BYTE      P46C
      02008026H   XDATA    BYTE      P46F
*SFR* 000000C0H.7 DATA     BIT       P47
      02008147H   XDATA    BYTE      P47C
      02008027H   XDATA    BYTE      P47F
*SFR* 000000D8H   DATA     BYTE      P5
*SFR* 000000D8H   DATA     BIT       P50
      02008148H   XDATA    BYTE      P50C
      02008028H   XDATA    BYTE      P50F
*SFR* 000000D8H.1 DATA     BIT       P51
      02008149H   XDATA    BYTE      P51C
      02008029H   XDATA    BYTE      P51F
*SFR* 000000D8H.2 DATA     BIT       P52
      0200814AH   XDATA    BYTE      P52C
      0200802AH   XDATA    BYTE      P52F
*SFR* 000000D8H.3 DATA     BIT       P53
      0200814BH   XDATA    BYTE      P53C
      0200802BH   XDATA    BYTE      P53F
*SFR* 000000D8H.4 DATA     BIT       P54
      0200814CH   XDATA    BYTE      P54C
      0200802CH   XDATA    BYTE      P54F
*SFR* 000000D8H.5 DATA     BIT       P55
      0200814DH   XDATA    BYTE      P55C
      0200802DH   XDATA    BYTE      P55F
*SFR* 000000D8H.6 DATA     BIT       P56
      0200814EH   XDATA    BYTE      P56C
      0200802EH   XDATA    BYTE      P56F
*SFR* 000000D8H.7 DATA     BIT       P57
      0200814FH   XDATA    BYTE      P57C
      0200802FH   XDATA    BYTE      P57F
*SFR* 000000A9H   DATA     BYTE      P6
      02008150H   XDATA    BYTE      P60C
      02008030H   XDATA    BYTE      P60F
      02008151H   XDATA    BYTE      P61C
      02008031H   XDATA    BYTE      P61F
      02008152H   XDATA    BYTE      P62C
LX51 LINKER/LOCATER V4.64.0.0                                                         04/13/2020  14:54:03  PAGE 14


      02008032H   XDATA    BYTE      P62F
      02008153H   XDATA    BYTE      P63C
      02008033H   XDATA    BYTE      P63F
      02008154H   XDATA    BYTE      P64C
      02008034H   XDATA    BYTE      P64F
      02008155H   XDATA    BYTE      P65C
      02008035H   XDATA    BYTE      P65F
      02008156H   XDATA    BYTE      P66C
      02008036H   XDATA    BYTE      P66F
      02008157H   XDATA    BYTE      P67C
      02008037H   XDATA    BYTE      P67F
*SFR* 000000D9H   DATA     BYTE      P7
      02008158H   XDATA    BYTE      P70C
      02008038H   XDATA    BYTE      P70F
      02008159H   XDATA    BYTE      P71C
      02008039H   XDATA    BYTE      P71F
      0200815AH   XDATA    BYTE      P72C
      0200803AH   XDATA    BYTE      P72F
      0200815BH   XDATA    BYTE      P73C
      0200803BH   XDATA    BYTE      P73F
      0200815CH   XDATA    BYTE      P74C
      0200803CH   XDATA    BYTE      P74F
      0200815DH   XDATA    BYTE      P75C
      0200803DH   XDATA    BYTE      P75F
      0200FC04H   XDATA    BYTE      PADRD
*SFR* 00000087H   DATA     BYTE      PCON
*SFR* 000000AEH   DATA     BYTE      PLLCON
      0000003BH   IDATA    BYTE      PreKeysFlagSN
*SFR* 000000B8H.4 DATA     BIT       PS0
*SFR* 000000B8H.6 DATA     BIT       PS1
*SFR* 000000D0H   DATA     BYTE      PSW
*SFR* 000000B8H.1 DATA     BIT       PT0
*SFR* 000000B8H.3 DATA     BIT       PT1
*SFR* 000000B8H.5 DATA     BIT       PT2
      0000002DH   DATA     ---       pTS_Info
      0200FC06H   XDATA    BYTE      PTSH
      0200FC05H   XDATA    BYTE      PTSL
*SFR* 00000086H   DATA     BYTE      PWCON
*SFR* 000000D4H   DATA     BYTE      PWMAIF
*SFR* 000000D5H   DATA     BYTE      PWMBIF
*SFR* 000000DEH   DATA     BYTE      PWMCFG
*SFR* 000000D6H   DATA     BYTE      PWMCIF
*SFR* 000000DCH   DATA     BYTE      PWMCMAX
*SFR* 000000DDH   DATA     BYTE      PWMCON
*SFR* 000000D7H   DATA     BYTE      PWMDIF
*SFR* 000000D1H   DATA     BYTE      PWMDIVH
*SFR* 000000DFH   DATA     BYTE      PWMDIVL
*SFR* 000000D3H   DATA     BYTE      PWMDUTH
*SFR* 000000D2H   DATA     BYTE      PWMDUTL
*SFR* 000000DAH   DATA     BYTE      PWMEN
*SFR* 000000DBH   DATA     BYTE      PWMUPD
*SFR* 000000B8H   DATA     BIT       PX0
*SFR* 000000B8H.2 DATA     BIT       PX1
      01000CACH   CONST    ---       pXSFR
*SFR* 00000098H.2 DATA     BIT       RB8
*SFR* 00000091H   DATA     BYTE      RCCON
*SFR* 0000009FH   DATA     BYTE      RCMSHH
*SFR* 0000009EH   DATA     BYTE      RCMSHL
*SFR* 00000097H   DATA     BYTE      RCMSLH
*SFR* 00000096H   DATA     BYTE      RCMSLL
*SFR* 00000095H   DATA     BYTE      RCTAGH
*SFR* 00000094H   DATA     BYTE      RCTAGL
      00000030H   DATA     BYTE      regAddr
*SFR* 00000098H.4 DATA     BIT       REN
      0200FC07H   XDATA    BYTE      REPSET
LX51 LINKER/LOCATER V4.64.0.0                                                         04/13/2020  14:54:03  PAGE 15


*SFR* 00000098H   DATA     BIT       RI0
*SFR* 000000D0H.3 DATA     BIT       RS0
*SFR* 000000D0H.4 DATA     BIT       RS1
*SFR* 000000ECH   DATA     BYTE      RTAH
*SFR* 000000EBH   DATA     BYTE      RTAM
*SFR* 000000EAH   DATA     BYTE      RTAS
*SFR* 000000F6H   DATA     BYTE      RTCDH
*SFR* 000000F5H   DATA     BYTE      RTCDL
*SFR* 000000F4H   DATA     BYTE      RTCH
*SFR* 000000EEH   DATA     BYTE      RTCIF
*SFR* 000000F3H   DATA     BYTE      RTCM
*SFR* 000000F1H   DATA     BYTE      RTCON
*SFR* 000000F2H   DATA     BYTE      RTCS
*SFR* 000000E9H   DATA     BYTE      RTCSS
*SFR* 000000EDH   DATA     BYTE      RTMSS
      00000031H   DATA     BYTE      rxOffset
*SFR* 00000099H   DATA     BYTE      S0BUF
*SFR* 00000098H   DATA     BYTE      S0CON
*SFR* 0000009BH   DATA     BYTE      S1BUF
*SFR* 0000009AH   DATA     BYTE      S1CON
*SFR* 0000009DH   DATA     BYTE      S1RELH
*SFR* 0000009CH   DATA     BYTE      S1RELL
*SFR* 000000A2H   DATA     BYTE      S2BUF
*SFR* 000000A1H   DATA     BYTE      S2CON
*SFR* 000000A4H   DATA     BYTE      S2RELH
*SFR* 000000A3H   DATA     BYTE      S2RELL
*SFR* 00000098H.7 DATA     BIT       SM0
*SFR* 00000098H.6 DATA     BIT       SM1
*SFR* 00000098H.5 DATA     BIT       SM2
      02008078H   XDATA    BYTE      SMCON
      0200807CH   XDATA    BYTE      SMDATH
      0200807BH   XDATA    BYTE      SMDATL
      0200807AH   XDATA    BYTE      SMDIV
      02008079H   XDATA    BYTE      SMSTA
      0200807EH   XDATA    BYTE      SMVTHH
      0200807DH   XDATA    BYTE      SMVTHL
*SFR* 00000081H   DATA     BYTE      SP
*SFR* 000000A5H   DATA     BYTE      SPCON
*SFR* 000000A6H   DATA     BYTE      SPDAT
      02008100H   XDATA    BYTE      SPMAX
*SFR* 000000A7H   DATA     BYTE      SPSTA
*SFR* 000000FFH   DATA     BYTE      STPSTH
*SFR* 000000FEH   DATA     BYTE      STPSTL
*DEL*:00000000H   CODE     ---       Sys_Clk_Set_IRCH
*DEL*:00000000H   CODE     ---       Sys_Clk_Set_IRCL
*DEL*:00000000H   CODE     ---       Sys_Clk_Set_TFRC
*DEL*:00000000H   CODE     ---       Sys_Clk_Set_XOSCL
      010009BDH   CODE     ---       SystemInit
*SFR* 000000CBH   DATA     BYTE      T2CH
*SFR* 000000CAH   DATA     BYTE      T2CL
*SFR* 000000C8H   DATA     BYTE      T2CON
*SFR* 000000C8H.3 DATA     BIT       T2IE
*SFR* 000000C9H   DATA     BYTE      T2MOD
*SFR* 000000C8H   DATA     BIT       T2P0
*SFR* 000000C8H.1 DATA     BIT       T2P1
*SFR* 000000C8H.4 DATA     BIT       T2R0
*SFR* 000000C8H.5 DATA     BIT       T2R1
*SFR* 00000098H.3 DATA     BIT       TB8
*SFR* 00000088H   DATA     BYTE      TCON
*SFR* 00000088H.5 DATA     BIT       TF0
*SFR* 00000088H.7 DATA     BIT       TF1
*SFR* 000000C8H.7 DATA     BIT       TF2
      02008087H   XDATA    BYTE      TFCFG
*SFR* 0000008CH   DATA     BYTE      TH0
*SFR* 0000008DH   DATA     BYTE      TH1
LX51 LINKER/LOCATER V4.64.0.0                                                         04/13/2020  14:54:03  PAGE 16


*SFR* 000000CDH   DATA     BYTE      TH2
*SFR* 00000098H.1 DATA     BIT       TI0
      00000026H   DATA     BYTE      TK_State
*SFR* 000000C2H   DATA     BYTE      TKCFG
*SFR* 000000C4H   DATA     BYTE      TKCHS
*SFR* 000000C1H   DATA     BYTE      TKCON
*SFR* 000000C7H   DATA     BYTE      TKIF
      02008090H   XDATA    BYTE      TKMAXF
      02008091H   XDATA    BYTE      TKMINF
*SFR* 000000CFH   DATA     BYTE      TKMSH
*SFR* 000000CEH   DATA     BYTE      TKMSL
*SFR* 000000C3H   DATA     BYTE      TKMTS
      02008103H   XDATA    BYTE      TKPWC
*SFR* 0000008AH   DATA     BYTE      TL0
*SFR* 0000008BH   DATA     BYTE      TL1
*SFR* 000000CCH   DATA     BYTE      TL2
      0200810AH   XDATA    BYTE      TLCKS
      0200810FH   XDATA    BYTE      TLCNTD
      0200810CH   XDATA    BYTE      TLCNTKH
      0200810BH   XDATA    BYTE      TLCNTKL
      0200810EH   XDATA    BYTE      TLCNTLH
      0200810DH   XDATA    BYTE      TLCNTLL
      02008110H   XDATA    BYTE      TLCOMS
      02008108H   XDATA    BYTE      TLCON
      02008107H   XDATA    BYTE      TLDAT
      02008106H   XDATA    BYTE      TLEN
      02008109H   XDATA    BYTE      TLFLG
*SFR* 00000089H   DATA     BYTE      TMOD
      020000B2H   XDATA    BYTE      TouchDebugID
      0200811FH   XDATA    BYTE      TPCTL
*SFR* 00000088H.4 DATA     BIT       TR0
*SFR* 00000088H.6 DATA     BIT       TR1
*SFR* 000000C8H.6 DATA     BIT       TR2
      01000889H   CODE     ---       TS_Action
      020000A3H   XDATA    ---       TS_AreaConfirmTimer
      00000028H   DATA     BYTE      TS_BaseCh
      02000011H   XDATA    ---       TS_BaseLineData
*DEL*:00000000H   CODE     ---       TS_BaseLineForceUpdate
      00000033H   IDATA    ---       TS_CH
      020000A9H   XDATA    ---       TS_CH_Debug
      00000039H   IDATA    BYTE      TS_Cnt
      00000020H.1 BIT      BIT       TS_CycleScanDoneFlag
      01000357H   CODE     ---       TS_DataFiltering
      0200001DH   XDATA    ---       TS_FilterBuf
      02000093H   XDATA    ---       TS_FilterPosIdx
      02000005H   XDATA    ---       TS_FirstAreaData
      01000572H   CODE     ---       TS_GetKey
      02000090H   XDATA    BYTE      TS_HalfSecCnt
      0100094DH   CODE     ---       TS_HS_ISR
      00000025H   DATA     BYTE      TS_Index
      01000D30H   CONST    ---       TS_INFO
      01000670H   CODE     ---       TS_init
      02000063H   XDATA    BYTE      TS_Init_Step
      010008C2H   CODE     ---       TS_IO_init
      010004C4H   CODE     ---       TS_ISR
      00000029H   DATA     WORD      TS_Key
      01000CF4H   CONST    ---       TS_KEY_CH_INFO_SEQ
      01000D18H   CONST    ---       TS_KEY_TAB
      0000002BH   DATA     WORD      TS_LongKeyTimer
      010008F1H   CODE     ---       TS_MS_ISR
      02000065H   XDATA    ---       TS_PostData
      02000074H   XDATA    ---       TS_RawData
      0000003AH   IDATA    BYTE      TS_RefCHBaseLineAdjuTimer
      020000A1H   XDATA    WORD      TS_RefChBaseLineData
      02000091H   XDATA    WORD      TS_RefPostData
LX51 LINKER/LOCATER V4.64.0.0                                                         04/13/2020  14:54:03  PAGE 17


      01000291H   CODE     ---       TS_RunInit
      01000800H   CODE     ---       TS_ScanStart
      00000020H.2 BIT      BIT       TS_StableFlag
      00000032H   IDATA    BYTE      TS_State
      020000A0H   XDATA    BYTE      TS_State_Debug
      0100018FH   CODE     ---       TSKey_DataDeal
      02000082H   XDATA    ---       TSKey_FingerThd
      0200009AH   XDATA    ---       TSKey_LongTouchLimitTimer
*SFR* 000000C8H.2 DATA     BIT       UCKS
*SFR* 00000093H   DATA     BYTE      VCKDH
*SFR* 00000092H   DATA     BYTE      VCKDL
*SFR* 000000AAH   DATA     BYTE      WDCON
*SFR* 000000ABH   DATA     BYTE      WDFLG
*SFR* 000000ADH   DATA     BYTE      WDVTHH
*SFR* 000000ACH   DATA     BYTE      WDVTHL
      01000D0CH   CONST    ---       WHEEL_SLIDER0_MAX_MIN_TAB
      020000AFH   XDATA    WORD      WheelSliderCapRateFilter
      02000073H   XDATA    BYTE      WheelSliderMaxIdx
      02000064H   XDATA    BYTE      WheelSliderRefCh



SYMBOL TABLE OF MODULE:  .\hex\ca51f2 (MAIN)

      VALUE       REP       CLASS    TYPE      SYMBOL NAME
      ====================================================
      ---         MODULE    ---      ---       MAIN
      02008007H   PUBLIC    XDATA    BYTE      P07F
      0200800EH   PUBLIC    XDATA    BYTE      P16F
      02008015H   PUBLIC    XDATA    BYTE      P25F
      0200801CH   PUBLIC    XDATA    BYTE      P34F
      02008023H   PUBLIC    XDATA    BYTE      P43F
      0200802AH   PUBLIC    XDATA    BYTE      P52F
      02008031H   PUBLIC    XDATA    BYTE      P61F
      02008038H   PUBLIC    XDATA    BYTE      P70F
      0200813FH   PUBLIC    XDATA    BYTE      P37C
      02008146H   PUBLIC    XDATA    BYTE      P46C
      0200814DH   PUBLIC    XDATA    BYTE      P55C
      02008154H   PUBLIC    XDATA    BYTE      P64C
      0200815BH   PUBLIC    XDATA    BYTE      P73C
      02008006H   PUBLIC    XDATA    BYTE      P06F
      0200800DH   PUBLIC    XDATA    BYTE      P15F
      02008014H   PUBLIC    XDATA    BYTE      P24F
      0200801BH   PUBLIC    XDATA    BYTE      P33F
      02008022H   PUBLIC    XDATA    BYTE      P42F
      02008029H   PUBLIC    XDATA    BYTE      P51F
      02008030H   PUBLIC    XDATA    BYTE      P60F
      0200804DH   PUBLIC    XDATA    BYTE      CPSTA
      02008137H   PUBLIC    XDATA    BYTE      P27C
      0200813EH   PUBLIC    XDATA    BYTE      P36C
      02008145H   PUBLIC    XDATA    BYTE      P45C
      0200814CH   PUBLIC    XDATA    BYTE      P54C
      02008153H   PUBLIC    XDATA    BYTE      P63C
      0200815AH   PUBLIC    XDATA    BYTE      P72C
      02008005H   PUBLIC    XDATA    BYTE      P05F
      0200800CH   PUBLIC    XDATA    BYTE      P14F
      02008013H   PUBLIC    XDATA    BYTE      P23F
      0200801AH   PUBLIC    XDATA    BYTE      P32F
      02008021H   PUBLIC    XDATA    BYTE      P41F
      02008028H   PUBLIC    XDATA    BYTE      P50F
      02008092H   PUBLIC    XDATA    BYTE      ATKNL
      0200812FH   PUBLIC    XDATA    BYTE      P17C
      02008136H   PUBLIC    XDATA    BYTE      P26C
      0200813DH   PUBLIC    XDATA    BYTE      P35C
      02008144H   PUBLIC    XDATA    BYTE      P44C
LX51 LINKER/LOCATER V4.64.0.0                                                         04/13/2020  14:54:03  PAGE 18


      0200814BH   PUBLIC    XDATA    BYTE      P53C
      02008152H   PUBLIC    XDATA    BYTE      P62C
      02008159H   PUBLIC    XDATA    BYTE      P71C
      02008004H   PUBLIC    XDATA    BYTE      P04F
      0200800BH   PUBLIC    XDATA    BYTE      P13F
      02008012H   PUBLIC    XDATA    BYTE      P22F
      02008019H   PUBLIC    XDATA    BYTE      P31F
      02008020H   PUBLIC    XDATA    BYTE      P40F
      02008107H   PUBLIC    XDATA    BYTE      TLDAT
      02008109H   PUBLIC    XDATA    BYTE      TLFLG
      02008127H   PUBLIC    XDATA    BYTE      P07C
      0200812EH   PUBLIC    XDATA    BYTE      P16C
      02008135H   PUBLIC    XDATA    BYTE      P25C
      0200813CH   PUBLIC    XDATA    BYTE      P34C
      02008143H   PUBLIC    XDATA    BYTE      P43C
      0200814AH   PUBLIC    XDATA    BYTE      P52C
      02008151H   PUBLIC    XDATA    BYTE      P61C
      02008158H   PUBLIC    XDATA    BYTE      P70C
      02008003H   PUBLIC    XDATA    BYTE      P03F
      0200800AH   PUBLIC    XDATA    BYTE      P12F
      02008011H   PUBLIC    XDATA    BYTE      P21F
      02008018H   PUBLIC    XDATA    BYTE      P30F
      02008066H   PUBLIC    XDATA    BYTE      MTGDL
      02008126H   PUBLIC    XDATA    BYTE      P06C
      0200812DH   PUBLIC    XDATA    BYTE      P15C
      02008134H   PUBLIC    XDATA    BYTE      P24C
      0200813BH   PUBLIC    XDATA    BYTE      P33C
      02008142H   PUBLIC    XDATA    BYTE      P42C
      02008149H   PUBLIC    XDATA    BYTE      P51C
      02008150H   PUBLIC    XDATA    BYTE      P60C
      02008002H   PUBLIC    XDATA    BYTE      P02F
      02008009H   PUBLIC    XDATA    BYTE      P11F
      02008010H   PUBLIC    XDATA    BYTE      P20F
      02008125H   PUBLIC    XDATA    BYTE      P05C
      0200812CH   PUBLIC    XDATA    BYTE      P14C
      02008133H   PUBLIC    XDATA    BYTE      P23C
      0200813AH   PUBLIC    XDATA    BYTE      P32C
      02008141H   PUBLIC    XDATA    BYTE      P41C
      02008148H   PUBLIC    XDATA    BYTE      P50C
      02008001H   PUBLIC    XDATA    BYTE      P01F
      02008008H   PUBLIC    XDATA    BYTE      P10F
      02008093H   PUBLIC    XDATA    BYTE      ATKNH
      02008124H   PUBLIC    XDATA    BYTE      P04C
      0200812BH   PUBLIC    XDATA    BYTE      P13C
      02008132H   PUBLIC    XDATA    BYTE      P22C
      02008139H   PUBLIC    XDATA    BYTE      P31C
      02008140H   PUBLIC    XDATA    BYTE      P40C
      02008000H   PUBLIC    XDATA    BYTE      P00F
      02008123H   PUBLIC    XDATA    BYTE      P03C
      0200812AH   PUBLIC    XDATA    BYTE      P12C
      02008131H   PUBLIC    XDATA    BYTE      P21C
      02008138H   PUBLIC    XDATA    BYTE      P30C
      0200804CH   PUBLIC    XDATA    BYTE      CPCKS
      02008122H   PUBLIC    XDATA    BYTE      P02C
      02008129H   PUBLIC    XDATA    BYTE      P11C
      02008130H   PUBLIC    XDATA    BYTE      P20C
      02008121H   PUBLIC    XDATA    BYTE      P01C
      02008128H   PUBLIC    XDATA    BYTE      P10C
      02008081H   PUBLIC    XDATA    BYTE      CKSEL
      02008120H   PUBLIC    XDATA    BYTE      P00C
      0200FC00H   PUBLIC    XDATA    BYTE      MECON
      0200FC02H   PUBLIC    XDATA    BYTE      FSDAT
      02008082H   PUBLIC    XDATA    BYTE      CKDIV
      02008080H   PUBLIC    XDATA    BYTE      CKCON
      0200FC01H   PUBLIC    XDATA    BYTE      FSCMD
LX51 LINKER/LOCATER V4.64.0.0                                                         04/13/2020  14:54:03  PAGE 19


      02008056H   PUBLIC    XDATA    BYTE      FT3SL
      02008117H   PUBLIC    XDATA    BYTE      LXCAD
      02008054H   PUBLIC    XDATA    BYTE      FT2SL
      0200FC04H   PUBLIC    XDATA    BYTE      PADRD
      02008052H   PUBLIC    XDATA    BYTE      FT1SL
      02008087H   PUBLIC    XDATA    BYTE      TFCFG
      02008050H   PUBLIC    XDATA    BYTE      FT0SL
      02008057H   PUBLIC    XDATA    BYTE      FT3SH
      02008055H   PUBLIC    XDATA    BYTE      FT2SH
      02008053H   PUBLIC    XDATA    BYTE      FT1SH
      02008051H   PUBLIC    XDATA    BYTE      FT0SH
      02008042H   PUBLIC    XDATA    BYTE      OSTRIM
      0200807DH   PUBLIC    XDATA    BYTE      SMVTHL
      02008071H   PUBLIC    XDATA    BYTE      HDCT9
      02008070H   PUBLIC    XDATA    BYTE      HDCT8
      0200807EH   PUBLIC    XDATA    BYTE      SMVTHH
      0200806FH   PUBLIC    XDATA    BYTE      HDCT7
      0200806EH   PUBLIC    XDATA    BYTE      HDCT6
      0200806DH   PUBLIC    XDATA    BYTE      HDCT5
      0200806CH   PUBLIC    XDATA    BYTE      HDCT4
      0200806BH   PUBLIC    XDATA    BYTE      HDCT3
      0200806AH   PUBLIC    XDATA    BYTE      HDCT2
      02008069H   PUBLIC    XDATA    BYTE      HDCT1
      0200FC07H   PUBLIC    XDATA    BYTE      REPSET
      02008068H   PUBLIC    XDATA    BYTE      HDCT0
      02008110H   PUBLIC    XDATA    BYTE      TLCOMS
      02008060H   PUBLIC    XDATA    BYTE      MOTCON
      02008074H   PUBLIC    XDATA    BYTE      MOTPLC
      02008090H   PUBLIC    XDATA    BYTE      TKMAXF
      02008091H   PUBLIC    XDATA    BYTE      TKMINF
      0200810FH   PUBLIC    XDATA    BYTE      TLCNTD
      02008062H   PUBLIC    XDATA    BYTE      MTGCON
      0200807BH   PUBLIC    XDATA    BYTE      SMDATL
      02008058H   PUBLIC    XDATA    BYTE      CTMCON
      02008065H   PUBLIC    XDATA    BYTE      MOTCMD
      02008064H   PUBLIC    XDATA    BYTE      MFPCON
      0200FC05H   PUBLIC    XDATA    BYTE      PTSL
      02008041H   PUBLIC    XDATA    BYTE      OPBCON
      02008063H   PUBLIC    XDATA    BYTE      MHLCON
      0200807CH   PUBLIC    XDATA    BYTE      SMDATH
      02008040H   PUBLIC    XDATA    BYTE      OPACON
      02008061H   PUBLIC    XDATA    BYTE      MOTCFG
      0200FC06H   PUBLIC    XDATA    BYTE      PTSH
      02008106H   PUBLIC    XDATA    BYTE      TLEN
      02008085H   PUBLIC    XDATA    BYTE      ILCFGL
      0200808AH   PUBLIC    XDATA    BYTE      ACPDLL
      02008083H   PUBLIC    XDATA    BYTE      IHCFGL
      02008086H   PUBLIC    XDATA    BYTE      ILCFGH
      0200808BH   PUBLIC    XDATA    BYTE      ACPDLH
      0200808CH   PUBLIC    XDATA    BYTE      ACPDHL
      02008084H   PUBLIC    XDATA    BYTE      IHCFGH
      02008101H   PUBLIC    XDATA    BYTE      I2CIOS
      0200808DH   PUBLIC    XDATA    BYTE      ACPDHH
      0200FC03H   PUBLIC    XDATA    BYTE      LOCK
      0200804BH   PUBLIC    XDATA    BYTE      CP3CON
      0200804AH   PUBLIC    XDATA    BYTE      CP2CON
      02008049H   PUBLIC    XDATA    BYTE      CP1CON
      02008048H   PUBLIC    XDATA    BYTE      CP0CON
      02008059H   PUBLIC    XDATA    BYTE      CTMVTHL
      02008088H   PUBLIC    XDATA    BYTE      ADCALL
      0200805AH   PUBLIC    XDATA    BYTE      CTMVTHH
      0200810DH   PUBLIC    XDATA    BYTE      TLCNTLL
      02008089H   PUBLIC    XDATA    BYTE      ADCALH
      0200810BH   PUBLIC    XDATA    BYTE      TLCNTKL
      0200810EH   PUBLIC    XDATA    BYTE      TLCNTLH
LX51 LINKER/LOCATER V4.64.0.0                                                         04/13/2020  14:54:03  PAGE 20


      0200810CH   PUBLIC    XDATA    BYTE      TLCNTKH
      0200805BH   PUBLIC    XDATA    BYTE      CTMCNTL
      0200805CH   PUBLIC    XDATA    BYTE      CTMCNTH
      02008100H   PUBLIC    XDATA    BYTE      SPMAX
      02008103H   PUBLIC    XDATA    BYTE      TKPWC
      02008079H   PUBLIC    XDATA    BYTE      SMSTA
      0200811FH   PUBLIC    XDATA    BYTE      TPCTL
      02008073H   PUBLIC    XDATA    BYTE      HDCT11
      02008072H   PUBLIC    XDATA    BYTE      HDCT10
      0200807AH   PUBLIC    XDATA    BYTE      SMDIV
      02008037H   PUBLIC    XDATA    BYTE      P67F
      0200802FH   PUBLIC    XDATA    BYTE      P57F
      02008036H   PUBLIC    XDATA    BYTE      P66F
      0200803DH   PUBLIC    XDATA    BYTE      P75F
      0200810AH   PUBLIC    XDATA    BYTE      TLCKS
      02008027H   PUBLIC    XDATA    BYTE      P47F
      0200802EH   PUBLIC    XDATA    BYTE      P56F
      02008035H   PUBLIC    XDATA    BYTE      P65F
      0200803CH   PUBLIC    XDATA    BYTE      P74F
      0200804EH   PUBLIC    XDATA    BYTE      CPVTC
      02008078H   PUBLIC    XDATA    BYTE      SMCON
      02008108H   PUBLIC    XDATA    BYTE      TLCON
      0200801FH   PUBLIC    XDATA    BYTE      P37F
      02008026H   PUBLIC    XDATA    BYTE      P46F
      0200802DH   PUBLIC    XDATA    BYTE      P55F
      02008034H   PUBLIC    XDATA    BYTE      P64F
      0200803BH   PUBLIC    XDATA    BYTE      P73F
      02008067H   PUBLIC    XDATA    BYTE      MOTIF
      02008157H   PUBLIC    XDATA    BYTE      P67C
      02008017H   PUBLIC    XDATA    BYTE      P27F
      0200801EH   PUBLIC    XDATA    BYTE      P36F
      02008025H   PUBLIC    XDATA    BYTE      P45F
      0200802CH   PUBLIC    XDATA    BYTE      P54F
      02008033H   PUBLIC    XDATA    BYTE      P63F
      0200803AH   PUBLIC    XDATA    BYTE      P72F
      0200814FH   PUBLIC    XDATA    BYTE      P57C
      02008156H   PUBLIC    XDATA    BYTE      P66C
      0200815DH   PUBLIC    XDATA    BYTE      P75C
      0200800FH   PUBLIC    XDATA    BYTE      P17F
      02008016H   PUBLIC    XDATA    BYTE      P26F
      0200801DH   PUBLIC    XDATA    BYTE      P35F
      02008024H   PUBLIC    XDATA    BYTE      P44F
      0200802BH   PUBLIC    XDATA    BYTE      P53F
      02008032H   PUBLIC    XDATA    BYTE      P62F
      02008039H   PUBLIC    XDATA    BYTE      P71F
      0200811EH   PUBLIC    XDATA    BYTE      FTCTL
      02008147H   PUBLIC    XDATA    BYTE      P47C
      0200814EH   PUBLIC    XDATA    BYTE      P56C
      02008155H   PUBLIC    XDATA    BYTE      P65C
      0200815CH   PUBLIC    XDATA    BYTE      P74C
      01000046H   PUBLIC    CODE     ---       main
      010009BDH   PUBLIC    CODE     ---       SystemInit
      000000E3H   SFRSYM    DATA     BYTE      LXDAT
      000000C4H   SFRSYM    DATA     BYTE      TKCHS
      00000080H   SFRSYM    DATA     BYTE      P0
      000000C1H   SFRSYM    DATA     BYTE      TKCON
      00000090H   SFRSYM    DATA     BYTE      P1
      000000A0H   SFRSYM    DATA     BYTE      P2
      000000B0H   SFRSYM    DATA     BYTE      P3
      000000D0H.6 SFRSYM    DATA     BIT       AC
      000000C0H   SFRSYM    DATA     BYTE      P4
      000000D8H   SFRSYM    DATA     BYTE      P5
      000000A5H   SFRSYM    DATA     BYTE      SPCON
      000000A8H.7 SFRSYM    DATA     BIT       EA
      000000E1H   SFRSYM    DATA     BYTE      LXCON
LX51 LINKER/LOCATER V4.64.0.0                                                         04/13/2020  14:54:03  PAGE 21


      000000A9H   SFRSYM    DATA     BYTE      P6
      000000C8H   SFRSYM    DATA     BIT       T2P0
      000000D9H   SFRSYM    DATA     BYTE      P7
      000000C8H.1 SFRSYM    DATA     BIT       T2P1
      000000F1H   SFRSYM    DATA     BYTE      RTCON
      000000C8H.4 SFRSYM    DATA     BIT       T2R0
      000000DAH   SFRSYM    DATA     BYTE      PWMEN
      000000CFH   SFRSYM    DATA     BYTE      TKMSH
      00000086H   SFRSYM    DATA     BYTE      PWCON
      000000C8H.5 SFRSYM    DATA     BIT       T2R1
      000000CEH   SFRSYM    DATA     BYTE      TKMSL
      000000A7H   SFRSYM    DATA     BYTE      SPSTA
      00000083H   SFRSYM    DATA     BYTE      DP0H
      000000A8H   SFRSYM    DATA     BYTE      IE
      00000085H   SFRSYM    DATA     BYTE      DP1H
      000000E9H   SFRSYM    DATA     BYTE      RTCSS
      00000082H   SFRSYM    DATA     BYTE      DP0L
      000000CBH   SFRSYM    DATA     BYTE      T2CH
      000000B3H   SFRSYM    DATA     BYTE      I2CADM
      00000084H   SFRSYM    DATA     BYTE      DP1L
      000000C8H.3 SFRSYM    DATA     BIT       T2IE
      000000C3H   SFRSYM    DATA     BYTE      TKMTS
      000000CAH   SFRSYM    DATA     BYTE      T2CL
      000000B2H   SFRSYM    DATA     BYTE      I2CADR
      000000B4H   SFRSYM    DATA     BYTE      I2CCCR
      000000B8H   SFRSYM    DATA     BYTE      IP
      000000B7H   SFRSYM    DATA     BYTE      I2CFLG
      000000B5H   SFRSYM    DATA     BYTE      I2CDAT
      000000EDH   SFRSYM    DATA     BYTE      RTMSS
      000000D0H.7 SFRSYM    DATA     BIT       CY
      000000BBH   SFRSYM    DATA     BYTE      ADCFGH
      000000DCH   SFRSYM    DATA     BYTE      PWMCMAX
      000000B1H   SFRSYM    DATA     BYTE      I2CCON
      000000D1H   SFRSYM    DATA     BYTE      PWMDIVH
      000000BAH   SFRSYM    DATA     BYTE      ADCFGL
      00000081H   SFRSYM    DATA     BYTE      SP
      000000F9H   SFRSYM    DATA     BYTE      EPIE
      000000D0H.2 SFRSYM    DATA     BIT       OV
      000000FAH   SFRSYM    DATA     BYTE      EPIF
      000000DFH   SFRSYM    DATA     BYTE      PWMDIVL
      000000B6H   SFRSYM    DATA     BYTE      I2CSTA
      000000E8H   SFRSYM    DATA     BYTE      EXIE
      000000D3H   SFRSYM    DATA     BYTE      PWMDUTH
      000000C7H   SFRSYM    DATA     BYTE      TKIF
      0000008FH   SFRSYM    DATA     BYTE      IT0CON
      00000080H   SFRSYM    DATA     BIT       P00
      000000ECH   SFRSYM    DATA     BYTE      RTAH
      000000D2H   SFRSYM    DATA     BYTE      PWMDUTL
      0000008EH   SFRSYM    DATA     BYTE      IT1CON
      00000090H   SFRSYM    DATA     BIT       P10
      00000080H.1 SFRSYM    DATA     BIT       P01
      0000009DH   SFRSYM    DATA     BYTE      S1RELH
      00000087H   SFRSYM    DATA     BYTE      PCON
      000000A0H   SFRSYM    DATA     BIT       P20
      00000090H.1 SFRSYM    DATA     BIT       P11
      00000080H.2 SFRSYM    DATA     BIT       P02
      000000E8H   SFRSYM    DATA     BIT       INT2EN
      000000F4H   SFRSYM    DATA     BYTE      RTCH
      000000A4H   SFRSYM    DATA     BYTE      S2RELH
      000000B0H   SFRSYM    DATA     BIT       P30
      000000A0H.1 SFRSYM    DATA     BIT       P21
      00000090H.2 SFRSYM    DATA     BIT       P12
      00000080H.3 SFRSYM    DATA     BIT       P03
      000000E8H.1 SFRSYM    DATA     BIT       INT3EN
      000000C0H   SFRSYM    DATA     BIT       P40
LX51 LINKER/LOCATER V4.64.0.0                                                         04/13/2020  14:54:03  PAGE 22


      000000B0H.1 SFRSYM    DATA     BIT       P31
      000000A0H.2 SFRSYM    DATA     BIT       P22
      00000090H.3 SFRSYM    DATA     BIT       P13
      00000080H.4 SFRSYM    DATA     BIT       P04
      000000E8H.2 SFRSYM    DATA     BIT       INT4EN
      000000D8H   SFRSYM    DATA     BIT       P50
      000000C0H.1 SFRSYM    DATA     BIT       P41
      000000B0H.2 SFRSYM    DATA     BIT       P32
      000000A0H.3 SFRSYM    DATA     BIT       P23
      00000090H.4 SFRSYM    DATA     BIT       P14
      00000080H.5 SFRSYM    DATA     BIT       P05
      000000E8H.3 SFRSYM    DATA     BIT       INT5EN
      000000EBH   SFRSYM    DATA     BYTE      RTAM
      0000009CH   SFRSYM    DATA     BYTE      S1RELL
      00000089H   SFRSYM    DATA     BYTE      TMOD
      00000088H   SFRSYM    DATA     BYTE      TCON
      000000D8H.1 SFRSYM    DATA     BIT       P51
      000000C0H.2 SFRSYM    DATA     BIT       P42
      000000B0H.3 SFRSYM    DATA     BIT       P33
      000000A0H.4 SFRSYM    DATA     BIT       P24
      00000090H.5 SFRSYM    DATA     BIT       P15
      00000080H.6 SFRSYM    DATA     BIT       P06
      000000E8H.4 SFRSYM    DATA     BIT       INT6EN
      000000A3H   SFRSYM    DATA     BYTE      S2RELL
      000000D8H.2 SFRSYM    DATA     BIT       P52
      000000C0H.3 SFRSYM    DATA     BIT       P43
      000000B0H.4 SFRSYM    DATA     BIT       P34
      000000A0H.5 SFRSYM    DATA     BIT       P25
      00000090H.6 SFRSYM    DATA     BIT       P16
      00000080H.7 SFRSYM    DATA     BIT       P07
      000000E8H.5 SFRSYM    DATA     BIT       INT7EN
      000000C8H.2 SFRSYM    DATA     BIT       UCKS
      000000F8H   SFRSYM    DATA     BYTE      EXIP
      000000F3H   SFRSYM    DATA     BYTE      RTCM
      000000D8H.3 SFRSYM    DATA     BIT       P53
      000000C0H.4 SFRSYM    DATA     BIT       P44
      000000B0H.5 SFRSYM    DATA     BIT       P35
      000000A0H.6 SFRSYM    DATA     BIT       P26
      00000090H.7 SFRSYM    DATA     BIT       P17
      000000E8H.6 SFRSYM    DATA     BIT       INT8EN
      000000D8H.4 SFRSYM    DATA     BIT       P54
      000000C0H.5 SFRSYM    DATA     BIT       P45
      000000B0H.6 SFRSYM    DATA     BIT       P36
      000000A0H.7 SFRSYM    DATA     BIT       P27
      000000E8H.7 SFRSYM    DATA     BIT       INT9EN
      000000D8H.5 SFRSYM    DATA     BIT       P55
      000000C0H.6 SFRSYM    DATA     BIT       P46
      000000B0H.7 SFRSYM    DATA     BIT       P37
      000000D8H.6 SFRSYM    DATA     BIT       P56
      000000C0H.7 SFRSYM    DATA     BIT       P47
      000000EAH   SFRSYM    DATA     BYTE      RTAS
      000000AFH   SFRSYM    DATA     BYTE      HVTH
      00000095H   SFRSYM    DATA     BYTE      RCTAGH
      000000D8H.7 SFRSYM    DATA     BIT       P57
      000000F2H   SFRSYM    DATA     BYTE      RTCS
      00000088H.1 SFRSYM    DATA     BIT       IE0
      00000088H.3 SFRSYM    DATA     BIT       IE1
      00000094H   SFRSYM    DATA     BYTE      RCTAGL
      000000F0H   SFRSYM    DATA     BYTE      B
      000000E7H   SFRSYM    DATA     BYTE      MDUDAT
      000000DEH   SFRSYM    DATA     BYTE      PWMCFG
      000000D4H   SFRSYM    DATA     BYTE      PWMAIF
      000000E0H   SFRSYM    DATA     BYTE      ACC
      000000D5H   SFRSYM    DATA     BYTE      PWMBIF
      0000009FH   SFRSYM    DATA     BYTE      RCMSHH
LX51 LINKER/LOCATER V4.64.0.0                                                         04/13/2020  14:54:03  PAGE 23


      000000A8H.4 SFRSYM    DATA     BIT       ES0
      000000EFH   SFRSYM    DATA     BYTE      LVDCON
      000000E6H   SFRSYM    DATA     BYTE      MDUCON
      000000D6H   SFRSYM    DATA     BYTE      PWMCIF
      000000A8H.1 SFRSYM    DATA     BIT       ET0
      000000A8H.6 SFRSYM    DATA     BIT       ES1
      000000D7H   SFRSYM    DATA     BYTE      PWMDIF
      000000A8H.3 SFRSYM    DATA     BIT       ET1
      00000088H.5 SFRSYM    DATA     BIT       TF0
      000000FDH   SFRSYM    DATA     BYTE      IDLSTH
      000000AEH   SFRSYM    DATA     BYTE      PLLCON
      000000A8H.5 SFRSYM    DATA     BIT       ET2
      00000098H   SFRSYM    DATA     BIT       RI0
      00000088H.7 SFRSYM    DATA     BIT       TF1
      0000009EH   SFRSYM    DATA     BYTE      RCMSHL
      00000097H   SFRSYM    DATA     BYTE      RCMSLH
      000000C8H.7 SFRSYM    DATA     BIT       TF2
      00000098H.2 SFRSYM    DATA     BIT       RB8
      0000008CH   SFRSYM    DATA     BYTE      TH0
      000000A8H   SFRSYM    DATA     BIT       EX0
      00000098H.1 SFRSYM    DATA     BIT       TI0
      00000088H   SFRSYM    DATA     BIT       IT0
      0000008DH   SFRSYM    DATA     BYTE      TH1
      000000A8H.2 SFRSYM    DATA     BIT       EX1
      00000098H.3 SFRSYM    DATA     BIT       TB8
      00000088H.2 SFRSYM    DATA     BIT       IT1
      000000FCH   SFRSYM    DATA     BYTE      IDLSTL
      000000CDH   SFRSYM    DATA     BYTE      TH2
      000000D0H   SFRSYM    DATA     BIT       P
      00000096H   SFRSYM    DATA     BYTE      RCMSLL
      00000098H.7 SFRSYM    DATA     BIT       SM0
      0000008AH   SFRSYM    DATA     BYTE      TL0
      00000098H.6 SFRSYM    DATA     BIT       SM1
      000000E5H   SFRSYM    DATA     BYTE      LXDIVH
      0000008BH   SFRSYM    DATA     BYTE      TL1
      00000098H.5 SFRSYM    DATA     BIT       SM2
      000000CCH   SFRSYM    DATA     BYTE      TL2
      000000B8H.4 SFRSYM    DATA     BIT       PS0
      000000B8H.1 SFRSYM    DATA     BIT       PT0
      000000B8H.6 SFRSYM    DATA     BIT       PS1
      000000B8H.3 SFRSYM    DATA     BIT       PT1
      000000D0H.3 SFRSYM    DATA     BIT       RS0
      000000E4H   SFRSYM    DATA     BYTE      LXDIVL
      000000BDH   SFRSYM    DATA     BYTE      ADCDH
      000000B8H.5 SFRSYM    DATA     BIT       PT2
      00000088H.4 SFRSYM    DATA     BIT       TR0
      000000D0H.4 SFRSYM    DATA     BIT       RS1
      000000DDH   SFRSYM    DATA     BYTE      PWMCON
      00000088H.6 SFRSYM    DATA     BIT       TR1
      000000ADH   SFRSYM    DATA     BYTE      WDVTHH
      000000C8H.6 SFRSYM    DATA     BIT       TR2
      000000B8H   SFRSYM    DATA     BIT       PX0
      000000B8H.2 SFRSYM    DATA     BIT       PX1
      000000BCH   SFRSYM    DATA     BYTE      ADCDL
      000000ACH   SFRSYM    DATA     BYTE      WDVTHL
      000000DBH   SFRSYM    DATA     BYTE      PWMUPD
      00000099H   SFRSYM    DATA     BYTE      S0BUF
      0000009BH   SFRSYM    DATA     BYTE      S1BUF
      000000A2H   SFRSYM    DATA     BYTE      S2BUF
      00000098H   SFRSYM    DATA     BYTE      S0CON
      00000098H.4 SFRSYM    DATA     BIT       REN
      0000009AH   SFRSYM    DATA     BYTE      S1CON
      000000B9H   SFRSYM    DATA     BYTE      ADCON
      000000A1H   SFRSYM    DATA     BYTE      S2CON
      000000D0H.1 SFRSYM    DATA     BIT       DPS
LX51 LINKER/LOCATER V4.64.0.0                                                         04/13/2020  14:54:03  PAGE 24


      000000C9H   SFRSYM    DATA     BYTE      T2MOD
      000000C8H   SFRSYM    DATA     BYTE      T2CON
      000000FFH   SFRSYM    DATA     BYTE      STPSTH
      000000BFH   SFRSYM    DATA     BYTE      CKMIF
      000000FEH   SFRSYM    DATA     BYTE      STPSTL
      000000C2H   SFRSYM    DATA     BYTE      TKCFG
      00000093H   SFRSYM    DATA     BYTE      VCKDH
      000000D0H.5 SFRSYM    DATA     BIT       F0
      000000E2H   SFRSYM    DATA     BYTE      LXCFG
      000000ABH   SFRSYM    DATA     BYTE      WDFLG
      00000092H   SFRSYM    DATA     BYTE      VCKDL
      000000FBH   SFRSYM    DATA     BYTE      EPCON
      000000F6H   SFRSYM    DATA     BYTE      RTCDH
      000000C6H   SFRSYM    DATA     BYTE      ATKMH
      00000091H   SFRSYM    DATA     BYTE      RCCON
      000000F7H   SFRSYM    DATA     BYTE      INDEX
      000000EEH   SFRSYM    DATA     BYTE      RTCIF
      000000BEH   SFRSYM    DATA     BYTE      CKMON
      000000F5H   SFRSYM    DATA     BYTE      RTCDL
      000000D0H   SFRSYM    DATA     BYTE      PSW
      000000C5H   SFRSYM    DATA     BYTE      ATKML
      000000AAH   SFRSYM    DATA     BYTE      WDCON
      000000A6H   SFRSYM    DATA     BYTE      SPDAT

      010009BDH   BLOCK     CODE     ---       LVL=0
      010009BDH   LINE      CODE     ---       #45
      010009BDH   LINE      CODE     ---       #46
      010009BDH   LINE      CODE     ---       #48
      010009C0H   LINE      CODE     ---       #51
      010009C5H   LINE      CODE     ---       #64
      010009CCH   LINE      CODE     ---       #65
      010009CFH   LINE      CODE     ---       #71
      010009D2H   LINE      CODE     ---       #72
      010009D5H   LINE      CODE     ---       #73
      010009D8H   LINE      CODE     ---       #75
      ---         BLOCKEND  ---      ---       LVL=0

      01000046H   BLOCK     CODE     ---       LVL=0
      01000046H   LINE      CODE     ---       #76
      01000046H   LINE      CODE     ---       #77
      01000046H   LINE      CODE     ---       #78
      01000049H   LINE      CODE     ---       #79
      0100004BH   LINE      CODE     ---       #81
      0100004EH   LINE      CODE     ---       #82
      0100004EH   LINE      CODE     ---       #83
      0100004EH   LINE      CODE     ---       #84
      01000051H   LINE      CODE     ---       #95
      01000055H   LINE      CODE     ---       #96
      01000055H   LINE      CODE     ---       #97
      01000055H   LINE      CODE     ---       #98
      01000055H   LINE      CODE     ---       #99
      01000055H   LINE      CODE     ---       #100
      01000055H   LINE      CODE     ---       #101
      01000055H   LINE      CODE     ---       #102
      01000055H   LINE      CODE     ---       #103
      01000055H   LINE      CODE     ---       #104
      01000055H   LINE      CODE     ---       #106
      01000055H   LINE      CODE     ---       #107
      01000055H   LINE      CODE     ---       #108
      01000055H   LINE      CODE     ---       #109
      01000055H   LINE      CODE     ---       #140
      01000059H   LINE      CODE     ---       #141
      01000059H   LINE      CODE     ---       #142
      ---         BLOCKEND  ---      ---       LVL=0

LX51 LINKER/LOCATER V4.64.0.0                                                         04/13/2020  14:54:03  PAGE 25


      ---         MODULE    ---      ---       DELAY
      00000006H   SYMBOL    DATA     WORD      n
      00000003H   SYMBOL    DATA     BYTE      i
      00000082H   SYMBOL    DATA     WORD      n

      ---         MODULE    ---      ---       SYSTEM_CLOCK
      0100097AH   PUBLIC    CODE     ---       _Sys_Clk_Set_PLL
      000000E3H   SFRSYM    DATA     BYTE      LXDAT
      000000C4H   SFRSYM    DATA     BYTE      TKCHS
      00000080H   SFRSYM    DATA     BYTE      P0
      000000C1H   SFRSYM    DATA     BYTE      TKCON
      00000090H   SFRSYM    DATA     BYTE      P1
      000000A0H   SFRSYM    DATA     BYTE      P2
      000000B0H   SFRSYM    DATA     BYTE      P3
      000000D0H.6 SFRSYM    DATA     BIT       AC
      000000C0H   SFRSYM    DATA     BYTE      P4
      000000D8H   SFRSYM    DATA     BYTE      P5
      000000A5H   SFRSYM    DATA     BYTE      SPCON
      000000A8H.7 SFRSYM    DATA     BIT       EA
      000000E1H   SFRSYM    DATA     BYTE      LXCON
      000000A9H   SFRSYM    DATA     BYTE      P6
      000000C8H   SFRSYM    DATA     BIT       T2P0
      000000D9H   SFRSYM    DATA     BYTE      P7
      000000C8H.1 SFRSYM    DATA     BIT       T2P1
      000000F1H   SFRSYM    DATA     BYTE      RTCON
      000000C8H.4 SFRSYM    DATA     BIT       T2R0
      000000DAH   SFRSYM    DATA     BYTE      PWMEN
      000000CFH   SFRSYM    DATA     BYTE      TKMSH
      00000086H   SFRSYM    DATA     BYTE      PWCON
      000000C8H.5 SFRSYM    DATA     BIT       T2R1
      000000CEH   SFRSYM    DATA     BYTE      TKMSL
      000000A7H   SFRSYM    DATA     BYTE      SPSTA
      00000083H   SFRSYM    DATA     BYTE      DP0H
      000000A8H   SFRSYM    DATA     BYTE      IE
      00000085H   SFRSYM    DATA     BYTE      DP1H
      000000E9H   SFRSYM    DATA     BYTE      RTCSS
      00000082H   SFRSYM    DATA     BYTE      DP0L
      000000CBH   SFRSYM    DATA     BYTE      T2CH
      000000B3H   SFRSYM    DATA     BYTE      I2CADM
      00000084H   SFRSYM    DATA     BYTE      DP1L
      000000C8H.3 SFRSYM    DATA     BIT       T2IE
      000000C3H   SFRSYM    DATA     BYTE      TKMTS
      000000CAH   SFRSYM    DATA     BYTE      T2CL
      000000B2H   SFRSYM    DATA     BYTE      I2CADR
      000000B4H   SFRSYM    DATA     BYTE      I2CCCR
      000000B8H   SFRSYM    DATA     BYTE      IP
      000000B7H   SFRSYM    DATA     BYTE      I2CFLG
      000000B5H   SFRSYM    DATA     BYTE      I2CDAT
      000000EDH   SFRSYM    DATA     BYTE      RTMSS
      000000D0H.7 SFRSYM    DATA     BIT       CY
      000000BBH   SFRSYM    DATA     BYTE      ADCFGH
      000000DCH   SFRSYM    DATA     BYTE      PWMCMAX
      000000B1H   SFRSYM    DATA     BYTE      I2CCON
      000000D1H   SFRSYM    DATA     BYTE      PWMDIVH
      000000BAH   SFRSYM    DATA     BYTE      ADCFGL
      00000081H   SFRSYM    DATA     BYTE      SP
      000000F9H   SFRSYM    DATA     BYTE      EPIE
      000000D0H.2 SFRSYM    DATA     BIT       OV
      000000FAH   SFRSYM    DATA     BYTE      EPIF
      000000DFH   SFRSYM    DATA     BYTE      PWMDIVL
      000000B6H   SFRSYM    DATA     BYTE      I2CSTA
      000000E8H   SFRSYM    DATA     BYTE      EXIE
      000000D3H   SFRSYM    DATA     BYTE      PWMDUTH
      000000C7H   SFRSYM    DATA     BYTE      TKIF
      0000008FH   SFRSYM    DATA     BYTE      IT0CON
LX51 LINKER/LOCATER V4.64.0.0                                                         04/13/2020  14:54:03  PAGE 26


      00000080H   SFRSYM    DATA     BIT       P00
      000000ECH   SFRSYM    DATA     BYTE      RTAH
      000000D2H   SFRSYM    DATA     BYTE      PWMDUTL
      0000008EH   SFRSYM    DATA     BYTE      IT1CON
      00000090H   SFRSYM    DATA     BIT       P10
      00000080H.1 SFRSYM    DATA     BIT       P01
      0000009DH   SFRSYM    DATA     BYTE      S1RELH
      00000087H   SFRSYM    DATA     BYTE      PCON
      000000A0H   SFRSYM    DATA     BIT       P20
      00000090H.1 SFRSYM    DATA     BIT       P11
      00000080H.2 SFRSYM    DATA     BIT       P02
      000000E8H   SFRSYM    DATA     BIT       INT2EN
      000000F4H   SFRSYM    DATA     BYTE      RTCH
      000000A4H   SFRSYM    DATA     BYTE      S2RELH
      000000B0H   SFRSYM    DATA     BIT       P30
      000000A0H.1 SFRSYM    DATA     BIT       P21
      00000090H.2 SFRSYM    DATA     BIT       P12
      00000080H.3 SFRSYM    DATA     BIT       P03
      000000E8H.1 SFRSYM    DATA     BIT       INT3EN
      000000C0H   SFRSYM    DATA     BIT       P40
      000000B0H.1 SFRSYM    DATA     BIT       P31
      000000A0H.2 SFRSYM    DATA     BIT       P22
      00000090H.3 SFRSYM    DATA     BIT       P13
      00000080H.4 SFRSYM    DATA     BIT       P04
      000000E8H.2 SFRSYM    DATA     BIT       INT4EN
      000000D8H   SFRSYM    DATA     BIT       P50
      000000C0H.1 SFRSYM    DATA     BIT       P41
      000000B0H.2 SFRSYM    DATA     BIT       P32
      000000A0H.3 SFRSYM    DATA     BIT       P23
      00000090H.4 SFRSYM    DATA     BIT       P14
      00000080H.5 SFRSYM    DATA     BIT       P05
      000000E8H.3 SFRSYM    DATA     BIT       INT5EN
      000000EBH   SFRSYM    DATA     BYTE      RTAM
      0000009CH   SFRSYM    DATA     BYTE      S1RELL
      00000089H   SFRSYM    DATA     BYTE      TMOD
      00000088H   SFRSYM    DATA     BYTE      TCON
      000000D8H.1 SFRSYM    DATA     BIT       P51
      000000C0H.2 SFRSYM    DATA     BIT       P42
      000000B0H.3 SFRSYM    DATA     BIT       P33
      000000A0H.4 SFRSYM    DATA     BIT       P24
      00000090H.5 SFRSYM    DATA     BIT       P15
      00000080H.6 SFRSYM    DATA     BIT       P06
      000000E8H.4 SFRSYM    DATA     BIT       INT6EN
      000000A3H   SFRSYM    DATA     BYTE      S2RELL
      000000D8H.2 SFRSYM    DATA     BIT       P52
      000000C0H.3 SFRSYM    DATA     BIT       P43
      000000B0H.4 SFRSYM    DATA     BIT       P34
      000000A0H.5 SFRSYM    DATA     BIT       P25
      00000090H.6 SFRSYM    DATA     BIT       P16
      00000080H.7 SFRSYM    DATA     BIT       P07
      000000E8H.5 SFRSYM    DATA     BIT       INT7EN
      000000C8H.2 SFRSYM    DATA     BIT       UCKS
      000000F8H   SFRSYM    DATA     BYTE      EXIP
      000000F3H   SFRSYM    DATA     BYTE      RTCM
      000000D8H.3 SFRSYM    DATA     BIT       P53
      000000C0H.4 SFRSYM    DATA     BIT       P44
      000000B0H.5 SFRSYM    DATA     BIT       P35
      000000A0H.6 SFRSYM    DATA     BIT       P26
      00000090H.7 SFRSYM    DATA     BIT       P17
      000000E8H.6 SFRSYM    DATA     BIT       INT8EN
      000000D8H.4 SFRSYM    DATA     BIT       P54
      000000C0H.5 SFRSYM    DATA     BIT       P45
      000000B0H.6 SFRSYM    DATA     BIT       P36
      000000A0H.7 SFRSYM    DATA     BIT       P27
      000000E8H.7 SFRSYM    DATA     BIT       INT9EN
LX51 LINKER/LOCATER V4.64.0.0                                                         04/13/2020  14:54:03  PAGE 27


      000000D8H.5 SFRSYM    DATA     BIT       P55
      000000C0H.6 SFRSYM    DATA     BIT       P46
      000000B0H.7 SFRSYM    DATA     BIT       P37
      000000D8H.6 SFRSYM    DATA     BIT       P56
      000000C0H.7 SFRSYM    DATA     BIT       P47
      000000EAH   SFRSYM    DATA     BYTE      RTAS
      000000AFH   SFRSYM    DATA     BYTE      HVTH
      00000095H   SFRSYM    DATA     BYTE      RCTAGH
      000000D8H.7 SFRSYM    DATA     BIT       P57
      000000F2H   SFRSYM    DATA     BYTE      RTCS
      00000088H.1 SFRSYM    DATA     BIT       IE0
      00000088H.3 SFRSYM    DATA     BIT       IE1
      00000094H   SFRSYM    DATA     BYTE      RCTAGL
      000000F0H   SFRSYM    DATA     BYTE      B
      000000E7H   SFRSYM    DATA     BYTE      MDUDAT
      000000DEH   SFRSYM    DATA     BYTE      PWMCFG
      000000D4H   SFRSYM    DATA     BYTE      PWMAIF
      000000E0H   SFRSYM    DATA     BYTE      ACC
      000000D5H   SFRSYM    DATA     BYTE      PWMBIF
      0000009FH   SFRSYM    DATA     BYTE      RCMSHH
      000000A8H.4 SFRSYM    DATA     BIT       ES0
      000000EFH   SFRSYM    DATA     BYTE      LVDCON
      000000E6H   SFRSYM    DATA     BYTE      MDUCON
      000000D6H   SFRSYM    DATA     BYTE      PWMCIF
      000000A8H.1 SFRSYM    DATA     BIT       ET0
      000000A8H.6 SFRSYM    DATA     BIT       ES1
      000000D7H   SFRSYM    DATA     BYTE      PWMDIF
      000000A8H.3 SFRSYM    DATA     BIT       ET1
      00000088H.5 SFRSYM    DATA     BIT       TF0
      000000FDH   SFRSYM    DATA     BYTE      IDLSTH
      000000AEH   SFRSYM    DATA     BYTE      PLLCON
      000000A8H.5 SFRSYM    DATA     BIT       ET2
      00000098H   SFRSYM    DATA     BIT       RI0
      00000088H.7 SFRSYM    DATA     BIT       TF1
      0000009EH   SFRSYM    DATA     BYTE      RCMSHL
      00000097H   SFRSYM    DATA     BYTE      RCMSLH
      000000C8H.7 SFRSYM    DATA     BIT       TF2
      00000098H.2 SFRSYM    DATA     BIT       RB8
      0000008CH   SFRSYM    DATA     BYTE      TH0
      000000A8H   SFRSYM    DATA     BIT       EX0
      00000098H.1 SFRSYM    DATA     BIT       TI0
      00000088H   SFRSYM    DATA     BIT       IT0
      0000008DH   SFRSYM    DATA     BYTE      TH1
      000000A8H.2 SFRSYM    DATA     BIT       EX1
      00000098H.3 SFRSYM    DATA     BIT       TB8
      00000088H.2 SFRSYM    DATA     BIT       IT1
      000000FCH   SFRSYM    DATA     BYTE      IDLSTL
      000000CDH   SFRSYM    DATA     BYTE      TH2
      000000D0H   SFRSYM    DATA     BIT       P
      00000096H   SFRSYM    DATA     BYTE      RCMSLL
      00000098H.7 SFRSYM    DATA     BIT       SM0
      0000008AH   SFRSYM    DATA     BYTE      TL0
      00000098H.6 SFRSYM    DATA     BIT       SM1
      000000E5H   SFRSYM    DATA     BYTE      LXDIVH
      0000008BH   SFRSYM    DATA     BYTE      TL1
      00000098H.5 SFRSYM    DATA     BIT       SM2
      000000CCH   SFRSYM    DATA     BYTE      TL2
      000000B8H.4 SFRSYM    DATA     BIT       PS0
      000000B8H.1 SFRSYM    DATA     BIT       PT0
      000000B8H.6 SFRSYM    DATA     BIT       PS1
      000000B8H.3 SFRSYM    DATA     BIT       PT1
      000000D0H.3 SFRSYM    DATA     BIT       RS0
      000000E4H   SFRSYM    DATA     BYTE      LXDIVL
      000000BDH   SFRSYM    DATA     BYTE      ADCDH
      000000B8H.5 SFRSYM    DATA     BIT       PT2
LX51 LINKER/LOCATER V4.64.0.0                                                         04/13/2020  14:54:03  PAGE 28


      00000088H.4 SFRSYM    DATA     BIT       TR0
      000000D0H.4 SFRSYM    DATA     BIT       RS1
      000000DDH   SFRSYM    DATA     BYTE      PWMCON
      00000088H.6 SFRSYM    DATA     BIT       TR1
      000000ADH   SFRSYM    DATA     BYTE      WDVTHH
      000000C8H.6 SFRSYM    DATA     BIT       TR2
      000000B8H   SFRSYM    DATA     BIT       PX0
      000000B8H.2 SFRSYM    DATA     BIT       PX1
      000000BCH   SFRSYM    DATA     BYTE      ADCDL
      000000ACH   SFRSYM    DATA     BYTE      WDVTHL
      000000DBH   SFRSYM    DATA     BYTE      PWMUPD
      00000099H   SFRSYM    DATA     BYTE      S0BUF
      0000009BH   SFRSYM    DATA     BYTE      S1BUF
      000000A2H   SFRSYM    DATA     BYTE      S2BUF
      00000098H   SFRSYM    DATA     BYTE      S0CON
      00000098H.4 SFRSYM    DATA     BIT       REN
      0000009AH   SFRSYM    DATA     BYTE      S1CON
      000000B9H   SFRSYM    DATA     BYTE      ADCON
      000000A1H   SFRSYM    DATA     BYTE      S2CON
      000000D0H.1 SFRSYM    DATA     BIT       DPS
      000000C9H   SFRSYM    DATA     BYTE      T2MOD
      000000C8H   SFRSYM    DATA     BYTE      T2CON
      000000FFH   SFRSYM    DATA     BYTE      STPSTH
      000000BFH   SFRSYM    DATA     BYTE      CKMIF
      000000FEH   SFRSYM    DATA     BYTE      STPSTL
      000000C2H   SFRSYM    DATA     BYTE      TKCFG
      00000093H   SFRSYM    DATA     BYTE      VCKDH
      000000D0H.5 SFRSYM    DATA     BIT       F0
      000000E2H   SFRSYM    DATA     BYTE      LXCFG
      000000ABH   SFRSYM    DATA     BYTE      WDFLG
      00000092H   SFRSYM    DATA     BYTE      VCKDL
      000000FBH   SFRSYM    DATA     BYTE      EPCON
      000000F6H   SFRSYM    DATA     BYTE      RTCDH
      000000C6H   SFRSYM    DATA     BYTE      ATKMH
      00000091H   SFRSYM    DATA     BYTE      RCCON
      000000F7H   SFRSYM    DATA     BYTE      INDEX
      000000EEH   SFRSYM    DATA     BYTE      RTCIF
      000000BEH   SFRSYM    DATA     BYTE      CKMON
      000000F5H   SFRSYM    DATA     BYTE      RTCDL
      000000D0H   SFRSYM    DATA     BYTE      PSW
      000000C5H   SFRSYM    DATA     BYTE      ATKML
      000000AAH   SFRSYM    DATA     BYTE      WDCON
      000000A6H   SFRSYM    DATA     BYTE      SPDAT

      010009D9H   BLOCK     CODE     ---       LVL=0
      ---         BLOCKEND  ---      ---       LVL=0

      0100097AH   BLOCK     CODE     ---       LVL=0
      00000007H   SYMBOL    DATA     BYTE      Multiple
      0100097AH   LINE      CODE     ---       #69
      0100097AH   LINE      CODE     ---       #70
      0100097AH   LINE      CODE     ---       #71
      01000986H   LINE      CODE     ---       #73
      01000992H   LINE      CODE     ---       #74
      01000997H   LINE      CODE     ---       #75
      0100099DH   LINE      CODE     ---       #76
      ---         BLOCKEND  ---      ---       LVL=0

      ---         MODULE    ---      ---       UART
      000000E3H   SFRSYM    DATA     BYTE      LXDAT
      000000C4H   SFRSYM    DATA     BYTE      TKCHS
      00000080H   SFRSYM    DATA     BYTE      P0
      000000C1H   SFRSYM    DATA     BYTE      TKCON
      00000090H   SFRSYM    DATA     BYTE      P1
      000000A0H   SFRSYM    DATA     BYTE      P2
LX51 LINKER/LOCATER V4.64.0.0                                                         04/13/2020  14:54:03  PAGE 29


      000000B0H   SFRSYM    DATA     BYTE      P3
      000000D0H.6 SFRSYM    DATA     BIT       AC
      000000C0H   SFRSYM    DATA     BYTE      P4
      000000D8H   SFRSYM    DATA     BYTE      P5
      000000A5H   SFRSYM    DATA     BYTE      SPCON
      000000A8H.7 SFRSYM    DATA     BIT       EA
      000000E1H   SFRSYM    DATA     BYTE      LXCON
      000000A9H   SFRSYM    DATA     BYTE      P6
      000000C8H   SFRSYM    DATA     BIT       T2P0
      000000D9H   SFRSYM    DATA     BYTE      P7
      000000C8H.1 SFRSYM    DATA     BIT       T2P1
      000000F1H   SFRSYM    DATA     BYTE      RTCON
      000000C8H.4 SFRSYM    DATA     BIT       T2R0
      000000DAH   SFRSYM    DATA     BYTE      PWMEN
      000000CFH   SFRSYM    DATA     BYTE      TKMSH
      00000086H   SFRSYM    DATA     BYTE      PWCON
      000000C8H.5 SFRSYM    DATA     BIT       T2R1
      000000CEH   SFRSYM    DATA     BYTE      TKMSL
      000000A7H   SFRSYM    DATA     BYTE      SPSTA
      00000083H   SFRSYM    DATA     BYTE      DP0H
      000000A8H   SFRSYM    DATA     BYTE      IE
      00000085H   SFRSYM    DATA     BYTE      DP1H
      000000E9H   SFRSYM    DATA     BYTE      RTCSS
      00000082H   SFRSYM    DATA     BYTE      DP0L
      000000CBH   SFRSYM    DATA     BYTE      T2CH
      000000B3H   SFRSYM    DATA     BYTE      I2CADM
      00000084H   SFRSYM    DATA     BYTE      DP1L
      000000C8H.3 SFRSYM    DATA     BIT       T2IE
      000000C3H   SFRSYM    DATA     BYTE      TKMTS
      000000CAH   SFRSYM    DATA     BYTE      T2CL
      000000B2H   SFRSYM    DATA     BYTE      I2CADR
      000000B4H   SFRSYM    DATA     BYTE      I2CCCR
      000000B8H   SFRSYM    DATA     BYTE      IP
      000000B7H   SFRSYM    DATA     BYTE      I2CFLG
      000000B5H   SFRSYM    DATA     BYTE      I2CDAT
      000000EDH   SFRSYM    DATA     BYTE      RTMSS
      000000D0H.7 SFRSYM    DATA     BIT       CY
      000000BBH   SFRSYM    DATA     BYTE      ADCFGH
      000000DCH   SFRSYM    DATA     BYTE      PWMCMAX
      000000B1H   SFRSYM    DATA     BYTE      I2CCON
      000000D1H   SFRSYM    DATA     BYTE      PWMDIVH
      000000BAH   SFRSYM    DATA     BYTE      ADCFGL
      00000081H   SFRSYM    DATA     BYTE      SP
      000000F9H   SFRSYM    DATA     BYTE      EPIE
      000000D0H.2 SFRSYM    DATA     BIT       OV
      000000FAH   SFRSYM    DATA     BYTE      EPIF
      000000DFH   SFRSYM    DATA     BYTE      PWMDIVL
      000000B6H   SFRSYM    DATA     BYTE      I2CSTA
      000000E8H   SFRSYM    DATA     BYTE      EXIE
      000000D3H   SFRSYM    DATA     BYTE      PWMDUTH
      000000C7H   SFRSYM    DATA     BYTE      TKIF
      0000008FH   SFRSYM    DATA     BYTE      IT0CON
      00000080H   SFRSYM    DATA     BIT       P00
      000000ECH   SFRSYM    DATA     BYTE      RTAH
      000000D2H   SFRSYM    DATA     BYTE      PWMDUTL
      0000008EH   SFRSYM    DATA     BYTE      IT1CON
      00000090H   SFRSYM    DATA     BIT       P10
      00000080H.1 SFRSYM    DATA     BIT       P01
      0000009DH   SFRSYM    DATA     BYTE      S1RELH
      00000087H   SFRSYM    DATA     BYTE      PCON
      000000A0H   SFRSYM    DATA     BIT       P20
      00000090H.1 SFRSYM    DATA     BIT       P11
      00000080H.2 SFRSYM    DATA     BIT       P02
      000000E8H   SFRSYM    DATA     BIT       INT2EN
      000000F4H   SFRSYM    DATA     BYTE      RTCH
LX51 LINKER/LOCATER V4.64.0.0                                                         04/13/2020  14:54:03  PAGE 30


      000000A4H   SFRSYM    DATA     BYTE      S2RELH
      000000B0H   SFRSYM    DATA     BIT       P30
      000000A0H.1 SFRSYM    DATA     BIT       P21
      00000090H.2 SFRSYM    DATA     BIT       P12
      00000080H.3 SFRSYM    DATA     BIT       P03
      000000E8H.1 SFRSYM    DATA     BIT       INT3EN
      000000C0H   SFRSYM    DATA     BIT       P40
      000000B0H.1 SFRSYM    DATA     BIT       P31
      000000A0H.2 SFRSYM    DATA     BIT       P22
      00000090H.3 SFRSYM    DATA     BIT       P13
      00000080H.4 SFRSYM    DATA     BIT       P04
      000000E8H.2 SFRSYM    DATA     BIT       INT4EN
      000000D8H   SFRSYM    DATA     BIT       P50
      000000C0H.1 SFRSYM    DATA     BIT       P41
      000000B0H.2 SFRSYM    DATA     BIT       P32
      000000A0H.3 SFRSYM    DATA     BIT       P23
      00000090H.4 SFRSYM    DATA     BIT       P14
      00000080H.5 SFRSYM    DATA     BIT       P05
      000000E8H.3 SFRSYM    DATA     BIT       INT5EN
      000000EBH   SFRSYM    DATA     BYTE      RTAM
      0000009CH   SFRSYM    DATA     BYTE      S1RELL
      00000089H   SFRSYM    DATA     BYTE      TMOD
      00000088H   SFRSYM    DATA     BYTE      TCON
      000000D8H.1 SFRSYM    DATA     BIT       P51
      000000C0H.2 SFRSYM    DATA     BIT       P42
      000000B0H.3 SFRSYM    DATA     BIT       P33
      000000A0H.4 SFRSYM    DATA     BIT       P24
      00000090H.5 SFRSYM    DATA     BIT       P15
      00000080H.6 SFRSYM    DATA     BIT       P06
      000000E8H.4 SFRSYM    DATA     BIT       INT6EN
      000000A3H   SFRSYM    DATA     BYTE      S2RELL
      000000D8H.2 SFRSYM    DATA     BIT       P52
      000000C0H.3 SFRSYM    DATA     BIT       P43
      000000B0H.4 SFRSYM    DATA     BIT       P34
      000000A0H.5 SFRSYM    DATA     BIT       P25
      00000090H.6 SFRSYM    DATA     BIT       P16
      00000080H.7 SFRSYM    DATA     BIT       P07
      000000E8H.5 SFRSYM    DATA     BIT       INT7EN
      000000C8H.2 SFRSYM    DATA     BIT       UCKS
      000000F8H   SFRSYM    DATA     BYTE      EXIP
      000000F3H   SFRSYM    DATA     BYTE      RTCM
      000000D8H.3 SFRSYM    DATA     BIT       P53
      000000C0H.4 SFRSYM    DATA     BIT       P44
      000000B0H.5 SFRSYM    DATA     BIT       P35
      000000A0H.6 SFRSYM    DATA     BIT       P26
      00000090H.7 SFRSYM    DATA     BIT       P17
      000000E8H.6 SFRSYM    DATA     BIT       INT8EN
      000000D8H.4 SFRSYM    DATA     BIT       P54
      000000C0H.5 SFRSYM    DATA     BIT       P45
      000000B0H.6 SFRSYM    DATA     BIT       P36
      000000A0H.7 SFRSYM    DATA     BIT       P27
      000000E8H.7 SFRSYM    DATA     BIT       INT9EN
      000000D8H.5 SFRSYM    DATA     BIT       P55
      000000C0H.6 SFRSYM    DATA     BIT       P46
      000000B0H.7 SFRSYM    DATA     BIT       P37
      000000D8H.6 SFRSYM    DATA     BIT       P56
      000000C0H.7 SFRSYM    DATA     BIT       P47
      000000EAH   SFRSYM    DATA     BYTE      RTAS
      000000AFH   SFRSYM    DATA     BYTE      HVTH
      00000095H   SFRSYM    DATA     BYTE      RCTAGH
      000000D8H.7 SFRSYM    DATA     BIT       P57
      000000F2H   SFRSYM    DATA     BYTE      RTCS
      00000088H.1 SFRSYM    DATA     BIT       IE0
      00000088H.3 SFRSYM    DATA     BIT       IE1
      00000094H   SFRSYM    DATA     BYTE      RCTAGL
LX51 LINKER/LOCATER V4.64.0.0                                                         04/13/2020  14:54:03  PAGE 31


      000000F0H   SFRSYM    DATA     BYTE      B
      000000E7H   SFRSYM    DATA     BYTE      MDUDAT
      000000DEH   SFRSYM    DATA     BYTE      PWMCFG
      000000D4H   SFRSYM    DATA     BYTE      PWMAIF
      000000E0H   SFRSYM    DATA     BYTE      ACC
      000000D5H   SFRSYM    DATA     BYTE      PWMBIF
      0000009FH   SFRSYM    DATA     BYTE      RCMSHH
      000000A8H.4 SFRSYM    DATA     BIT       ES0
      000000EFH   SFRSYM    DATA     BYTE      LVDCON
      000000E6H   SFRSYM    DATA     BYTE      MDUCON
      000000D6H   SFRSYM    DATA     BYTE      PWMCIF
      000000A8H.1 SFRSYM    DATA     BIT       ET0
      000000A8H.6 SFRSYM    DATA     BIT       ES1
      000000D7H   SFRSYM    DATA     BYTE      PWMDIF
      000000A8H.3 SFRSYM    DATA     BIT       ET1
      00000088H.5 SFRSYM    DATA     BIT       TF0
      000000FDH   SFRSYM    DATA     BYTE      IDLSTH
      000000AEH   SFRSYM    DATA     BYTE      PLLCON
      000000A8H.5 SFRSYM    DATA     BIT       ET2
      00000098H   SFRSYM    DATA     BIT       RI0
      00000088H.7 SFRSYM    DATA     BIT       TF1
      0000009EH   SFRSYM    DATA     BYTE      RCMSHL
      00000097H   SFRSYM    DATA     BYTE      RCMSLH
      000000C8H.7 SFRSYM    DATA     BIT       TF2
      00000098H.2 SFRSYM    DATA     BIT       RB8
      0000008CH   SFRSYM    DATA     BYTE      TH0
      000000A8H   SFRSYM    DATA     BIT       EX0
      00000098H.1 SFRSYM    DATA     BIT       TI0
      00000088H   SFRSYM    DATA     BIT       IT0
      0000008DH   SFRSYM    DATA     BYTE      TH1
      000000A8H.2 SFRSYM    DATA     BIT       EX1
      00000098H.3 SFRSYM    DATA     BIT       TB8
      00000088H.2 SFRSYM    DATA     BIT       IT1
      000000FCH   SFRSYM    DATA     BYTE      IDLSTL
      000000CDH   SFRSYM    DATA     BYTE      TH2
      000000D0H   SFRSYM    DATA     BIT       P
      00000096H   SFRSYM    DATA     BYTE      RCMSLL
      00000098H.7 SFRSYM    DATA     BIT       SM0
      0000008AH   SFRSYM    DATA     BYTE      TL0
      00000098H.6 SFRSYM    DATA     BIT       SM1
      000000E5H   SFRSYM    DATA     BYTE      LXDIVH
      0000008BH   SFRSYM    DATA     BYTE      TL1
      00000098H.5 SFRSYM    DATA     BIT       SM2
      000000CCH   SFRSYM    DATA     BYTE      TL2
      000000B8H.4 SFRSYM    DATA     BIT       PS0
      000000B8H.1 SFRSYM    DATA     BIT       PT0
      000000B8H.6 SFRSYM    DATA     BIT       PS1
      000000B8H.3 SFRSYM    DATA     BIT       PT1
      000000D0H.3 SFRSYM    DATA     BIT       RS0
      000000E4H   SFRSYM    DATA     BYTE      LXDIVL
      000000BDH   SFRSYM    DATA     BYTE      ADCDH
      000000B8H.5 SFRSYM    DATA     BIT       PT2
      00000088H.4 SFRSYM    DATA     BIT       TR0
      000000D0H.4 SFRSYM    DATA     BIT       RS1
      000000DDH   SFRSYM    DATA     BYTE      PWMCON
      00000088H.6 SFRSYM    DATA     BIT       TR1
      000000ADH   SFRSYM    DATA     BYTE      WDVTHH
      000000C8H.6 SFRSYM    DATA     BIT       TR2
      000000B8H   SFRSYM    DATA     BIT       PX0
      000000B8H.2 SFRSYM    DATA     BIT       PX1
      000000BCH   SFRSYM    DATA     BYTE      ADCDL
      000000ACH   SFRSYM    DATA     BYTE      WDVTHL
      000000DBH   SFRSYM    DATA     BYTE      PWMUPD
      00000099H   SFRSYM    DATA     BYTE      S0BUF
      0000009BH   SFRSYM    DATA     BYTE      S1BUF
LX51 LINKER/LOCATER V4.64.0.0                                                         04/13/2020  14:54:03  PAGE 32


      000000A2H   SFRSYM    DATA     BYTE      S2BUF
      00000098H   SFRSYM    DATA     BYTE      S0CON
      00000098H.4 SFRSYM    DATA     BIT       REN
      0000009AH   SFRSYM    DATA     BYTE      S1CON
      000000B9H   SFRSYM    DATA     BYTE      ADCON
      000000A1H   SFRSYM    DATA     BYTE      S2CON
      000000D0H.1 SFRSYM    DATA     BIT       DPS
      000000C9H   SFRSYM    DATA     BYTE      T2MOD
      000000C8H   SFRSYM    DATA     BYTE      T2CON
      000000FFH   SFRSYM    DATA     BYTE      STPSTH
      000000BFH   SFRSYM    DATA     BYTE      CKMIF
      000000FEH   SFRSYM    DATA     BYTE      STPSTL
      000000C2H   SFRSYM    DATA     BYTE      TKCFG
      00000093H   SFRSYM    DATA     BYTE      VCKDH
      000000D0H.5 SFRSYM    DATA     BIT       F0
      000000E2H   SFRSYM    DATA     BYTE      LXCFG
      000000ABH   SFRSYM    DATA     BYTE      WDFLG
      00000092H   SFRSYM    DATA     BYTE      VCKDL
      000000FBH   SFRSYM    DATA     BYTE      EPCON
      000000F6H   SFRSYM    DATA     BYTE      RTCDH
      000000C6H   SFRSYM    DATA     BYTE      ATKMH
      00000091H   SFRSYM    DATA     BYTE      RCCON
      000000F7H   SFRSYM    DATA     BYTE      INDEX
      000000EEH   SFRSYM    DATA     BYTE      RTCIF
      000000BEH   SFRSYM    DATA     BYTE      CKMON
      000000F5H   SFRSYM    DATA     BYTE      RTCDL
      000000D0H   SFRSYM    DATA     BYTE      PSW
      000000C5H   SFRSYM    DATA     BYTE      ATKML
      000000AAH   SFRSYM    DATA     BYTE      WDCON
      000000A6H   SFRSYM    DATA     BYTE      SPDAT

      ---         MODULE    ---      ---       INTERRUPT
      01000003H   PUBLIC    CODE     ---       INT6_ISR
      0100084AH   PUBLIC    CODE     ---       INT3_ISR
      01000739H   PUBLIC    CODE     ---       INT8_ISR
      000000E3H   SFRSYM    DATA     BYTE      LXDAT
      000000C4H   SFRSYM    DATA     BYTE      TKCHS
      00000080H   SFRSYM    DATA     BYTE      P0
      000000C1H   SFRSYM    DATA     BYTE      TKCON
      00000090H   SFRSYM    DATA     BYTE      P1
      000000A0H   SFRSYM    DATA     BYTE      P2
      000000B0H   SFRSYM    DATA     BYTE      P3
      000000D0H.6 SFRSYM    DATA     BIT       AC
      000000C0H   SFRSYM    DATA     BYTE      P4
      000000D8H   SFRSYM    DATA     BYTE      P5
      000000A5H   SFRSYM    DATA     BYTE      SPCON
      000000A8H.7 SFRSYM    DATA     BIT       EA
      000000E1H   SFRSYM    DATA     BYTE      LXCON
      000000A9H   SFRSYM    DATA     BYTE      P6
      000000C8H   SFRSYM    DATA     BIT       T2P0
      000000D9H   SFRSYM    DATA     BYTE      P7
      000000C8H.1 SFRSYM    DATA     BIT       T2P1
      000000F1H   SFRSYM    DATA     BYTE      RTCON
      000000C8H.4 SFRSYM    DATA     BIT       T2R0
      000000DAH   SFRSYM    DATA     BYTE      PWMEN
      000000CFH   SFRSYM    DATA     BYTE      TKMSH
      00000086H   SFRSYM    DATA     BYTE      PWCON
      000000C8H.5 SFRSYM    DATA     BIT       T2R1
      000000CEH   SFRSYM    DATA     BYTE      TKMSL
      000000A7H   SFRSYM    DATA     BYTE      SPSTA
      00000083H   SFRSYM    DATA     BYTE      DP0H
      000000A8H   SFRSYM    DATA     BYTE      IE
      00000085H   SFRSYM    DATA     BYTE      DP1H
      000000E9H   SFRSYM    DATA     BYTE      RTCSS
      00000082H   SFRSYM    DATA     BYTE      DP0L
LX51 LINKER/LOCATER V4.64.0.0                                                         04/13/2020  14:54:03  PAGE 33


      000000CBH   SFRSYM    DATA     BYTE      T2CH
      000000B3H   SFRSYM    DATA     BYTE      I2CADM
      00000084H   SFRSYM    DATA     BYTE      DP1L
      000000C8H.3 SFRSYM    DATA     BIT       T2IE
      000000C3H   SFRSYM    DATA     BYTE      TKMTS
      000000CAH   SFRSYM    DATA     BYTE      T2CL
      000000B2H   SFRSYM    DATA     BYTE      I2CADR
      000000B4H   SFRSYM    DATA     BYTE      I2CCCR
      000000B8H   SFRSYM    DATA     BYTE      IP
      000000B7H   SFRSYM    DATA     BYTE      I2CFLG
      000000B5H   SFRSYM    DATA     BYTE      I2CDAT
      000000EDH   SFRSYM    DATA     BYTE      RTMSS
      000000D0H.7 SFRSYM    DATA     BIT       CY
      000000BBH   SFRSYM    DATA     BYTE      ADCFGH
      000000DCH   SFRSYM    DATA     BYTE      PWMCMAX
      000000B1H   SFRSYM    DATA     BYTE      I2CCON
      000000D1H   SFRSYM    DATA     BYTE      PWMDIVH
      000000BAH   SFRSYM    DATA     BYTE      ADCFGL
      00000081H   SFRSYM    DATA     BYTE      SP
      000000F9H   SFRSYM    DATA     BYTE      EPIE
      000000D0H.2 SFRSYM    DATA     BIT       OV
      000000FAH   SFRSYM    DATA     BYTE      EPIF
      000000DFH   SFRSYM    DATA     BYTE      PWMDIVL
      000000B6H   SFRSYM    DATA     BYTE      I2CSTA
      000000E8H   SFRSYM    DATA     BYTE      EXIE
      000000D3H   SFRSYM    DATA     BYTE      PWMDUTH
      000000C7H   SFRSYM    DATA     BYTE      TKIF
      0000008FH   SFRSYM    DATA     BYTE      IT0CON
      00000080H   SFRSYM    DATA     BIT       P00
      000000ECH   SFRSYM    DATA     BYTE      RTAH
      000000D2H   SFRSYM    DATA     BYTE      PWMDUTL
      0000008EH   SFRSYM    DATA     BYTE      IT1CON
      00000090H   SFRSYM    DATA     BIT       P10
      00000080H.1 SFRSYM    DATA     BIT       P01
      0000009DH   SFRSYM    DATA     BYTE      S1RELH
      00000087H   SFRSYM    DATA     BYTE      PCON
      000000A0H   SFRSYM    DATA     BIT       P20
      00000090H.1 SFRSYM    DATA     BIT       P11
      00000080H.2 SFRSYM    DATA     BIT       P02
      000000E8H   SFRSYM    DATA     BIT       INT2EN
      000000F4H   SFRSYM    DATA     BYTE      RTCH
      000000A4H   SFRSYM    DATA     BYTE      S2RELH
      000000B0H   SFRSYM    DATA     BIT       P30
      000000A0H.1 SFRSYM    DATA     BIT       P21
      00000090H.2 SFRSYM    DATA     BIT       P12
      00000080H.3 SFRSYM    DATA     BIT       P03
      000000E8H.1 SFRSYM    DATA     BIT       INT3EN
      000000C0H   SFRSYM    DATA     BIT       P40
      000000B0H.1 SFRSYM    DATA     BIT       P31
      000000A0H.2 SFRSYM    DATA     BIT       P22
      00000090H.3 SFRSYM    DATA     BIT       P13
      00000080H.4 SFRSYM    DATA     BIT       P04
      000000E8H.2 SFRSYM    DATA     BIT       INT4EN
      000000D8H   SFRSYM    DATA     BIT       P50
      000000C0H.1 SFRSYM    DATA     BIT       P41
      000000B0H.2 SFRSYM    DATA     BIT       P32
      000000A0H.3 SFRSYM    DATA     BIT       P23
      00000090H.4 SFRSYM    DATA     BIT       P14
      00000080H.5 SFRSYM    DATA     BIT       P05
      000000E8H.3 SFRSYM    DATA     BIT       INT5EN
      000000EBH   SFRSYM    DATA     BYTE      RTAM
      0000009CH   SFRSYM    DATA     BYTE      S1RELL
      00000089H   SFRSYM    DATA     BYTE      TMOD
      00000088H   SFRSYM    DATA     BYTE      TCON
      000000D8H.1 SFRSYM    DATA     BIT       P51
LX51 LINKER/LOCATER V4.64.0.0                                                         04/13/2020  14:54:03  PAGE 34


      000000C0H.2 SFRSYM    DATA     BIT       P42
      000000B0H.3 SFRSYM    DATA     BIT       P33
      000000A0H.4 SFRSYM    DATA     BIT       P24
      00000090H.5 SFRSYM    DATA     BIT       P15
      00000080H.6 SFRSYM    DATA     BIT       P06
      000000E8H.4 SFRSYM    DATA     BIT       INT6EN
      000000A3H   SFRSYM    DATA     BYTE      S2RELL
      000000D8H.2 SFRSYM    DATA     BIT       P52
      000000C0H.3 SFRSYM    DATA     BIT       P43
      000000B0H.4 SFRSYM    DATA     BIT       P34
      000000A0H.5 SFRSYM    DATA     BIT       P25
      00000090H.6 SFRSYM    DATA     BIT       P16
      00000080H.7 SFRSYM    DATA     BIT       P07
      000000E8H.5 SFRSYM    DATA     BIT       INT7EN
      000000C8H.2 SFRSYM    DATA     BIT       UCKS
      000000F8H   SFRSYM    DATA     BYTE      EXIP
      000000F3H   SFRSYM    DATA     BYTE      RTCM
      000000D8H.3 SFRSYM    DATA     BIT       P53
      000000C0H.4 SFRSYM    DATA     BIT       P44
      000000B0H.5 SFRSYM    DATA     BIT       P35
      000000A0H.6 SFRSYM    DATA     BIT       P26
      00000090H.7 SFRSYM    DATA     BIT       P17
      000000E8H.6 SFRSYM    DATA     BIT       INT8EN
      000000D8H.4 SFRSYM    DATA     BIT       P54
      000000C0H.5 SFRSYM    DATA     BIT       P45
      000000B0H.6 SFRSYM    DATA     BIT       P36
      000000A0H.7 SFRSYM    DATA     BIT       P27
      000000E8H.7 SFRSYM    DATA     BIT       INT9EN
      000000D8H.5 SFRSYM    DATA     BIT       P55
      000000C0H.6 SFRSYM    DATA     BIT       P46
      000000B0H.7 SFRSYM    DATA     BIT       P37
      000000D8H.6 SFRSYM    DATA     BIT       P56
      000000C0H.7 SFRSYM    DATA     BIT       P47
      000000EAH   SFRSYM    DATA     BYTE      RTAS
      000000AFH   SFRSYM    DATA     BYTE      HVTH
      00000095H   SFRSYM    DATA     BYTE      RCTAGH
      000000D8H.7 SFRSYM    DATA     BIT       P57
      000000F2H   SFRSYM    DATA     BYTE      RTCS
      00000088H.1 SFRSYM    DATA     BIT       IE0
      00000088H.3 SFRSYM    DATA     BIT       IE1
      00000094H   SFRSYM    DATA     BYTE      RCTAGL
      000000F0H   SFRSYM    DATA     BYTE      B
      000000E7H   SFRSYM    DATA     BYTE      MDUDAT
      000000DEH   SFRSYM    DATA     BYTE      PWMCFG
      000000D4H   SFRSYM    DATA     BYTE      PWMAIF
      000000E0H   SFRSYM    DATA     BYTE      ACC
      000000D5H   SFRSYM    DATA     BYTE      PWMBIF
      0000009FH   SFRSYM    DATA     BYTE      RCMSHH
      000000A8H.4 SFRSYM    DATA     BIT       ES0
      000000EFH   SFRSYM    DATA     BYTE      LVDCON
      000000E6H   SFRSYM    DATA     BYTE      MDUCON
      000000D6H   SFRSYM    DATA     BYTE      PWMCIF
      000000A8H.1 SFRSYM    DATA     BIT       ET0
      000000A8H.6 SFRSYM    DATA     BIT       ES1
      000000D7H   SFRSYM    DATA     BYTE      PWMDIF
      000000A8H.3 SFRSYM    DATA     BIT       ET1
      00000088H.5 SFRSYM    DATA     BIT       TF0
      000000FDH   SFRSYM    DATA     BYTE      IDLSTH
      000000AEH   SFRSYM    DATA     BYTE      PLLCON
      000000A8H.5 SFRSYM    DATA     BIT       ET2
      00000098H   SFRSYM    DATA     BIT       RI0
      00000088H.7 SFRSYM    DATA     BIT       TF1
      0000009EH   SFRSYM    DATA     BYTE      RCMSHL
      00000097H   SFRSYM    DATA     BYTE      RCMSLH
      000000C8H.7 SFRSYM    DATA     BIT       TF2
LX51 LINKER/LOCATER V4.64.0.0                                                         04/13/2020  14:54:03  PAGE 35


      00000098H.2 SFRSYM    DATA     BIT       RB8
      0000008CH   SFRSYM    DATA     BYTE      TH0
      000000A8H   SFRSYM    DATA     BIT       EX0
      00000098H.1 SFRSYM    DATA     BIT       TI0
      00000088H   SFRSYM    DATA     BIT       IT0
      0000008DH   SFRSYM    DATA     BYTE      TH1
      000000A8H.2 SFRSYM    DATA     BIT       EX1
      00000098H.3 SFRSYM    DATA     BIT       TB8
      00000088H.2 SFRSYM    DATA     BIT       IT1
      000000FCH   SFRSYM    DATA     BYTE      IDLSTL
      000000CDH   SFRSYM    DATA     BYTE      TH2
      000000D0H   SFRSYM    DATA     BIT       P
      00000096H   SFRSYM    DATA     BYTE      RCMSLL
      00000098H.7 SFRSYM    DATA     BIT       SM0
      0000008AH   SFRSYM    DATA     BYTE      TL0
      00000098H.6 SFRSYM    DATA     BIT       SM1
      000000E5H   SFRSYM    DATA     BYTE      LXDIVH
      0000008BH   SFRSYM    DATA     BYTE      TL1
      00000098H.5 SFRSYM    DATA     BIT       SM2
      000000CCH   SFRSYM    DATA     BYTE      TL2
      000000B8H.4 SFRSYM    DATA     BIT       PS0
      000000B8H.1 SFRSYM    DATA     BIT       PT0
      000000B8H.6 SFRSYM    DATA     BIT       PS1
      000000B8H.3 SFRSYM    DATA     BIT       PT1
      000000D0H.3 SFRSYM    DATA     BIT       RS0
      000000E4H   SFRSYM    DATA     BYTE      LXDIVL
      000000BDH   SFRSYM    DATA     BYTE      ADCDH
      000000B8H.5 SFRSYM    DATA     BIT       PT2
      00000088H.4 SFRSYM    DATA     BIT       TR0
      000000D0H.4 SFRSYM    DATA     BIT       RS1
      000000DDH   SFRSYM    DATA     BYTE      PWMCON
      00000088H.6 SFRSYM    DATA     BIT       TR1
      000000ADH   SFRSYM    DATA     BYTE      WDVTHH
      000000C8H.6 SFRSYM    DATA     BIT       TR2
      000000B8H   SFRSYM    DATA     BIT       PX0
      000000B8H.2 SFRSYM    DATA     BIT       PX1
      000000BCH   SFRSYM    DATA     BYTE      ADCDL
      000000ACH   SFRSYM    DATA     BYTE      WDVTHL
      000000DBH   SFRSYM    DATA     BYTE      PWMUPD
      00000099H   SFRSYM    DATA     BYTE      S0BUF
      0000009BH   SFRSYM    DATA     BYTE      S1BUF
      000000A2H   SFRSYM    DATA     BYTE      S2BUF
      00000098H   SFRSYM    DATA     BYTE      S0CON
      00000098H.4 SFRSYM    DATA     BIT       REN
      0000009AH   SFRSYM    DATA     BYTE      S1CON
      000000B9H   SFRSYM    DATA     BYTE      ADCON
      000000A1H   SFRSYM    DATA     BYTE      S2CON
      000000D0H.1 SFRSYM    DATA     BIT       DPS
      000000C9H   SFRSYM    DATA     BYTE      T2MOD
      000000C8H   SFRSYM    DATA     BYTE      T2CON
      000000FFH   SFRSYM    DATA     BYTE      STPSTH
      000000BFH   SFRSYM    DATA     BYTE      CKMIF
      000000FEH   SFRSYM    DATA     BYTE      STPSTL
      000000C2H   SFRSYM    DATA     BYTE      TKCFG
      00000093H   SFRSYM    DATA     BYTE      VCKDH
      000000D0H.5 SFRSYM    DATA     BIT       F0
      000000E2H   SFRSYM    DATA     BYTE      LXCFG
      000000ABH   SFRSYM    DATA     BYTE      WDFLG
      00000092H   SFRSYM    DATA     BYTE      VCKDL
      000000FBH   SFRSYM    DATA     BYTE      EPCON
      000000F6H   SFRSYM    DATA     BYTE      RTCDH
      000000C6H   SFRSYM    DATA     BYTE      ATKMH
      00000091H   SFRSYM    DATA     BYTE      RCCON
      000000F7H   SFRSYM    DATA     BYTE      INDEX
      000000EEH   SFRSYM    DATA     BYTE      RTCIF
LX51 LINKER/LOCATER V4.64.0.0                                                         04/13/2020  14:54:03  PAGE 36


      000000BEH   SFRSYM    DATA     BYTE      CKMON
      000000F5H   SFRSYM    DATA     BYTE      RTCDL
      000000D0H   SFRSYM    DATA     BYTE      PSW
      000000C5H   SFRSYM    DATA     BYTE      ATKML
      000000AAH   SFRSYM    DATA     BYTE      WDCON
      000000A6H   SFRSYM    DATA     BYTE      SPDAT

      01000739H   BLOCK     CODE     ---       LVL=0
      01000739H   LINE      CODE     ---       #24
      01000756H   LINE      CODE     ---       #26
      0100075BH   LINE      CODE     ---       #27
      0100075BH   LINE      CODE     ---       #28
      0100075EH   LINE      CODE     ---       #29
      01000761H   LINE      CODE     ---       #30
      01000767H   LINE      CODE     ---       #31
      01000767H   LINE      CODE     ---       #32
      0100076FH   LINE      CODE     ---       #33
      0100076FH   LINE      CODE     ---       #34
      0100076FH   LINE      CODE     ---       #35
      01000774H   LINE      CODE     ---       #36
      01000774H   LINE      CODE     ---       #37
      01000777H   LINE      CODE     ---       #38
      0100077AH   LINE      CODE     ---       #39
      0100077AH   LINE      CODE     ---       #40
      ---         BLOCKEND  ---      ---       LVL=0

      0100084AH   BLOCK     CODE     ---       LVL=0
      0100084AH   LINE      CODE     ---       #41
      01000867H   LINE      CODE     ---       #43
      0100086BH   LINE      CODE     ---       #44
      0100086BH   LINE      CODE     ---       #45
      0100086EH   LINE      CODE     ---       #46
      0100086EH   LINE      CODE     ---       #47
      ---         BLOCKEND  ---      ---       LVL=0

      01000003H   BLOCK     CODE     ---       LVL=0
      01000003H   LINE      CODE     ---       #48
      01000020H   LINE      CODE     ---       #51
      01000025H   LINE      CODE     ---       #52
      01000025H   LINE      CODE     ---       #53
      01000028H   LINE      CODE     ---       #54
      01000028H   LINE      CODE     ---       #56
      ---         BLOCKEND  ---      ---       LVL=0

      ---         MODULE    ---      ---       DEBUG
      00000031H   PUBLIC    DATA     BYTE      rxOffset
      00000030H   PUBLIC    DATA     BYTE      regAddr
      00000020H.3 PUBLIC    BIT      BIT       iicReadMode
      0000002DH   PUBLIC    DATA     ---       pTS_Info
      020000B2H   PUBLIC    XDATA    BYTE      TouchDebugID
      01000D30H   PUBLIC    CONST    ---       TS_INFO
      01000795H   PUBLIC    CODE     ---       Debug_ParamLoad
      0100099EH   PUBLIC    CODE     ---       Debug_init
      010005FDH   PUBLIC    CODE     ---       I2C_ISR
      000000E3H   SFRSYM    DATA     BYTE      LXDAT
      000000C4H   SFRSYM    DATA     BYTE      TKCHS
      00000080H   SFRSYM    DATA     BYTE      P0
      000000C1H   SFRSYM    DATA     BYTE      TKCON
      00000090H   SFRSYM    DATA     BYTE      P1
      000000A0H   SFRSYM    DATA     BYTE      P2
      000000B0H   SFRSYM    DATA     BYTE      P3
      000000D0H.6 SFRSYM    DATA     BIT       AC
      000000C0H   SFRSYM    DATA     BYTE      P4
      000000D8H   SFRSYM    DATA     BYTE      P5
      000000A5H   SFRSYM    DATA     BYTE      SPCON
LX51 LINKER/LOCATER V4.64.0.0                                                         04/13/2020  14:54:03  PAGE 37


      000000A8H.7 SFRSYM    DATA     BIT       EA
      000000E1H   SFRSYM    DATA     BYTE      LXCON
      000000A9H   SFRSYM    DATA     BYTE      P6
      000000C8H   SFRSYM    DATA     BIT       T2P0
      000000D9H   SFRSYM    DATA     BYTE      P7
      000000C8H.1 SFRSYM    DATA     BIT       T2P1
      000000F1H   SFRSYM    DATA     BYTE      RTCON
      000000C8H.4 SFRSYM    DATA     BIT       T2R0
      000000DAH   SFRSYM    DATA     BYTE      PWMEN
      000000CFH   SFRSYM    DATA     BYTE      TKMSH
      00000086H   SFRSYM    DATA     BYTE      PWCON
      000000C8H.5 SFRSYM    DATA     BIT       T2R1
      000000CEH   SFRSYM    DATA     BYTE      TKMSL
      000000A7H   SFRSYM    DATA     BYTE      SPSTA
      00000083H   SFRSYM    DATA     BYTE      DP0H
      000000A8H   SFRSYM    DATA     BYTE      IE
      00000085H   SFRSYM    DATA     BYTE      DP1H
      000000E9H   SFRSYM    DATA     BYTE      RTCSS
      00000082H   SFRSYM    DATA     BYTE      DP0L
      000000CBH   SFRSYM    DATA     BYTE      T2CH
      000000B3H   SFRSYM    DATA     BYTE      I2CADM
      00000084H   SFRSYM    DATA     BYTE      DP1L
      000000C8H.3 SFRSYM    DATA     BIT       T2IE
      000000C3H   SFRSYM    DATA     BYTE      TKMTS
      000000CAH   SFRSYM    DATA     BYTE      T2CL
      000000B2H   SFRSYM    DATA     BYTE      I2CADR
      000000B4H   SFRSYM    DATA     BYTE      I2CCCR
      000000B8H   SFRSYM    DATA     BYTE      IP
      000000B7H   SFRSYM    DATA     BYTE      I2CFLG
      000000B5H   SFRSYM    DATA     BYTE      I2CDAT
      000000EDH   SFRSYM    DATA     BYTE      RTMSS
      000000D0H.7 SFRSYM    DATA     BIT       CY
      000000BBH   SFRSYM    DATA     BYTE      ADCFGH
      000000DCH   SFRSYM    DATA     BYTE      PWMCMAX
      000000B1H   SFRSYM    DATA     BYTE      I2CCON
      000000D1H   SFRSYM    DATA     BYTE      PWMDIVH
      000000BAH   SFRSYM    DATA     BYTE      ADCFGL
      00000081H   SFRSYM    DATA     BYTE      SP
      000000F9H   SFRSYM    DATA     BYTE      EPIE
      000000D0H.2 SFRSYM    DATA     BIT       OV
      000000FAH   SFRSYM    DATA     BYTE      EPIF
      000000DFH   SFRSYM    DATA     BYTE      PWMDIVL
      000000B6H   SFRSYM    DATA     BYTE      I2CSTA
      000000E8H   SFRSYM    DATA     BYTE      EXIE
      000000D3H   SFRSYM    DATA     BYTE      PWMDUTH
      000000C7H   SFRSYM    DATA     BYTE      TKIF
      0000008FH   SFRSYM    DATA     BYTE      IT0CON
      00000080H   SFRSYM    DATA     BIT       P00
      000000ECH   SFRSYM    DATA     BYTE      RTAH
      000000D2H   SFRSYM    DATA     BYTE      PWMDUTL
      0000008EH   SFRSYM    DATA     BYTE      IT1CON
      00000090H   SFRSYM    DATA     BIT       P10
      00000080H.1 SFRSYM    DATA     BIT       P01
      0000009DH   SFRSYM    DATA     BYTE      S1RELH
      00000087H   SFRSYM    DATA     BYTE      PCON
      000000A0H   SFRSYM    DATA     BIT       P20
      00000090H.1 SFRSYM    DATA     BIT       P11
      00000080H.2 SFRSYM    DATA     BIT       P02
      000000E8H   SFRSYM    DATA     BIT       INT2EN
      000000F4H   SFRSYM    DATA     BYTE      RTCH
      000000A4H   SFRSYM    DATA     BYTE      S2RELH
      000000B0H   SFRSYM    DATA     BIT       P30
      000000A0H.1 SFRSYM    DATA     BIT       P21
      00000090H.2 SFRSYM    DATA     BIT       P12
      00000080H.3 SFRSYM    DATA     BIT       P03
LX51 LINKER/LOCATER V4.64.0.0                                                         04/13/2020  14:54:03  PAGE 38


      000000E8H.1 SFRSYM    DATA     BIT       INT3EN
      000000C0H   SFRSYM    DATA     BIT       P40
      000000B0H.1 SFRSYM    DATA     BIT       P31
      000000A0H.2 SFRSYM    DATA     BIT       P22
      00000090H.3 SFRSYM    DATA     BIT       P13
      00000080H.4 SFRSYM    DATA     BIT       P04
      000000E8H.2 SFRSYM    DATA     BIT       INT4EN
      000000D8H   SFRSYM    DATA     BIT       P50
      000000C0H.1 SFRSYM    DATA     BIT       P41
      000000B0H.2 SFRSYM    DATA     BIT       P32
      000000A0H.3 SFRSYM    DATA     BIT       P23
      00000090H.4 SFRSYM    DATA     BIT       P14
      00000080H.5 SFRSYM    DATA     BIT       P05
      000000E8H.3 SFRSYM    DATA     BIT       INT5EN
      000000EBH   SFRSYM    DATA     BYTE      RTAM
      0000009CH   SFRSYM    DATA     BYTE      S1RELL
      00000089H   SFRSYM    DATA     BYTE      TMOD
      00000088H   SFRSYM    DATA     BYTE      TCON
      000000D8H.1 SFRSYM    DATA     BIT       P51
      000000C0H.2 SFRSYM    DATA     BIT       P42
      000000B0H.3 SFRSYM    DATA     BIT       P33
      000000A0H.4 SFRSYM    DATA     BIT       P24
      00000090H.5 SFRSYM    DATA     BIT       P15
      00000080H.6 SFRSYM    DATA     BIT       P06
      000000E8H.4 SFRSYM    DATA     BIT       INT6EN
      000000A3H   SFRSYM    DATA     BYTE      S2RELL
      000000D8H.2 SFRSYM    DATA     BIT       P52
      000000C0H.3 SFRSYM    DATA     BIT       P43
      000000B0H.4 SFRSYM    DATA     BIT       P34
      000000A0H.5 SFRSYM    DATA     BIT       P25
      00000090H.6 SFRSYM    DATA     BIT       P16
      00000080H.7 SFRSYM    DATA     BIT       P07
      000000E8H.5 SFRSYM    DATA     BIT       INT7EN
      000000C8H.2 SFRSYM    DATA     BIT       UCKS
      000000F8H   SFRSYM    DATA     BYTE      EXIP
      000000F3H   SFRSYM    DATA     BYTE      RTCM
      000000D8H.3 SFRSYM    DATA     BIT       P53
      000000C0H.4 SFRSYM    DATA     BIT       P44
      000000B0H.5 SFRSYM    DATA     BIT       P35
      000000A0H.6 SFRSYM    DATA     BIT       P26
      00000090H.7 SFRSYM    DATA     BIT       P17
      000000E8H.6 SFRSYM    DATA     BIT       INT8EN
      000000D8H.4 SFRSYM    DATA     BIT       P54
      000000C0H.5 SFRSYM    DATA     BIT       P45
      000000B0H.6 SFRSYM    DATA     BIT       P36
      000000A0H.7 SFRSYM    DATA     BIT       P27
      000000E8H.7 SFRSYM    DATA     BIT       INT9EN
      000000D8H.5 SFRSYM    DATA     BIT       P55
      000000C0H.6 SFRSYM    DATA     BIT       P46
      000000B0H.7 SFRSYM    DATA     BIT       P37
      000000D8H.6 SFRSYM    DATA     BIT       P56
      000000C0H.7 SFRSYM    DATA     BIT       P47
      000000EAH   SFRSYM    DATA     BYTE      RTAS
      000000AFH   SFRSYM    DATA     BYTE      HVTH
      00000095H   SFRSYM    DATA     BYTE      RCTAGH
      000000D8H.7 SFRSYM    DATA     BIT       P57
      000000F2H   SFRSYM    DATA     BYTE      RTCS
      00000088H.1 SFRSYM    DATA     BIT       IE0
      00000088H.3 SFRSYM    DATA     BIT       IE1
      00000094H   SFRSYM    DATA     BYTE      RCTAGL
      000000F0H   SFRSYM    DATA     BYTE      B
      000000E7H   SFRSYM    DATA     BYTE      MDUDAT
      000000DEH   SFRSYM    DATA     BYTE      PWMCFG
      000000D4H   SFRSYM    DATA     BYTE      PWMAIF
      000000E0H   SFRSYM    DATA     BYTE      ACC
LX51 LINKER/LOCATER V4.64.0.0                                                         04/13/2020  14:54:03  PAGE 39


      000000D5H   SFRSYM    DATA     BYTE      PWMBIF
      0000009FH   SFRSYM    DATA     BYTE      RCMSHH
      000000A8H.4 SFRSYM    DATA     BIT       ES0
      000000EFH   SFRSYM    DATA     BYTE      LVDCON
      000000E6H   SFRSYM    DATA     BYTE      MDUCON
      000000D6H   SFRSYM    DATA     BYTE      PWMCIF
      000000A8H.1 SFRSYM    DATA     BIT       ET0
      000000A8H.6 SFRSYM    DATA     BIT       ES1
      000000D7H   SFRSYM    DATA     BYTE      PWMDIF
      000000A8H.3 SFRSYM    DATA     BIT       ET1
      00000088H.5 SFRSYM    DATA     BIT       TF0
      000000FDH   SFRSYM    DATA     BYTE      IDLSTH
      000000AEH   SFRSYM    DATA     BYTE      PLLCON
      000000A8H.5 SFRSYM    DATA     BIT       ET2
      00000098H   SFRSYM    DATA     BIT       RI0
      00000088H.7 SFRSYM    DATA     BIT       TF1
      0000009EH   SFRSYM    DATA     BYTE      RCMSHL
      00000097H   SFRSYM    DATA     BYTE      RCMSLH
      000000C8H.7 SFRSYM    DATA     BIT       TF2
      00000098H.2 SFRSYM    DATA     BIT       RB8
      0000008CH   SFRSYM    DATA     BYTE      TH0
      000000A8H   SFRSYM    DATA     BIT       EX0
      00000098H.1 SFRSYM    DATA     BIT       TI0
      00000088H   SFRSYM    DATA     BIT       IT0
      0000008DH   SFRSYM    DATA     BYTE      TH1
      000000A8H.2 SFRSYM    DATA     BIT       EX1
      00000098H.3 SFRSYM    DATA     BIT       TB8
      00000088H.2 SFRSYM    DATA     BIT       IT1
      000000FCH   SFRSYM    DATA     BYTE      IDLSTL
      000000CDH   SFRSYM    DATA     BYTE      TH2
      000000D0H   SFRSYM    DATA     BIT       P
      00000096H   SFRSYM    DATA     BYTE      RCMSLL
      00000098H.7 SFRSYM    DATA     BIT       SM0
      0000008AH   SFRSYM    DATA     BYTE      TL0
      00000098H.6 SFRSYM    DATA     BIT       SM1
      000000E5H   SFRSYM    DATA     BYTE      LXDIVH
      0000008BH   SFRSYM    DATA     BYTE      TL1
      00000098H.5 SFRSYM    DATA     BIT       SM2
      000000CCH   SFRSYM    DATA     BYTE      TL2
      000000B8H.4 SFRSYM    DATA     BIT       PS0
      000000B8H.1 SFRSYM    DATA     BIT       PT0
      000000B8H.6 SFRSYM    DATA     BIT       PS1
      000000B8H.3 SFRSYM    DATA     BIT       PT1
      000000D0H.3 SFRSYM    DATA     BIT       RS0
      000000E4H   SFRSYM    DATA     BYTE      LXDIVL
      000000BDH   SFRSYM    DATA     BYTE      ADCDH
      000000B8H.5 SFRSYM    DATA     BIT       PT2
      00000088H.4 SFRSYM    DATA     BIT       TR0
      000000D0H.4 SFRSYM    DATA     BIT       RS1
      000000DDH   SFRSYM    DATA     BYTE      PWMCON
      00000088H.6 SFRSYM    DATA     BIT       TR1
      000000ADH   SFRSYM    DATA     BYTE      WDVTHH
      000000C8H.6 SFRSYM    DATA     BIT       TR2
      000000B8H   SFRSYM    DATA     BIT       PX0
      000000B8H.2 SFRSYM    DATA     BIT       PX1
      000000BCH   SFRSYM    DATA     BYTE      ADCDL
      000000ACH   SFRSYM    DATA     BYTE      WDVTHL
      000000DBH   SFRSYM    DATA     BYTE      PWMUPD
      00000099H   SFRSYM    DATA     BYTE      S0BUF
      0000009BH   SFRSYM    DATA     BYTE      S1BUF
      000000A2H   SFRSYM    DATA     BYTE      S2BUF
      00000098H   SFRSYM    DATA     BYTE      S0CON
      00000098H.4 SFRSYM    DATA     BIT       REN
      0000009AH   SFRSYM    DATA     BYTE      S1CON
      000000B9H   SFRSYM    DATA     BYTE      ADCON
LX51 LINKER/LOCATER V4.64.0.0                                                         04/13/2020  14:54:03  PAGE 40


      000000A1H   SFRSYM    DATA     BYTE      S2CON
      000000D0H.1 SFRSYM    DATA     BIT       DPS
      000000C9H   SFRSYM    DATA     BYTE      T2MOD
      000000C8H   SFRSYM    DATA     BYTE      T2CON
      000000FFH   SFRSYM    DATA     BYTE      STPSTH
      000000BFH   SFRSYM    DATA     BYTE      CKMIF
      000000FEH   SFRSYM    DATA     BYTE      STPSTL
      000000C2H   SFRSYM    DATA     BYTE      TKCFG
      00000093H   SFRSYM    DATA     BYTE      VCKDH
      000000D0H.5 SFRSYM    DATA     BIT       F0
      000000E2H   SFRSYM    DATA     BYTE      LXCFG
      000000ABH   SFRSYM    DATA     BYTE      WDFLG
      00000092H   SFRSYM    DATA     BYTE      VCKDL
      000000FBH   SFRSYM    DATA     BYTE      EPCON
      000000F6H   SFRSYM    DATA     BYTE      RTCDH
      000000C6H   SFRSYM    DATA     BYTE      ATKMH
      00000091H   SFRSYM    DATA     BYTE      RCCON
      000000F7H   SFRSYM    DATA     BYTE      INDEX
      000000EEH   SFRSYM    DATA     BYTE      RTCIF
      000000BEH   SFRSYM    DATA     BYTE      CKMON
      000000F5H   SFRSYM    DATA     BYTE      RTCDL
      000000D0H   SFRSYM    DATA     BYTE      PSW
      000000C5H   SFRSYM    DATA     BYTE      ATKML
      000000AAH   SFRSYM    DATA     BYTE      WDCON
      000000A6H   SFRSYM    DATA     BYTE      SPDAT

      0100005EH   BLOCK     CODE     ---       LVL=0
      ---         BLOCKEND  ---      ---       LVL=0

      010005FDH   BLOCK     CODE     ---       LVL=0
      010005FDH   BLOCK     CODE     NEAR LAB  LVL=1
      00000007H   SYMBOL    DATA     BYTE      Sta_Temp
      ---         BLOCKEND  ---      ---       LVL=1
      010005FDH   LINE      CODE     ---       #48
      010005FDH   LINE      CODE     ---       #49
      010005FDH   LINE      CODE     ---       #51
      01000603H   LINE      CODE     ---       #52
      01000605H   LINE      CODE     ---       #53
      01000608H   LINE      CODE     ---       #54
      01000608H   LINE      CODE     ---       #55
      0100060BH   LINE      CODE     ---       #56
      0100060DH   LINE      CODE     ---       #57
      0100060DH   LINE      CODE     ---       #58
      0100060FH   LINE      CODE     ---       #59
      01000614H   LINE      CODE     ---       #60
      01000614H   LINE      CODE     ---       #61
      01000617H   LINE      CODE     ---       #62
      01000617H   LINE      CODE     ---       #63
      01000619H   LINE      CODE     ---       #64
      01000623H   LINE      CODE     ---       #65
      01000625H   LINE      CODE     ---       #67
      01000625H   LINE      CODE     ---       #68
      0100062AH   LINE      CODE     ---       #69
      0100062AH   LINE      CODE     ---       #70
      0100062DH   LINE      CODE     ---       #71
      01000645H   LINE      CODE     ---       #72
      01000648H   LINE      CODE     ---       #73
      01000648H   LINE      CODE     ---       #74
      0100064AH   LINE      CODE     ---       #76
      0100064AH   LINE      CODE     ---       #77
      01000655H   LINE      CODE     ---       #78
      01000657H   LINE      CODE     ---       #79
      0100065AH   LINE      CODE     ---       #80
      0100065AH   LINE      CODE     ---       #81
      0100065AH   LINE      CODE     ---       #82
LX51 LINKER/LOCATER V4.64.0.0                                                         04/13/2020  14:54:03  PAGE 41


      0100065CH   LINE      CODE     ---       #83
      0100065FH   LINE      CODE     ---       #84
      0100065FH   LINE      CODE     ---       #85
      0100066AH   LINE      CODE     ---       #86
      0100066CH   LINE      CODE     ---       #87
      0100066CH   LINE      CODE     ---       #88
      0100066CH   LINE      CODE     ---       #89
      0100066CH   LINE      CODE     ---       #90
      0100066CH   LINE      CODE     ---       #91
      0100066FH   LINE      CODE     ---       #92
      ---         BLOCKEND  ---      ---       LVL=0

      0100099EH   BLOCK     CODE     ---       LVL=0
      0100099EH   LINE      CODE     ---       #93
      0100099EH   LINE      CODE     ---       #94
      0100099EH   LINE      CODE     ---       #100
      010009A4H   LINE      CODE     ---       #101
      010009AAH   LINE      CODE     ---       #102
      010009AEH   LINE      CODE     ---       #113
      010009B1H   LINE      CODE     ---       #114
      010009B4H   LINE      CODE     ---       #115
      010009B7H   LINE      CODE     ---       #117
      010009B9H   LINE      CODE     ---       #118
      010009BCH   LINE      CODE     ---       #119
      ---         BLOCKEND  ---      ---       LVL=0

      01000795H   BLOCK     CODE     ---       LVL=0
      01000795H   BLOCK     CODE     NEAR LAB  LVL=1
      00000007H   SYMBOL    DATA     BYTE      i
      ---         BLOCKEND  ---      ---       LVL=1
      01000795H   LINE      CODE     ---       #120
      01000795H   LINE      CODE     ---       #121
      01000795H   LINE      CODE     ---       #123
      010007A4H   LINE      CODE     ---       #124
      010007ABH   LINE      CODE     ---       #125
      010007B1H   LINE      CODE     ---       #126
      010007B3H   LINE      CODE     ---       #127
      010007B3H   LINE      CODE     ---       #128
      010007C5H   LINE      CODE     ---       #129
      010007C9H   LINE      CODE     ---       #130
      010007D8H   LINE      CODE     ---       #131
      010007E7H   LINE      CODE     ---       #132
      ---         BLOCKEND  ---      ---       LVL=0

      ---         MODULE    ---      ---       TS_API
      020000B1H   PUBLIC    XDATA    BYTE      Key_Cnt_Debug
      020000AFH   PUBLIC    XDATA    WORD      WheelSliderCapRateFilter
      0000003BH   PUBLIC    IDATA    BYTE      PreKeysFlagSN
      00000020H.2 PUBLIC    BIT      BIT       TS_StableFlag
      020000A9H   PUBLIC    XDATA    ---       TS_CH_Debug
      020000A3H   PUBLIC    XDATA    ---       TS_AreaConfirmTimer
      020000A1H   PUBLIC    XDATA    WORD      TS_RefChBaseLineData
      020000A0H   PUBLIC    XDATA    BYTE      TS_State_Debug
      0200009AH   PUBLIC    XDATA    ---       TSKey_LongTouchLimitTimer
      02000093H   PUBLIC    XDATA    ---       TS_FilterPosIdx
      02000091H   PUBLIC    XDATA    WORD      TS_RefPostData
      0000002BH   PUBLIC    DATA     WORD      TS_LongKeyTimer
      02000090H   PUBLIC    XDATA    BYTE      TS_HalfSecCnt
      0000003AH   PUBLIC    IDATA    BYTE      TS_RefCHBaseLineAdjuTimer
      0200008FH   PUBLIC    XDATA    BYTE      KeysFlagSN
      0200008EH   PUBLIC    XDATA    BYTE      EnterStopScanTimer
      02000082H   PUBLIC    XDATA    ---       TSKey_FingerThd
      00000029H   PUBLIC    DATA     WORD      TS_Key
      00000028H   PUBLIC    DATA     BYTE      TS_BaseCh
      02000074H   PUBLIC    XDATA    ---       TS_RawData
LX51 LINKER/LOCATER V4.64.0.0                                                         04/13/2020  14:54:03  PAGE 42


      02000073H   PUBLIC    XDATA    BYTE      WheelSliderMaxIdx
      00000039H   PUBLIC    IDATA    BYTE      TS_Cnt
      02000065H   PUBLIC    XDATA    ---       TS_PostData
      02000064H   PUBLIC    XDATA    BYTE      WheelSliderRefCh
      02000063H   PUBLIC    XDATA    BYTE      TS_Init_Step
      00000033H   PUBLIC    IDATA    ---       TS_CH
      0200001DH   PUBLIC    XDATA    ---       TS_FilterBuf
      02000011H   PUBLIC    XDATA    ---       TS_BaseLineData
      00000032H   PUBLIC    IDATA    BYTE      TS_State
      02000005H   PUBLIC    XDATA    ---       TS_FirstAreaData
      00000027H   PUBLIC    DATA     BYTE      ActiveTouchType
      00000020H.1 PUBLIC    BIT      BIT       TS_CycleScanDoneFlag
      02000001H   PUBLIC    XDATA    DWORD     KeysFlagSN_Debug
      00000026H   PUBLIC    DATA     BYTE      TK_State
      00000025H   PUBLIC    DATA     BYTE      TS_Index
      01000D18H   PUBLIC    CONST    ---       TS_KEY_TAB
      01000D13H   PUBLIC    CONST    ---       AREA_CONFIRM_TIME_TAB
      01000D0DH   PUBLIC    CONST    ---       MASK_TAB
      01000D0CH   PUBLIC    CONST    ---       WHEEL_SLIDER0_MAX_MIN_TAB
      01000CF4H   PUBLIC    CONST    ---       TS_KEY_CH_INFO_SEQ
      01000572H   PUBLIC    CODE     ---       TS_GetKey
      01000889H   PUBLIC    CODE     ---       TS_Action
      01000670H   PUBLIC    CODE     ---       TS_init
      0100018FH   PUBLIC    CODE     ---       TSKey_DataDeal
      01000291H   PUBLIC    CODE     ---       TS_RunInit
      01000357H   PUBLIC    CODE     ---       TS_DataFiltering
      010004C4H   PUBLIC    CODE     ---       TS_ISR
      0100094DH   PUBLIC    CODE     ---       TS_HS_ISR
      010008F1H   PUBLIC    CODE     ---       TS_MS_ISR
      000000E3H   SFRSYM    DATA     BYTE      LXDAT
      000000C4H   SFRSYM    DATA     BYTE      TKCHS
      00000080H   SFRSYM    DATA     BYTE      P0
      000000C1H   SFRSYM    DATA     BYTE      TKCON
      00000090H   SFRSYM    DATA     BYTE      P1
      000000A0H   SFRSYM    DATA     BYTE      P2
      000000B0H   SFRSYM    DATA     BYTE      P3
      000000D0H.6 SFRSYM    DATA     BIT       AC
      000000C0H   SFRSYM    DATA     BYTE      P4
      000000D8H   SFRSYM    DATA     BYTE      P5
      000000A5H   SFRSYM    DATA     BYTE      SPCON
      000000A8H.7 SFRSYM    DATA     BIT       EA
      000000E1H   SFRSYM    DATA     BYTE      LXCON
      000000A9H   SFRSYM    DATA     BYTE      P6
      000000C8H   SFRSYM    DATA     BIT       T2P0
      000000D9H   SFRSYM    DATA     BYTE      P7
      000000C8H.1 SFRSYM    DATA     BIT       T2P1
      000000F1H   SFRSYM    DATA     BYTE      RTCON
      000000C8H.4 SFRSYM    DATA     BIT       T2R0
      000000DAH   SFRSYM    DATA     BYTE      PWMEN
      000000CFH   SFRSYM    DATA     BYTE      TKMSH
      00000086H   SFRSYM    DATA     BYTE      PWCON
      000000C8H.5 SFRSYM    DATA     BIT       T2R1
      000000CEH   SFRSYM    DATA     BYTE      TKMSL
      000000A7H   SFRSYM    DATA     BYTE      SPSTA
      00000083H   SFRSYM    DATA     BYTE      DP0H
      000000A8H   SFRSYM    DATA     BYTE      IE
      00000085H   SFRSYM    DATA     BYTE      DP1H
      000000E9H   SFRSYM    DATA     BYTE      RTCSS
      00000082H   SFRSYM    DATA     BYTE      DP0L
      000000CBH   SFRSYM    DATA     BYTE      T2CH
      000000B3H   SFRSYM    DATA     BYTE      I2CADM
      00000084H   SFRSYM    DATA     BYTE      DP1L
      000000C8H.3 SFRSYM    DATA     BIT       T2IE
      000000C3H   SFRSYM    DATA     BYTE      TKMTS
      000000CAH   SFRSYM    DATA     BYTE      T2CL
LX51 LINKER/LOCATER V4.64.0.0                                                         04/13/2020  14:54:03  PAGE 43


      000000B2H   SFRSYM    DATA     BYTE      I2CADR
      000000B4H   SFRSYM    DATA     BYTE      I2CCCR
      000000B8H   SFRSYM    DATA     BYTE      IP
      000000B7H   SFRSYM    DATA     BYTE      I2CFLG
      000000B5H   SFRSYM    DATA     BYTE      I2CDAT
      000000EDH   SFRSYM    DATA     BYTE      RTMSS
      000000D0H.7 SFRSYM    DATA     BIT       CY
      000000BBH   SFRSYM    DATA     BYTE      ADCFGH
      000000DCH   SFRSYM    DATA     BYTE      PWMCMAX
      000000B1H   SFRSYM    DATA     BYTE      I2CCON
      000000D1H   SFRSYM    DATA     BYTE      PWMDIVH
      000000BAH   SFRSYM    DATA     BYTE      ADCFGL
      00000081H   SFRSYM    DATA     BYTE      SP
      000000F9H   SFRSYM    DATA     BYTE      EPIE
      000000D0H.2 SFRSYM    DATA     BIT       OV
      000000FAH   SFRSYM    DATA     BYTE      EPIF
      000000DFH   SFRSYM    DATA     BYTE      PWMDIVL
      000000B6H   SFRSYM    DATA     BYTE      I2CSTA
      000000E8H   SFRSYM    DATA     BYTE      EXIE
      000000D3H   SFRSYM    DATA     BYTE      PWMDUTH
      000000C7H   SFRSYM    DATA     BYTE      TKIF
      0000008FH   SFRSYM    DATA     BYTE      IT0CON
      00000080H   SFRSYM    DATA     BIT       P00
      000000ECH   SFRSYM    DATA     BYTE      RTAH
      000000D2H   SFRSYM    DATA     BYTE      PWMDUTL
      0000008EH   SFRSYM    DATA     BYTE      IT1CON
      00000090H   SFRSYM    DATA     BIT       P10
      00000080H.1 SFRSYM    DATA     BIT       P01
      0000009DH   SFRSYM    DATA     BYTE      S1RELH
      00000087H   SFRSYM    DATA     BYTE      PCON
      000000A0H   SFRSYM    DATA     BIT       P20
      00000090H.1 SFRSYM    DATA     BIT       P11
      00000080H.2 SFRSYM    DATA     BIT       P02
      000000E8H   SFRSYM    DATA     BIT       INT2EN
      000000F4H   SFRSYM    DATA     BYTE      RTCH
      000000A4H   SFRSYM    DATA     BYTE      S2RELH
      000000B0H   SFRSYM    DATA     BIT       P30
      000000A0H.1 SFRSYM    DATA     BIT       P21
      00000090H.2 SFRSYM    DATA     BIT       P12
      00000080H.3 SFRSYM    DATA     BIT       P03
      000000E8H.1 SFRSYM    DATA     BIT       INT3EN
      000000C0H   SFRSYM    DATA     BIT       P40
      000000B0H.1 SFRSYM    DATA     BIT       P31
      000000A0H.2 SFRSYM    DATA     BIT       P22
      00000090H.3 SFRSYM    DATA     BIT       P13
      00000080H.4 SFRSYM    DATA     BIT       P04
      000000E8H.2 SFRSYM    DATA     BIT       INT4EN
      000000D8H   SFRSYM    DATA     BIT       P50
      000000C0H.1 SFRSYM    DATA     BIT       P41
      000000B0H.2 SFRSYM    DATA     BIT       P32
      000000A0H.3 SFRSYM    DATA     BIT       P23
      00000090H.4 SFRSYM    DATA     BIT       P14
      00000080H.5 SFRSYM    DATA     BIT       P05
      000000E8H.3 SFRSYM    DATA     BIT       INT5EN
      000000EBH   SFRSYM    DATA     BYTE      RTAM
      0000009CH   SFRSYM    DATA     BYTE      S1RELL
      00000089H   SFRSYM    DATA     BYTE      TMOD
      00000088H   SFRSYM    DATA     BYTE      TCON
      000000D8H.1 SFRSYM    DATA     BIT       P51
      000000C0H.2 SFRSYM    DATA     BIT       P42
      000000B0H.3 SFRSYM    DATA     BIT       P33
      000000A0H.4 SFRSYM    DATA     BIT       P24
      00000090H.5 SFRSYM    DATA     BIT       P15
      00000080H.6 SFRSYM    DATA     BIT       P06
      000000E8H.4 SFRSYM    DATA     BIT       INT6EN
LX51 LINKER/LOCATER V4.64.0.0                                                         04/13/2020  14:54:03  PAGE 44


      000000A3H   SFRSYM    DATA     BYTE      S2RELL
      000000D8H.2 SFRSYM    DATA     BIT       P52
      000000C0H.3 SFRSYM    DATA     BIT       P43
      000000B0H.4 SFRSYM    DATA     BIT       P34
      000000A0H.5 SFRSYM    DATA     BIT       P25
      00000090H.6 SFRSYM    DATA     BIT       P16
      00000080H.7 SFRSYM    DATA     BIT       P07
      000000E8H.5 SFRSYM    DATA     BIT       INT7EN
      000000C8H.2 SFRSYM    DATA     BIT       UCKS
      000000F8H   SFRSYM    DATA     BYTE      EXIP
      000000F3H   SFRSYM    DATA     BYTE      RTCM
      000000D8H.3 SFRSYM    DATA     BIT       P53
      000000C0H.4 SFRSYM    DATA     BIT       P44
      000000B0H.5 SFRSYM    DATA     BIT       P35
      000000A0H.6 SFRSYM    DATA     BIT       P26
      00000090H.7 SFRSYM    DATA     BIT       P17
      000000E8H.6 SFRSYM    DATA     BIT       INT8EN
      000000D8H.4 SFRSYM    DATA     BIT       P54
      000000C0H.5 SFRSYM    DATA     BIT       P45
      000000B0H.6 SFRSYM    DATA     BIT       P36
      000000A0H.7 SFRSYM    DATA     BIT       P27
      000000E8H.7 SFRSYM    DATA     BIT       INT9EN
      000000D8H.5 SFRSYM    DATA     BIT       P55
      000000C0H.6 SFRSYM    DATA     BIT       P46
      000000B0H.7 SFRSYM    DATA     BIT       P37
      000000D8H.6 SFRSYM    DATA     BIT       P56
      000000C0H.7 SFRSYM    DATA     BIT       P47
      000000EAH   SFRSYM    DATA     BYTE      RTAS
      000000AFH   SFRSYM    DATA     BYTE      HVTH
      00000095H   SFRSYM    DATA     BYTE      RCTAGH
      000000D8H.7 SFRSYM    DATA     BIT       P57
      000000F2H   SFRSYM    DATA     BYTE      RTCS
      00000088H.1 SFRSYM    DATA     BIT       IE0
      00000088H.3 SFRSYM    DATA     BIT       IE1
      00000094H   SFRSYM    DATA     BYTE      RCTAGL
      000000F0H   SFRSYM    DATA     BYTE      B
      000000E7H   SFRSYM    DATA     BYTE      MDUDAT
      000000DEH   SFRSYM    DATA     BYTE      PWMCFG
      000000D4H   SFRSYM    DATA     BYTE      PWMAIF
      000000E0H   SFRSYM    DATA     BYTE      ACC
      000000D5H   SFRSYM    DATA     BYTE      PWMBIF
      0000009FH   SFRSYM    DATA     BYTE      RCMSHH
      000000A8H.4 SFRSYM    DATA     BIT       ES0
      000000EFH   SFRSYM    DATA     BYTE      LVDCON
      000000E6H   SFRSYM    DATA     BYTE      MDUCON
      000000D6H   SFRSYM    DATA     BYTE      PWMCIF
      000000A8H.1 SFRSYM    DATA     BIT       ET0
      000000A8H.6 SFRSYM    DATA     BIT       ES1
      000000D7H   SFRSYM    DATA     BYTE      PWMDIF
      000000A8H.3 SFRSYM    DATA     BIT       ET1
      00000088H.5 SFRSYM    DATA     BIT       TF0
      000000FDH   SFRSYM    DATA     BYTE      IDLSTH
      000000AEH   SFRSYM    DATA     BYTE      PLLCON
      000000A8H.5 SFRSYM    DATA     BIT       ET2
      00000098H   SFRSYM    DATA     BIT       RI0
      00000088H.7 SFRSYM    DATA     BIT       TF1
      0000009EH   SFRSYM    DATA     BYTE      RCMSHL
      00000097H   SFRSYM    DATA     BYTE      RCMSLH
      000000C8H.7 SFRSYM    DATA     BIT       TF2
      00000098H.2 SFRSYM    DATA     BIT       RB8
      0000008CH   SFRSYM    DATA     BYTE      TH0
      000000A8H   SFRSYM    DATA     BIT       EX0
      00000098H.1 SFRSYM    DATA     BIT       TI0
      00000088H   SFRSYM    DATA     BIT       IT0
      0000008DH   SFRSYM    DATA     BYTE      TH1
LX51 LINKER/LOCATER V4.64.0.0                                                         04/13/2020  14:54:03  PAGE 45


      000000A8H.2 SFRSYM    DATA     BIT       EX1
      00000098H.3 SFRSYM    DATA     BIT       TB8
      00000088H.2 SFRSYM    DATA     BIT       IT1
      000000FCH   SFRSYM    DATA     BYTE      IDLSTL
      000000CDH   SFRSYM    DATA     BYTE      TH2
      000000D0H   SFRSYM    DATA     BIT       P
      00000096H   SFRSYM    DATA     BYTE      RCMSLL
      00000098H.7 SFRSYM    DATA     BIT       SM0
      0000008AH   SFRSYM    DATA     BYTE      TL0
      00000098H.6 SFRSYM    DATA     BIT       SM1
      000000E5H   SFRSYM    DATA     BYTE      LXDIVH
      0000008BH   SFRSYM    DATA     BYTE      TL1
      00000098H.5 SFRSYM    DATA     BIT       SM2
      000000CCH   SFRSYM    DATA     BYTE      TL2
      000000B8H.4 SFRSYM    DATA     BIT       PS0
      000000B8H.1 SFRSYM    DATA     BIT       PT0
      000000B8H.6 SFRSYM    DATA     BIT       PS1
      000000B8H.3 SFRSYM    DATA     BIT       PT1
      000000D0H.3 SFRSYM    DATA     BIT       RS0
      000000E4H   SFRSYM    DATA     BYTE      LXDIVL
      000000BDH   SFRSYM    DATA     BYTE      ADCDH
      000000B8H.5 SFRSYM    DATA     BIT       PT2
      00000088H.4 SFRSYM    DATA     BIT       TR0
      000000D0H.4 SFRSYM    DATA     BIT       RS1
      000000DDH   SFRSYM    DATA     BYTE      PWMCON
      00000088H.6 SFRSYM    DATA     BIT       TR1
      000000ADH   SFRSYM    DATA     BYTE      WDVTHH
      000000C8H.6 SFRSYM    DATA     BIT       TR2
      000000B8H   SFRSYM    DATA     BIT       PX0
      000000B8H.2 SFRSYM    DATA     BIT       PX1
      000000BCH   SFRSYM    DATA     BYTE      ADCDL
      000000ACH   SFRSYM    DATA     BYTE      WDVTHL
      000000DBH   SFRSYM    DATA     BYTE      PWMUPD
      00000099H   SFRSYM    DATA     BYTE      S0BUF
      0000009BH   SFRSYM    DATA     BYTE      S1BUF
      000000A2H   SFRSYM    DATA     BYTE      S2BUF
      00000098H   SFRSYM    DATA     BYTE      S0CON
      00000098H.4 SFRSYM    DATA     BIT       REN
      0000009AH   SFRSYM    DATA     BYTE      S1CON
      000000B9H   SFRSYM    DATA     BYTE      ADCON
      000000A1H   SFRSYM    DATA     BYTE      S2CON
      000000D0H.1 SFRSYM    DATA     BIT       DPS
      000000C9H   SFRSYM    DATA     BYTE      T2MOD
      000000C8H   SFRSYM    DATA     BYTE      T2CON
      000000FFH   SFRSYM    DATA     BYTE      STPSTH
      000000BFH   SFRSYM    DATA     BYTE      CKMIF
      000000FEH   SFRSYM    DATA     BYTE      STPSTL
      000000C2H   SFRSYM    DATA     BYTE      TKCFG
      00000093H   SFRSYM    DATA     BYTE      VCKDH
      000000D0H.5 SFRSYM    DATA     BIT       F0
      000000E2H   SFRSYM    DATA     BYTE      LXCFG
      000000ABH   SFRSYM    DATA     BYTE      WDFLG
      00000092H   SFRSYM    DATA     BYTE      VCKDL
      000000FBH   SFRSYM    DATA     BYTE      EPCON
      000000F6H   SFRSYM    DATA     BYTE      RTCDH
      000000C6H   SFRSYM    DATA     BYTE      ATKMH
      00000091H   SFRSYM    DATA     BYTE      RCCON
      000000F7H   SFRSYM    DATA     BYTE      INDEX
      000000EEH   SFRSYM    DATA     BYTE      RTCIF
      000000BEH   SFRSYM    DATA     BYTE      CKMON
      000000F5H   SFRSYM    DATA     BYTE      RTCDL
      000000D0H   SFRSYM    DATA     BYTE      PSW
      000000C5H   SFRSYM    DATA     BYTE      ATKML
      000000AAH   SFRSYM    DATA     BYTE      WDCON
      000000A6H   SFRSYM    DATA     BYTE      SPDAT
LX51 LINKER/LOCATER V4.64.0.0                                                         04/13/2020  14:54:03  PAGE 46



      01000411H   BLOCK     CODE     ---       LVL=0
      ---         BLOCKEND  ---      ---       LVL=0

      010008F1H   BLOCK     CODE     ---       LVL=0
      010008F1H   BLOCK     CODE     NEAR LAB  LVL=1
      02000000H   SYMBOL    XDATA    BYTE      ms_cnt
      00000007H   SYMBOL    DATA     BYTE      i
      ---         BLOCKEND  ---      ---       LVL=1
      010008F1H   LINE      CODE     ---       #137
      010008F1H   LINE      CODE     ---       #138
      010008F1H   LINE      CODE     ---       #142
      010008F7H   LINE      CODE     ---       #143
      010008FDH   LINE      CODE     ---       #144
      010008FDH   LINE      CODE     ---       #145
      010008FFH   LINE      CODE     ---       #146
      01000909H   LINE      CODE     ---       #147
      01000909H   LINE      CODE     ---       #148
      01000912H   LINE      CODE     ---       #149
      01000912H   LINE      CODE     ---       #150
      0100091BH   LINE      CODE     ---       #151
      0100091BH   LINE      CODE     ---       #152
      0100091EH   LINE      CODE     ---       #168
      0100091EH   LINE      CODE     ---       #169
      ---         BLOCKEND  ---      ---       LVL=0

      0100094DH   BLOCK     CODE     ---       LVL=0
      0100094DH   BLOCK     CODE     NEAR LAB  LVL=1
      00000007H   SYMBOL    DATA     BYTE      i
      ---         BLOCKEND  ---      ---       LVL=1
      0100094DH   LINE      CODE     ---       #170
      0100094DH   LINE      CODE     ---       #171
      0100094DH   LINE      CODE     ---       #177
      01000953H   LINE      CODE     ---       #186
      01000955H   LINE      CODE     ---       #187
      01000955H   LINE      CODE     ---       #188
      0100095EH   LINE      CODE     ---       #189
      0100095EH   LINE      CODE     ---       #190
      01000967H   LINE      CODE     ---       #191
      01000967H   LINE      CODE     ---       #192
      0100096BH   LINE      CODE     ---       #203
      01000970H   LINE      CODE     ---       #204
      01000970H   LINE      CODE     ---       #205
      01000971H   LINE      CODE     ---       #206
      01000971H   LINE      CODE     ---       #207
      01000977H   LINE      CODE     ---       #208
      01000977H   LINE      CODE     ---       #209
      01000979H   LINE      CODE     ---       #210
      01000979H   LINE      CODE     ---       #211
      ---         BLOCKEND  ---      ---       LVL=0

      010004C4H   BLOCK     CODE     ---       LVL=0
      010004C4H   BLOCK     CODE     NEAR LAB  LVL=1
      00000008H   SYMBOL    DATA     BYTE      index_copy
      00000005H   SYMBOL    DATA     BYTE      i
      00000009H   SYMBOL    DATA     ---       TS_Data
      ---         BLOCKEND  ---      ---       LVL=1
      010004C4H   LINE      CODE     ---       #212
      010004C4H   LINE      CODE     ---       #213
      010004C4H   LINE      CODE     ---       #223
      010004CCH   LINE      CODE     ---       #224
      010004CCH   LINE      CODE     ---       #225
      010004D0H   LINE      CODE     ---       #226
      010004D0H   LINE      CODE     ---       #227
      010004D3H   LINE      CODE     ---       #228
LX51 LINKER/LOCATER V4.64.0.0                                                         04/13/2020  14:54:03  PAGE 47


      010004D5H   LINE      CODE     ---       #229
      010004D5H   LINE      CODE     ---       #230
      010004EEH   LINE      CODE     ---       #231
      010004EEH   LINE      CODE     ---       #232
      010004FBH   LINE      CODE     ---       #233
      010004FDH   LINE      CODE     ---       #234
      01000505H   LINE      CODE     ---       #235
      0100050DH   LINE      CODE     ---       #236
      0100050DH   LINE      CODE     ---       #237
      01000511H   LINE      CODE     ---       #238
      01000513H   LINE      CODE     ---       #239
      01000513H   LINE      CODE     ---       #272
      01000513H   LINE      CODE     ---       #274
      01000527H   LINE      CODE     ---       #278
      01000527H   LINE      CODE     ---       #279
      01000539H   LINE      CODE     ---       #280
      01000539H   LINE      CODE     ---       #281
      01000539H   LINE      CODE     ---       #282
      01000539H   LINE      CODE     ---       #283
      0100053DH   LINE      CODE     ---       #312
      01000553H   LINE      CODE     ---       #313
      01000553H   LINE      CODE     ---       #315
      01000555H   LINE      CODE     ---       #329
      01000558H   LINE      CODE     ---       #330
      0100055AH   LINE      CODE     ---       #332
      0100055AH   LINE      CODE     ---       #333
      01000560H   LINE      CODE     ---       #334
      01000560H   LINE      CODE     ---       #335
      01000563H   LINE      CODE     ---       #336
      0100056BH   LINE      CODE     ---       #337
      0100056EH   LINE      CODE     ---       #338
      01000571H   LINE      CODE     ---       #339
      ---         BLOCKEND  ---      ---       LVL=0

      01000357H   BLOCK     CODE     ---       LVL=0
      01000357H   BLOCK     CODE     NEAR LAB  LVL=1
      00000015H   SYMBOL    DATA     BYTE      i
      00000007H   SYMBOL    DATA     BYTE      j
      00000016H   SYMBOL    DATA     WORD      DataSum
      00000018H   SYMBOL    DATA     WORD      DataMax
      0000001AH   SYMBOL    DATA     WORD      DataMin
      ---         BLOCKEND  ---      ---       LVL=1
      01000357H   LINE      CODE     ---       #340
      01000357H   LINE      CODE     ---       #341
      01000357H   LINE      CODE     ---       #347
      0100036BH   LINE      CODE     ---       #348
      0100036BH   LINE      CODE     ---       #352
      01000371H   LINE      CODE     ---       #353
      0100037AH   LINE      CODE     ---       #354
      0100037AH   LINE      CODE     ---       #355
      0100037FH   LINE      CODE     ---       #356
      0100037FH   LINE      CODE     ---       #357
      01000381H   LINE      CODE     ---       #358
      010003A0H   LINE      CODE     ---       #359
      010003A2H   LINE      CODE     ---       #361
      010003A7H   LINE      CODE     ---       #362
      010003ABH   LINE      CODE     ---       #363
      010003B1H   LINE      CODE     ---       #364
      010003B3H   LINE      CODE     ---       #365
      010003B3H   LINE      CODE     ---       #366
      010003CBH   LINE      CODE     ---       #368
      010003D4H   LINE      CODE     ---       #369
      010003D4H   LINE      CODE     ---       #370
      010003D8H   LINE      CODE     ---       #371
      010003D8H   LINE      CODE     ---       #372
LX51 LINKER/LOCATER V4.64.0.0                                                         04/13/2020  14:54:03  PAGE 48


      010003E1H   LINE      CODE     ---       #373
      010003E1H   LINE      CODE     ---       #374
      010003E5H   LINE      CODE     ---       #375
      010003E5H   LINE      CODE     ---       #377
      010003E9H   LINE      CODE     ---       #381
      0100040CH   LINE      CODE     ---       #384
      01000410H   LINE      CODE     ---       #385
      ---         BLOCKEND  ---      ---       LVL=0

      01000291H   BLOCK     CODE     ---       LVL=0
      01000291H   BLOCK     CODE     NEAR LAB  LVL=1
      00000015H   SYMBOL    DATA     BYTE      i
      00000007H   SYMBOL    DATA     BYTE      j
      00000021H   SYMBOL    DATA     BYTE      TS_ScanTimes
      ---         BLOCKEND  ---      ---       LVL=1
      01000291H   LINE      CODE     ---       #433
      01000291H   LINE      CODE     ---       #434
      01000291H   LINE      CODE     ---       #440
      01000297H   LINE      CODE     ---       #441
      01000297H   LINE      CODE     ---       #454
      01000299H   LINE      CODE     ---       #455
      0100029DH   LINE      CODE     ---       #456
      0100029FH   LINE      CODE     ---       #457
      010002A2H   LINE      CODE     ---       #463
      010002A8H   LINE      CODE     ---       #464
      010002ABH   LINE      CODE     ---       #466
      010002ACH   LINE      CODE     ---       #507
      010002B6H   LINE      CODE     ---       #508
      010002B6H   LINE      CODE     ---       #509
      010002BBH   LINE      CODE     ---       #510
      010002BBH   LINE      CODE     ---       #511
      010002BDH   LINE      CODE     ---       #512
      010002C5H   LINE      CODE     ---       #513
      010002C5H   LINE      CODE     ---       #515
      010002C5H   LINE      CODE     ---       #549
      010002C9H   LINE      CODE     ---       #550
      010002DAH   LINE      CODE     ---       #551
      010002DAH   LINE      CODE     ---       #552
      010002DCH   LINE      CODE     ---       #553
      010002DCH   LINE      CODE     ---       #554
      010002F9H   LINE      CODE     ---       #555
      010002FDH   LINE      CODE     ---       #556
      01000306H   LINE      CODE     ---       #561
      0100030DH   LINE      CODE     ---       #562
      01000318H   LINE      CODE     ---       #563
      01000320H   LINE      CODE     ---       #583
      01000344H   LINE      CODE     ---       #585
      0100034BH   LINE      CODE     ---       #589
      0100034FH   LINE      CODE     ---       #598
      01000352H   LINE      CODE     ---       #600
      01000356H   LINE      CODE     ---       #601
      01000356H   LINE      CODE     ---       #602
      01000356H   LINE      CODE     ---       #603
      ---         BLOCKEND  ---      ---       LVL=0

      0100018FH   BLOCK     CODE     ---       LVL=0
      0100018FH   BLOCK     CODE     NEAR LAB  LVL=1
      00000015H   SYMBOL    DATA     BYTE      i
      00000016H   SYMBOL    DATA     BYTE      TouchArea
      00000017H   SYMBOL    DATA     BYTE      NowArea
      ---         BLOCKEND  ---      ---       LVL=1
      0100018FH   LINE      CODE     ---       #707
      0100018FH   LINE      CODE     ---       #708
      0100018FH   LINE      CODE     ---       #715
      01000192H   LINE      CODE     ---       #716
LX51 LINKER/LOCATER V4.64.0.0                                                         04/13/2020  14:54:03  PAGE 49


      01000192H   LINE      CODE     ---       #728
      0100019AH   LINE      CODE     ---       #729
      010001A2H   LINE      CODE     ---       #731
      010001AEH   LINE      CODE     ---       #732
      010001AEH   LINE      CODE     ---       #733
      010001B0H   LINE      CODE     ---       #734
      010001B0H   LINE      CODE     ---       #741
      010001B4H   LINE      CODE     ---       #742
      010001B4H   LINE      CODE     ---       #743
      010001B8H   LINE      CODE     ---       #744
      010001B8H   LINE      CODE     ---       #745
      010001BDH   LINE      CODE     ---       #746
      010001BDH   LINE      CODE     ---       #747
      010001C5H   LINE      CODE     ---       #748
      010001C5H   LINE      CODE     ---       #749
      010001C8H   LINE      CODE     ---       #751
      010001CEH   LINE      CODE     ---       #753
      010001D4H   LINE      CODE     ---       #754
      010001D4H   LINE      CODE     ---       #755
      010001D6H   LINE      CODE     ---       #757
      010001D6H   LINE      CODE     ---       #764
      010001DCH   LINE      CODE     ---       #766
      010001E2H   LINE      CODE     ---       #767
      010001E2H   LINE      CODE     ---       #768
      010001EDH   LINE      CODE     ---       #769
      010001EDH   LINE      CODE     ---       #770
      010001EDH   LINE      CODE     ---       #774
      010001EDH   LINE      CODE     ---       #779
      010001EDH   LINE      CODE     ---       #781
      010001EDH   LINE      CODE     ---       #782
      010001EFH   LINE      CODE     ---       #784
      010001EFH   LINE      CODE     ---       #785
      010001F4H   LINE      CODE     ---       #786
      010001F4H   LINE      CODE     ---       #787
      010001FAH   LINE      CODE     ---       #788
      010001FAH   LINE      CODE     ---       #793
      010001FEH   LINE      CODE     ---       #795
      010001FEH   LINE      CODE     ---       #796
      010001FEH   LINE      CODE     ---       #800
      010001FEH   LINE      CODE     ---       #801
      01000200H   LINE      CODE     ---       #809
      01000200H   LINE      CODE     ---       #811
      01000200H   LINE      CODE     ---       #812
      01000204H   LINE      CODE     ---       #813
      01000204H   LINE      CODE     ---       #814
      01000207H   LINE      CODE     ---       #815
      01000209H   LINE      CODE     ---       #816
      0100020BH   LINE      CODE     ---       #817
      0100020BH   LINE      CODE     ---       #818
      0100020BH   LINE      CODE     ---       #819
      01000210H   LINE      CODE     ---       #820
      01000210H   LINE      CODE     ---       #821
      01000216H   LINE      CODE     ---       #822
      01000218H   LINE      CODE     ---       #823
      0100021AH   LINE      CODE     ---       #824
      0100021AH   LINE      CODE     ---       #825
      01000234H   LINE      CODE     ---       #826
      01000234H   LINE      CODE     ---       #827
      0100023AH   LINE      CODE     ---       #828
      0100023AH   LINE      CODE     ---       #829
      0100023DH   LINE      CODE     ---       #830
      01000249H   LINE      CODE     ---       #835
      0100024BH   LINE      CODE     ---       #836
      0100024BH   LINE      CODE     ---       #837
      0100024DH   LINE      CODE     ---       #839
LX51 LINKER/LOCATER V4.64.0.0                                                         04/13/2020  14:54:03  PAGE 50


      0100024DH   LINE      CODE     ---       #840
      01000250H   LINE      CODE     ---       #841
      01000257H   LINE      CODE     ---       #842
      01000257H   LINE      CODE     ---       #843
      01000262H   LINE      CODE     ---       #917
      01000269H   LINE      CODE     ---       #920
      0100026BH   LINE      CODE     ---       #921
      0100026BH   LINE      CODE     ---       #922
      0100026EH   LINE      CODE     ---       #923
      0100026FH   LINE      CODE     ---       #925
      0100026FH   LINE      CODE     ---       #926
      01000272H   LINE      CODE     ---       #927
      01000272H   LINE      CODE     ---       #928
      ---         BLOCKEND  ---      ---       LVL=0

      01000670H   BLOCK     CODE     ---       LVL=0
      01000670H   BLOCK     CODE     NEAR LAB  LVL=1
      00000006H   SYMBOL    DATA     BYTE      i
      00000007H   SYMBOL    DATA     BYTE      ch_idx
      ---         BLOCKEND  ---      ---       LVL=1
      01000670H   LINE      CODE     ---       #1147
      01000670H   LINE      CODE     ---       #1148
      01000670H   LINE      CODE     ---       #1151
      01000673H   LINE      CODE     ---       #1156
      01000677H   LINE      CODE     ---       #1157
      01000679H   LINE      CODE     ---       #1158
      0100067AH   LINE      CODE     ---       #1159
      0100067AH   LINE      CODE     ---       #1170
      01000695H   LINE      CODE     ---       #1174
      01000699H   LINE      CODE     ---       #1177
      010006A0H   LINE      CODE     ---       #1178
      010006A7H   LINE      CODE     ---       #1184
      010006AAH   LINE      CODE     ---       #1185
      010006ADH   LINE      CODE     ---       #1187
      010006AFH   LINE      CODE     ---       #1189
      010006B2H   LINE      CODE     ---       #1192
      010006B5H   LINE      CODE     ---       #1197
      010006B8H   LINE      CODE     ---       #1198
      010006BEH   LINE      CODE     ---       #1246
      010006C0H   LINE      CODE     ---       #1248
      010006C2H   LINE      CODE     ---       #1250
      010006C7H   LINE      CODE     ---       #1251
      010006CAH   LINE      CODE     ---       #1253
      010006CCH   LINE      CODE     ---       #1272
      010006CFH   LINE      CODE     ---       #1273
      010006D3H   LINE      CODE     ---       #1279
      010006D5H   LINE      CODE     ---       #1280
      010006D9H   LINE      CODE     ---       #1283
      ---         BLOCKEND  ---      ---       LVL=0

      01000889H   BLOCK     CODE     ---       LVL=0
      01000889H   LINE      CODE     ---       #1285
      01000889H   LINE      CODE     ---       #1286
      01000889H   LINE      CODE     ---       #1287
      01000892H   LINE      CODE     ---       #1288
      01000892H   LINE      CODE     ---       #1289
      01000892H   LINE      CODE     ---       #1290
      01000895H   LINE      CODE     ---       #1291
      01000897H   LINE      CODE     ---       #1292
      01000897H   LINE      CODE     ---       #1293
      0100089AH   LINE      CODE     ---       #1294
      0100089AH   LINE      CODE     ---       #1295
      0100089CH   LINE      CODE     ---       #1301
      0100089FH   LINE      CODE     ---       #1302
      010008A1H   LINE      CODE     ---       #1304
LX51 LINKER/LOCATER V4.64.0.0                                                         04/13/2020  14:54:03  PAGE 51


      010008A7H   LINE      CODE     ---       #1305
      010008A7H   LINE      CODE     ---       #1306
      010008AAH   LINE      CODE     ---       #1307
      010008AAH   LINE      CODE     ---       #1310
      010008ADH   LINE      CODE     ---       #1346
      010008ADH   LINE      CODE     ---       #1347
      010008B6H   LINE      CODE     ---       #1348
      010008B6H   LINE      CODE     ---       #1349
      010008B9H   LINE      CODE     ---       #1350
      010008BCH   LINE      CODE     ---       #1351
      010008BFH   LINE      CODE     ---       #1352
      010008BFH   LINE      CODE     ---       #1353
      010008BFH   LINE      CODE     ---       #1354
      010008BFH   LINE      CODE     ---       #1355
      010008BFH   LINE      CODE     ---       #1356
      010008BFH   LINE      CODE     ---       #1363
      ---         BLOCKEND  ---      ---       LVL=0

      01000572H   BLOCK     CODE     ---       LVL=0
      01000572H   BLOCK     CODE     NEAR LAB  LVL=1
      00000022H   SYMBOL    DATA     WORD      KeyBak
      00000020H.0 SYMBOL    BIT      BIT       LongFlag
      00000024H   SYMBOL    DATA     BYTE      KeyidxBak
      00000007H   SYMBOL    DATA     BYTE      i
      ---         BLOCKEND  ---      ---       LVL=1
      01000572H   LINE      CODE     ---       #1607
      01000572H   LINE      CODE     ---       #1608
      01000572H   LINE      CODE     ---       #1618
      01000577H   LINE      CODE     ---       #1619
      0100057BH   LINE      CODE     ---       #1620
      0100057BH   LINE      CODE     ---       #1639
      01000581H   LINE      CODE     ---       #1640
      01000581H   LINE      CODE     ---       #1641
      01000583H   LINE      CODE     ---       #1642
      01000583H   LINE      CODE     ---       #1643
      01000590H   LINE      CODE     ---       #1644
      01000590H   LINE      CODE     ---       #1645
      01000592H   LINE      CODE     ---       #1646
      0100059CH   LINE      CODE     ---       #1647
      0100059EH   LINE      CODE     ---       #1648
      0100059EH   LINE      CODE     ---       #1649
      010005A2H   LINE      CODE     ---       #1650
      010005A8H   LINE      CODE     ---       #1651
      010005AAH   LINE      CODE     ---       #1652
      010005B0H   LINE      CODE     ---       #1653
      010005B3H   LINE      CODE     ---       #1654
      010005B3H   LINE      CODE     ---       #1656
      010005B4H   LINE      CODE     ---       #1657
      010005BAH   LINE      CODE     ---       #1658
      010005BAH   LINE      CODE     ---       #1712
      010005C8H   LINE      CODE     ---       #1713
      010005C8H   LINE      CODE     ---       #1714
      010005CEH   LINE      CODE     ---       #1715
      010005CEH   LINE      CODE     ---       #1716
      010005D1H   LINE      CODE     ---       #1717
      010005D1H   LINE      CODE     ---       #1718
      010005D3H   LINE      CODE     ---       #1719
      010005D7H   LINE      CODE     ---       #1720
      010005D9H   LINE      CODE     ---       #1722
      010005D9H   LINE      CODE     ---       #1723
      010005E2H   LINE      CODE     ---       #1724
      010005E2H   LINE      CODE     ---       #1725
      010005E8H   LINE      CODE     ---       #1726
      010005E8H   LINE      CODE     ---       #1727
      010005E9H   LINE      CODE     ---       #1729
LX51 LINKER/LOCATER V4.64.0.0                                                         04/13/2020  14:54:03  PAGE 52


      010005E9H   LINE      CODE     ---       #1730
      010005EEH   LINE      CODE     ---       #1731
      010005EEH   LINE      CODE     ---       #1732
      010005F0H   LINE      CODE     ---       #1733
      010005F2H   LINE      CODE     ---       #1735
      010005F2H   LINE      CODE     ---       #1736
      010005F9H   LINE      CODE     ---       #1737
      010005F9H   LINE      CODE     ---       #1738
      010005FCH   LINE      CODE     ---       #1739
      010005FCH   LINE      CODE     ---       #1741
      010005FCH   LINE      CODE     ---       #1851
      ---         BLOCKEND  ---      ---       LVL=0

      ---         MODULE    ---      ---       TS_SEVICE
      01000CACH   PUBLIC    CONST    ---       pXSFR
      010007E8H   PUBLIC    CODE     ---       _TS_AreaConfirmTimerSet
      0100091FH   PUBLIC    CODE     ---       _TS_AreaDeviateDetection
      00000020H.4 PUBLIC    BIT      BIT       ?_TS_GetDataArea?BIT
      010006DAH   PUBLIC    CODE     ---       _TS_GetDataArea
      01000800H   PUBLIC    CODE     ---       TS_ScanStart
      010008C2H   PUBLIC    CODE     ---       TS_IO_init
      000000E3H   SFRSYM    DATA     BYTE      LXDAT
      000000C4H   SFRSYM    DATA     BYTE      TKCHS
      00000080H   SFRSYM    DATA     BYTE      P0
      000000C1H   SFRSYM    DATA     BYTE      TKCON
      00000090H   SFRSYM    DATA     BYTE      P1
      000000A0H   SFRSYM    DATA     BYTE      P2
      000000B0H   SFRSYM    DATA     BYTE      P3
      000000D0H.6 SFRSYM    DATA     BIT       AC
      000000C0H   SFRSYM    DATA     BYTE      P4
      000000D8H   SFRSYM    DATA     BYTE      P5
      000000A5H   SFRSYM    DATA     BYTE      SPCON
      000000A8H.7 SFRSYM    DATA     BIT       EA
      000000E1H   SFRSYM    DATA     BYTE      LXCON
      000000A9H   SFRSYM    DATA     BYTE      P6
      000000C8H   SFRSYM    DATA     BIT       T2P0
      000000D9H   SFRSYM    DATA     BYTE      P7
      000000C8H.1 SFRSYM    DATA     BIT       T2P1
      000000F1H   SFRSYM    DATA     BYTE      RTCON
      000000C8H.4 SFRSYM    DATA     BIT       T2R0
      000000DAH   SFRSYM    DATA     BYTE      PWMEN
      000000CFH   SFRSYM    DATA     BYTE      TKMSH
      00000086H   SFRSYM    DATA     BYTE      PWCON
      000000C8H.5 SFRSYM    DATA     BIT       T2R1
      000000CEH   SFRSYM    DATA     BYTE      TKMSL
      000000A7H   SFRSYM    DATA     BYTE      SPSTA
      00000083H   SFRSYM    DATA     BYTE      DP0H
      000000A8H   SFRSYM    DATA     BYTE      IE
      00000085H   SFRSYM    DATA     BYTE      DP1H
      000000E9H   SFRSYM    DATA     BYTE      RTCSS
      00000082H   SFRSYM    DATA     BYTE      DP0L
      000000CBH   SFRSYM    DATA     BYTE      T2CH
      000000B3H   SFRSYM    DATA     BYTE      I2CADM
      00000084H   SFRSYM    DATA     BYTE      DP1L
      000000C8H.3 SFRSYM    DATA     BIT       T2IE
      000000C3H   SFRSYM    DATA     BYTE      TKMTS
      000000CAH   SFRSYM    DATA     BYTE      T2CL
      000000B2H   SFRSYM    DATA     BYTE      I2CADR
      000000B4H   SFRSYM    DATA     BYTE      I2CCCR
      000000B8H   SFRSYM    DATA     BYTE      IP
      000000B7H   SFRSYM    DATA     BYTE      I2CFLG
      000000B5H   SFRSYM    DATA     BYTE      I2CDAT
      000000EDH   SFRSYM    DATA     BYTE      RTMSS
      000000D0H.7 SFRSYM    DATA     BIT       CY
      000000BBH   SFRSYM    DATA     BYTE      ADCFGH
LX51 LINKER/LOCATER V4.64.0.0                                                         04/13/2020  14:54:03  PAGE 53


      000000DCH   SFRSYM    DATA     BYTE      PWMCMAX
      000000B1H   SFRSYM    DATA     BYTE      I2CCON
      000000D1H   SFRSYM    DATA     BYTE      PWMDIVH
      000000BAH   SFRSYM    DATA     BYTE      ADCFGL
      00000081H   SFRSYM    DATA     BYTE      SP
      000000F9H   SFRSYM    DATA     BYTE      EPIE
      000000D0H.2 SFRSYM    DATA     BIT       OV
      000000FAH   SFRSYM    DATA     BYTE      EPIF
      000000DFH   SFRSYM    DATA     BYTE      PWMDIVL
      000000B6H   SFRSYM    DATA     BYTE      I2CSTA
      000000E8H   SFRSYM    DATA     BYTE      EXIE
      000000D3H   SFRSYM    DATA     BYTE      PWMDUTH
      000000C7H   SFRSYM    DATA     BYTE      TKIF
      0000008FH   SFRSYM    DATA     BYTE      IT0CON
      00000080H   SFRSYM    DATA     BIT       P00
      000000ECH   SFRSYM    DATA     BYTE      RTAH
      000000D2H   SFRSYM    DATA     BYTE      PWMDUTL
      0000008EH   SFRSYM    DATA     BYTE      IT1CON
      00000090H   SFRSYM    DATA     BIT       P10
      00000080H.1 SFRSYM    DATA     BIT       P01
      0000009DH   SFRSYM    DATA     BYTE      S1RELH
      00000087H   SFRSYM    DATA     BYTE      PCON
      000000A0H   SFRSYM    DATA     BIT       P20
      00000090H.1 SFRSYM    DATA     BIT       P11
      00000080H.2 SFRSYM    DATA     BIT       P02
      000000E8H   SFRSYM    DATA     BIT       INT2EN
      000000F4H   SFRSYM    DATA     BYTE      RTCH
      000000A4H   SFRSYM    DATA     BYTE      S2RELH
      000000B0H   SFRSYM    DATA     BIT       P30
      000000A0H.1 SFRSYM    DATA     BIT       P21
      00000090H.2 SFRSYM    DATA     BIT       P12
      00000080H.3 SFRSYM    DATA     BIT       P03
      000000E8H.1 SFRSYM    DATA     BIT       INT3EN
      000000C0H   SFRSYM    DATA     BIT       P40
      000000B0H.1 SFRSYM    DATA     BIT       P31
      000000A0H.2 SFRSYM    DATA     BIT       P22
      00000090H.3 SFRSYM    DATA     BIT       P13
      00000080H.4 SFRSYM    DATA     BIT       P04
      000000E8H.2 SFRSYM    DATA     BIT       INT4EN
      000000D8H   SFRSYM    DATA     BIT       P50
      000000C0H.1 SFRSYM    DATA     BIT       P41
      000000B0H.2 SFRSYM    DATA     BIT       P32
      000000A0H.3 SFRSYM    DATA     BIT       P23
      00000090H.4 SFRSYM    DATA     BIT       P14
      00000080H.5 SFRSYM    DATA     BIT       P05
      000000E8H.3 SFRSYM    DATA     BIT       INT5EN
      000000EBH   SFRSYM    DATA     BYTE      RTAM
      0000009CH   SFRSYM    DATA     BYTE      S1RELL
      00000089H   SFRSYM    DATA     BYTE      TMOD
      00000088H   SFRSYM    DATA     BYTE      TCON
      000000D8H.1 SFRSYM    DATA     BIT       P51
      000000C0H.2 SFRSYM    DATA     BIT       P42
      000000B0H.3 SFRSYM    DATA     BIT       P33
      000000A0H.4 SFRSYM    DATA     BIT       P24
      00000090H.5 SFRSYM    DATA     BIT       P15
      00000080H.6 SFRSYM    DATA     BIT       P06
      000000E8H.4 SFRSYM    DATA     BIT       INT6EN
      000000A3H   SFRSYM    DATA     BYTE      S2RELL
      000000D8H.2 SFRSYM    DATA     BIT       P52
      000000C0H.3 SFRSYM    DATA     BIT       P43
      000000B0H.4 SFRSYM    DATA     BIT       P34
      000000A0H.5 SFRSYM    DATA     BIT       P25
      00000090H.6 SFRSYM    DATA     BIT       P16
      00000080H.7 SFRSYM    DATA     BIT       P07
      000000E8H.5 SFRSYM    DATA     BIT       INT7EN
LX51 LINKER/LOCATER V4.64.0.0                                                         04/13/2020  14:54:03  PAGE 54


      000000C8H.2 SFRSYM    DATA     BIT       UCKS
      000000F8H   SFRSYM    DATA     BYTE      EXIP
      000000F3H   SFRSYM    DATA     BYTE      RTCM
      000000D8H.3 SFRSYM    DATA     BIT       P53
      000000C0H.4 SFRSYM    DATA     BIT       P44
      000000B0H.5 SFRSYM    DATA     BIT       P35
      000000A0H.6 SFRSYM    DATA     BIT       P26
      00000090H.7 SFRSYM    DATA     BIT       P17
      000000E8H.6 SFRSYM    DATA     BIT       INT8EN
      000000D8H.4 SFRSYM    DATA     BIT       P54
      000000C0H.5 SFRSYM    DATA     BIT       P45
      000000B0H.6 SFRSYM    DATA     BIT       P36
      000000A0H.7 SFRSYM    DATA     BIT       P27
      000000E8H.7 SFRSYM    DATA     BIT       INT9EN
      000000D8H.5 SFRSYM    DATA     BIT       P55
      000000C0H.6 SFRSYM    DATA     BIT       P46
      000000B0H.7 SFRSYM    DATA     BIT       P37
      000000D8H.6 SFRSYM    DATA     BIT       P56
      000000C0H.7 SFRSYM    DATA     BIT       P47
      000000EAH   SFRSYM    DATA     BYTE      RTAS
      000000AFH   SFRSYM    DATA     BYTE      HVTH
      00000095H   SFRSYM    DATA     BYTE      RCTAGH
      000000D8H.7 SFRSYM    DATA     BIT       P57
      000000F2H   SFRSYM    DATA     BYTE      RTCS
      00000088H.1 SFRSYM    DATA     BIT       IE0
      00000088H.3 SFRSYM    DATA     BIT       IE1
      00000094H   SFRSYM    DATA     BYTE      RCTAGL
      000000F0H   SFRSYM    DATA     BYTE      B
      000000E7H   SFRSYM    DATA     BYTE      MDUDAT
      000000DEH   SFRSYM    DATA     BYTE      PWMCFG
      000000D4H   SFRSYM    DATA     BYTE      PWMAIF
      000000E0H   SFRSYM    DATA     BYTE      ACC
      000000D5H   SFRSYM    DATA     BYTE      PWMBIF
      0000009FH   SFRSYM    DATA     BYTE      RCMSHH
      000000A8H.4 SFRSYM    DATA     BIT       ES0
      000000EFH   SFRSYM    DATA     BYTE      LVDCON
      000000E6H   SFRSYM    DATA     BYTE      MDUCON
      000000D6H   SFRSYM    DATA     BYTE      PWMCIF
      000000A8H.1 SFRSYM    DATA     BIT       ET0
      000000A8H.6 SFRSYM    DATA     BIT       ES1
      000000D7H   SFRSYM    DATA     BYTE      PWMDIF
      000000A8H.3 SFRSYM    DATA     BIT       ET1
      00000088H.5 SFRSYM    DATA     BIT       TF0
      000000FDH   SFRSYM    DATA     BYTE      IDLSTH
      000000AEH   SFRSYM    DATA     BYTE      PLLCON
      000000A8H.5 SFRSYM    DATA     BIT       ET2
      00000098H   SFRSYM    DATA     BIT       RI0
      00000088H.7 SFRSYM    DATA     BIT       TF1
      0000009EH   SFRSYM    DATA     BYTE      RCMSHL
      00000097H   SFRSYM    DATA     BYTE      RCMSLH
      000000C8H.7 SFRSYM    DATA     BIT       TF2
      00000098H.2 SFRSYM    DATA     BIT       RB8
      0000008CH   SFRSYM    DATA     BYTE      TH0
      000000A8H   SFRSYM    DATA     BIT       EX0
      00000098H.1 SFRSYM    DATA     BIT       TI0
      00000088H   SFRSYM    DATA     BIT       IT0
      0000008DH   SFRSYM    DATA     BYTE      TH1
      000000A8H.2 SFRSYM    DATA     BIT       EX1
      00000098H.3 SFRSYM    DATA     BIT       TB8
      00000088H.2 SFRSYM    DATA     BIT       IT1
      000000FCH   SFRSYM    DATA     BYTE      IDLSTL
      000000CDH   SFRSYM    DATA     BYTE      TH2
      000000D0H   SFRSYM    DATA     BIT       P
      00000096H   SFRSYM    DATA     BYTE      RCMSLL
      00000098H.7 SFRSYM    DATA     BIT       SM0
LX51 LINKER/LOCATER V4.64.0.0                                                         04/13/2020  14:54:03  PAGE 55


      0000008AH   SFRSYM    DATA     BYTE      TL0
      00000098H.6 SFRSYM    DATA     BIT       SM1
      000000E5H   SFRSYM    DATA     BYTE      LXDIVH
      0000008BH   SFRSYM    DATA     BYTE      TL1
      00000098H.5 SFRSYM    DATA     BIT       SM2
      000000CCH   SFRSYM    DATA     BYTE      TL2
      000000B8H.4 SFRSYM    DATA     BIT       PS0
      000000B8H.1 SFRSYM    DATA     BIT       PT0
      000000B8H.6 SFRSYM    DATA     BIT       PS1
      000000B8H.3 SFRSYM    DATA     BIT       PT1
      000000D0H.3 SFRSYM    DATA     BIT       RS0
      000000E4H   SFRSYM    DATA     BYTE      LXDIVL
      000000BDH   SFRSYM    DATA     BYTE      ADCDH
      000000B8H.5 SFRSYM    DATA     BIT       PT2
      00000088H.4 SFRSYM    DATA     BIT       TR0
      000000D0H.4 SFRSYM    DATA     BIT       RS1
      000000DDH   SFRSYM    DATA     BYTE      PWMCON
      00000088H.6 SFRSYM    DATA     BIT       TR1
      000000ADH   SFRSYM    DATA     BYTE      WDVTHH
      000000C8H.6 SFRSYM    DATA     BIT       TR2
      000000B8H   SFRSYM    DATA     BIT       PX0
      000000B8H.2 SFRSYM    DATA     BIT       PX1
      000000BCH   SFRSYM    DATA     BYTE      ADCDL
      000000ACH   SFRSYM    DATA     BYTE      WDVTHL
      000000DBH   SFRSYM    DATA     BYTE      PWMUPD
      00000099H   SFRSYM    DATA     BYTE      S0BUF
      0000009BH   SFRSYM    DATA     BYTE      S1BUF
      000000A2H   SFRSYM    DATA     BYTE      S2BUF
      00000098H   SFRSYM    DATA     BYTE      S0CON
      00000098H.4 SFRSYM    DATA     BIT       REN
      0000009AH   SFRSYM    DATA     BYTE      S1CON
      000000B9H   SFRSYM    DATA     BYTE      ADCON
      000000A1H   SFRSYM    DATA     BYTE      S2CON
      000000D0H.1 SFRSYM    DATA     BIT       DPS
      000000C9H   SFRSYM    DATA     BYTE      T2MOD
      000000C8H   SFRSYM    DATA     BYTE      T2CON
      000000FFH   SFRSYM    DATA     BYTE      STPSTH
      000000BFH   SFRSYM    DATA     BYTE      CKMIF
      000000FEH   SFRSYM    DATA     BYTE      STPSTL
      000000C2H   SFRSYM    DATA     BYTE      TKCFG
      00000093H   SFRSYM    DATA     BYTE      VCKDH
      000000D0H.5 SFRSYM    DATA     BIT       F0
      000000E2H   SFRSYM    DATA     BYTE      LXCFG
      000000ABH   SFRSYM    DATA     BYTE      WDFLG
      00000092H   SFRSYM    DATA     BYTE      VCKDL
      000000FBH   SFRSYM    DATA     BYTE      EPCON
      000000F6H   SFRSYM    DATA     BYTE      RTCDH
      000000C6H   SFRSYM    DATA     BYTE      ATKMH
      00000091H   SFRSYM    DATA     BYTE      RCCON
      000000F7H   SFRSYM    DATA     BYTE      INDEX
      000000EEH   SFRSYM    DATA     BYTE      RTCIF
      000000BEH   SFRSYM    DATA     BYTE      CKMON
      000000F5H   SFRSYM    DATA     BYTE      RTCDL
      000000D0H   SFRSYM    DATA     BYTE      PSW
      000000C5H   SFRSYM    DATA     BYTE      ATKML
      000000AAH   SFRSYM    DATA     BYTE      WDCON
      000000A6H   SFRSYM    DATA     BYTE      SPDAT

      0100006EH   BLOCK     CODE     ---       LVL=0
      ---         BLOCKEND  ---      ---       LVL=0

      010008C2H   BLOCK     CODE     ---       LVL=0
      010008C2H   BLOCK     CODE     NEAR LAB  LVL=1
      00000007H   SYMBOL    DATA     BYTE      i
      00000001H   SYMBOL    DATA     ---       pPinS
LX51 LINKER/LOCATER V4.64.0.0                                                         04/13/2020  14:54:03  PAGE 56


      ---         BLOCKEND  ---      ---       LVL=1
      010008C2H   LINE      CODE     ---       #41
      010008C2H   LINE      CODE     ---       #42
      010008C2H   LINE      CODE     ---       #45
      010008C8H   LINE      CODE     ---       #46
      010008D3H   LINE      CODE     ---       #47
      010008D3H   LINE      CODE     ---       #48
      010008E8H   LINE      CODE     ---       #49
      010008EDH   LINE      CODE     ---       #50
      010008F0H   LINE      CODE     ---       #51
      ---         BLOCKEND  ---      ---       LVL=0

      01000800H   BLOCK     CODE     ---       LVL=0
      01000800H   BLOCK     CODE     NEAR LAB  LVL=1
      00000007H   SYMBOL    DATA     BYTE      i
      00000006H   SYMBOL    DATA     BYTE      j
      ---         BLOCKEND  ---      ---       LVL=1
      01000800H   LINE      CODE     ---       #52
      01000800H   LINE      CODE     ---       #53
      01000800H   LINE      CODE     ---       #55
      01000808H   LINE      CODE     ---       #56
      01000808H   LINE      CODE     ---       #57
      0100081FH   LINE      CODE     ---       #58
      0100081FH   LINE      CODE     ---       #59
      01000821H   LINE      CODE     ---       #60
      01000824H   LINE      CODE     ---       #61
      0100082DH   LINE      CODE     ---       #62
      0100082DH   LINE      CODE     ---       #63
      0100082FH   LINE      CODE     ---       #64
      01000832H   LINE      CODE     ---       #65
      01000835H   LINE      CODE     ---       #66
      01000835H   LINE      CODE     ---       #67
      01000835H   LINE      CODE     ---       #68
      01000837H   LINE      CODE     ---       #69
      01000843H   LINE      CODE     ---       #70
      01000846H   LINE      CODE     ---       #71
      01000849H   LINE      CODE     ---       #72
      ---         BLOCKEND  ---      ---       LVL=0

      010006DAH   BLOCK     CODE     ---       LVL=0
      00000001H   SYMBOL    DATA     BYTE      ts_ch
      00000004H   SYMBOL    DATA     WORD      ts_data
      00000018H   SYMBOL    DATA     INT       NoiseThd
      00000020H.4 SYMBOL    BIT      BIT       key_pressed_flag
      010006E0H   BLOCK     CODE     NEAR LAB  LVL=1
      00000002H   SYMBOL    DATA     INT       Delta
      00000006H   SYMBOL    DATA     INT       FingerThd
      ---         BLOCKEND  ---      ---       LVL=1
      010006DAH   LINE      CODE     ---       #73
      010006E0H   LINE      CODE     ---       #74
      010006E0H   LINE      CODE     ---       #78
      010006F0H   LINE      CODE     ---       #79
      010006F7H   LINE      CODE     ---       #81
      010006FAH   LINE      CODE     ---       #82
      010006FAH   LINE      CODE     ---       #83
      01000705H   LINE      CODE     ---       #84
      01000705H   LINE      CODE     ---       #86
      0100070DH   LINE      CODE     ---       #87
      0100071BH   LINE      CODE     ---       #88
      01000726H   LINE      CODE     ---       #89
      01000738H   LINE      CODE     ---       #90
      01000738H   LINE      CODE     ---       #91
      ---         BLOCKEND  ---      ---       LVL=0

      0100091FH   BLOCK     CODE     ---       LVL=0
LX51 LINKER/LOCATER V4.64.0.0                                                         04/13/2020  14:54:03  PAGE 57


      00000006H   SYMBOL    DATA     WORD      cmp_data
      00000004H   SYMBOL    DATA     WORD      real_data
      00000002H   SYMBOL    DATA     INT       range
      0100091FH   BLOCK     CODE     NEAR LAB  LVL=1
      00000006H   SYMBOL    DATA     INT       Delta
      ---         BLOCKEND  ---      ---       LVL=1
      0100091FH   LINE      CODE     ---       #92
      0100091FH   LINE      CODE     ---       #93
      0100091FH   LINE      CODE     ---       #95
      01000926H   LINE      CODE     ---       #96
      01000947H   LINE      CODE     ---       #97
      01000947H   LINE      CODE     ---       #98
      0100094AH   LINE      CODE     ---       #99
      0100094AH   LINE      CODE     ---       #101
      0100094AH   LINE      CODE     ---       #102
      0100094CH   LINE      CODE     ---       #103
      0100094CH   LINE      CODE     ---       #104
      ---         BLOCKEND  ---      ---       LVL=0

      010007E8H   BLOCK     CODE     ---       LVL=0
      00000007H   SYMBOL    DATA     BYTE      ts_ch
      00000005H   SYMBOL    DATA     BYTE      area
      010007E8H   LINE      CODE     ---       #117
      010007E8H   LINE      CODE     ---       #118
      010007E8H   LINE      CODE     ---       #119
      010007FAH   LINE      CODE     ---       #120
      ---         BLOCKEND  ---      ---       LVL=0
      00000001H   SYMBOL    DATA     BYTE      Slider_Cnt
      00000007H   SYMBOL    DATA     BYTE      i
      00000006H   SYMBOL    DATA     BYTE      j
      00000006H   SYMBOL    DATA     WORD      CalcTemp3
      00000005H   SYMBOL    DATA     BYTE      DeltaRate
      00000004H   SYMBOL    DATA     INT       PosOffset
      00000006H   SYMBOL    DATA     WORD      CalcTemp3
      00000005H   SYMBOL    DATA     BYTE      DeltaRate
      00000006H   SYMBOL    DATA     INT       PosOffset

      ---         MODULE    ---      ---       ?C_STARTUP
      01000000H   PUBLIC    CODE     ---       ?C_STARTUP
      000000E0H   SYMBOL    DATA     ---       ACC
      000000F0H   SYMBOL    DATA     ---       B
      00000083H   SYMBOL    DATA     ---       DPH
      00000082H   SYMBOL    DATA     ---       DPL
      00000000H   SYMBOL    NUMBER   ---       IBPSTACK
      00000100H   SYMBOL    NUMBER   ---       IBPSTACKTOP
      00000080H   SYMBOL    NUMBER   ---       IDATALEN
      01000C17H   SYMBOL    CODE     ---       IDATALOOP
      00000000H   SYMBOL    NUMBER   ---       PBPSTACK
      00000100H   SYMBOL    NUMBER   ---       PBPSTACKTOP
      00000000H   SYMBOL    NUMBER   ---       PDATALEN
      00000000H   SYMBOL    NUMBER   ---       PDATASTART
      00000000H   SYMBOL    NUMBER   ---       PPAGE
      00000000H   SYMBOL    NUMBER   ---       PPAGEENABLE
      000000A0H   SYMBOL    DATA     ---       PPAGE_SFR
      00000081H   SYMBOL    DATA     ---       SP
      01000C14H   SYMBOL    CODE     ---       STARTUP1
      00000000H   SYMBOL    NUMBER   ---       XBPSTACK
      00000000H   SYMBOL    NUMBER   ---       XBPSTACKTOP
      00000000H   SYMBOL    NUMBER   ---       XDATALEN
      00000000H   SYMBOL    NUMBER   ---       XDATASTART
      01000000H   LINE      CODE     ---       #126
      01000C14H   LINE      CODE     ---       #133
      01000C16H   LINE      CODE     ---       #134
      01000C17H   LINE      CODE     ---       #135
      01000C18H   LINE      CODE     ---       #136
LX51 LINKER/LOCATER V4.64.0.0                                                         04/13/2020  14:54:03  PAGE 58


      01000C1AH   LINE      CODE     ---       #185
      01000C1DH   LINE      CODE     ---       #196

      ---         MODULE    ---      ---       ?C_INIT
      01000C5BH   PUBLIC    CODE     ---       ?C_START

      ---         MODULE    ---      ---       ?C?CLDOPTR
      010009E1H   PUBLIC    CODE     ---       ?C?CLDOPTR

      ---         MODULE    ---      ---       ?C?CSTPTR
      01000A0EH   PUBLIC    CODE     ---       ?C?CSTPTR

      ---         MODULE    ---      ---       ?C?CSTOPTR
      01000A20H   PUBLIC    CODE     ---       ?C?CSTOPTR

      ---         MODULE    ---      ---       ?C?IMUL
      01000A42H   PUBLIC    CODE     ---       ?C?IMUL

      ---         MODULE    ---      ---       ?C?UIDIV
      01000A54H   PUBLIC    CODE     ---       ?C?UIDIV

      ---         MODULE    ---      ---       ?C?SIDIV
      01000AA9H   PUBLIC    CODE     ---       ?C?SIDIV

      ---         MODULE    ---      ---       ?C?IILDX
      01000ADFH   PUBLIC    CODE     ---       ?C?IILDX

      ---         MODULE    ---      ---       ?C?ULDIV
      01000B31H   PUBLIC    CODE     ---       ?C?ULDIV

      ---         MODULE    ---      ---       ?C?LSTXDATA
      01000BC3H   PUBLIC    CODE     ---       ?C?LSTXDATA

      ---         MODULE    ---      ---       ?C?OFFXADD
      01000BCFH   PUBLIC    CODE     ---       ?C?OFFXADD

      ---         MODULE    ---      ---       ?C?PLDCODE
      01000BDBH   PUBLIC    CODE     ---       ?C?PLDCODE

      ---         MODULE    ---      ---       ?C?LIMUL
      01000BE7H   PUBLIC    CODE     ---       ?C?LIMUL

Program Size: data=56.5 xdata=397 const=162 code=3236
LX51 RUN COMPLETE.  0 WARNING(S),  0 ERROR(S)
